:109B7500414952434F544543004256332E35302018
:109B850048554E00414B4B5500532F4E21464149F8
:109B95004C555245005245454E54455221532F4E82
:109BA50000434F4E5441435420414952434F54457D
:109BB5004300475053004032444000403344400086
:109BC5004B492021554A20404D454E75000A160047
:109BD5000180000300007E0000FE00001E0000362C
:109BE5000003E60001C4000000000FFFE0534154EC
:109BF5005320404B4552455300414C544940434145
:109C05004C202023004B455045524E596F00534F71
:109C15005252454E44005445524B45502020005465
:109C250045524D494B202000564152494F20202096
:109C3500004241524F4752414D005554564E414CFA
:109C45002020004B6F5A454C4920200046504F4E6E
:109C5500544B2020004A454C454B20202000414CC8
:109C65004150202020002020202141544C2120203B
:109C750020205441560020545241434B2142452057
:109C8500200020545241434B214B492020004D4197
:109C9500524B004952414E592D46454E54004553AD
:109CA5005A414B2D46454E5400214B494C455020B9
:109CB50020015554564F4E4056414C014D414720C9
:109CC5004245414C4C2001524550754C45534B681B
:109CD5006901464C4947485420414C4C0146504F78
:109CE5004E544F4B206869015554564F4E414C4BCD
:109CF5006869014C45475445522020686901424531
:109D0500414C4C4954206869004D4147204245412A
:109D15004C4C20004241524F404D414720200047C6
:109D25005053204D4147202000514E4820202020EF
:109D3500402148504100464C005245504E41504C40
:109D45004F207552455320003E214B494C4550202C
:109D55002000214B494C455001564A4154535A0164
:109D65004B554C44202001544F524F4C2000214B61
:109D7500494C4550202001434F4D3A2020202020BA
:109D85002001544E432031232035374B01544E4397
:109D950020312320392E36010150574340313023DD
:109DA5004035374B01505743403130234031394B13
:109DB50001014D5850403130234035374B014D5846
:109DC500502034232035374B014D58502031232066
:109DD50035374B014D5850403130234031394B0117
:109DE5004D58502031232031394B002156495353CA
:109DF5005A412001465020554A2020202020014666
:109E050050204D4153494B202001465020546F525C
:109E15004C2020200101434F4D3A01465054204625
:109E25004F4741442001465054204B754C44202057
:109E3500016F535A40465054404B754C01014650F2
:109E4500544F4B2054415620014D494E40465040F9
:109E5500546F524C0049524E5921544156004D45BC
:109E65004E542000414B5455414C5340504F5A2EAF
:109E7500005441524F4C20202020002053544F5273
:109E8500452157505420002046554C4C2000214078
:109E9500546F524C455300535A4552004952444160
:109EA50000555342200055534220004C495354005D
:109EB5004B754C4400204154564954454C492E4855
:109EC500494241202000214B494C45502020015555
:109ED50054564E4C4056414C01554A204650202080
:0D9EE5002020200155545620535A45524B61
:109EF2002001464F524449542055545601465020A1
:109F0200546F524C4553200155545620546F524CB5
:109F120045530143594C2052414449555301434F43
:109F22004D3A0155545620464F474144200155545D
:109F320056204B754C44202001505245434845431E
:109F42004B005554562156414C20200055404A4062
:109F5200200020554A2040504F5A402100214046BF
:109F62004F52444954204000464F52444954002124
:109F7200404650544B40544F524C005554564E405C
:109F8200544F524C004E454D2075524553202000EF
:109F92002140555456404B754C44002020524144B8
:109FA20049555300214B494C4550014C45475452A9
:109FB20040546F4C5421014C45475452404E455A2F
:109FC20020014F53535A214C4721544F5201014310
:109FD2004F4D3A014C4547545220464F4744014C9D
:109FE20045475452204B754C44004C45475452202F
:109FF2004E455A202020202020004D4F5A474154E0
:10A002002000464F524741534420202000534B41E9
:10A012004C2020582F592020564953535A2000547F
:10A02200415620546F524C004155544F2E42452008
:10A03200004155544F2E4B4920002020534B414C98
:10A042004100544156204B4D2000544156204E4D64
:10A052002000214B494C4550202001564152494F86
:10A0620020202068690158432D4245414C4C6869C3
:10A07200015645522D4245414C686901414C544CB0
:10A08200414E4F536869014B455045524E596F68D6
:10A0920069010101414C41502D4D4F442001475966
:10A0A200415249204245414C015445535A5452456C
:10A0B2005020016F535A2152455021546F520021B2
:10A0C2004B494C455020200153754C5948414E474D
:10A0D2000153754C59212D0153754C59404D4F4434
:10A0E2000153754C5940494E560156415220544332
:10A0F20040202040230148414E4745526F015641BE
:10A1020052494F204E554C4C0148414E474D414714
:10A112002001504552494F44555301564152204166
:10A12200564020304023014E4554544F2D014841A2
:10A132004E475445535A54200053754C5948414E8A
:10A142004700532D48414E47214B49004E494E434B
:10A1520053214455414C00564152494F204E554CD3
:10A162004C005641524A2031302050455243494713
:10A172002020004E554C4C415A4153202020202093
:10A18200202000214B494C45502020015554564F68
:10A192004E414C20014155544F43454E540101411B
:10A1A200544C2F544156200153494B4C204B414CA7
:10A1B2000153535A0101535A454C21542D55500114
:10A1C20043454E5421542D55500157415950542165
:10A1D20042524700214B494C4550202001535441E3
:10A1E20052544049446F2001454C536F200144456D
:10A1F2004C54413A2001546F42535A6F526F5320CC
:10A202000155544F4C530143594C53494740202068
:10A212004023015554564056414C4C200101010146
:10A2220043594C520143594C21495246454C002155
:10A232004B494C45502020010145475347014B41B2
:10A24200545440302C402023014B4F4E5452535A09
:10A2520054014E4D45412131383301494D50454C51
:0DA262004C455201494D502D43414C0143E4
:10A26F002D564152494F0154454320202040303054
:10A27F0040250141004E4F20414750532F464C007F
:10A28F00414C54492D475053202000464C47542DE4
:10A29F004C4556454C0041475053203C3E20464CC0
:10A2AF00004046504E54204C4554455A494B2020AF
:10A2BF0020400046504F4E5420202000204B494C48
:10A2CF00455020202100464F474144202000535A3B
:10A2DF00414240003C2D204C495354202D3E20201C
:10A2EF00455849540053454C004E455854004B6F48
:10A2FF0056204650202000454C6F5A6F2046500084
:10A30F00535A415240546F524C006F53535A40545A
:10A31F006F524C004B49202020202020202020006D
:10A32F00204B4920004750532048494241202000EC
:10A33F00205441524F4C202020005554564E4C0073
:10A34F004B4F5A454C49004C4953544100455445D5
:10A35F00004D41474030007552455320555456200B
:10A36F00200054554C40534F4B20200021404C4966
:10A37F00534056414C20002046504056414C4C21F2
:10A38F0020002140464F47414420204000202040DC
:10A39F004F4B4540202021004F4B45005641520066
:10A3AF00464958004741544521580053545254567A
:10A3BF004E4C20202000535443594C2000404B4911
:10A3CF00200054502000406A40494E200040674012
:10A3DF004F55540020204849424120202100204B56
:10A3EF00494C5000535A4552004947454E00554A73
:10A3FF00202020414C4C2020535A45524B004B4FAC
:10A40F0056202020202056414C2020204B49005818
:10A41F0043542D464C49474854200055534544005A
:10A42F00454E54455220004D4D2E4D4D4D20004D63
:10A43F004D2753532E530057475321383400204094
:10A44F00554054404D402000554054404D0020553C
:10A45F00544320004C4F43414C00535749535347EB
:10A46F004400414C54005355494058004156474011
:10A47F002030402300353030003136343000205D3D
:10A48F00203130404B632F70005D2020203140631E
:10A49F002F2300205D202035404B5453005D203288
:10A4AF0030304046504D00406340204B63004654CF
:10A4BF00204B6300406340204E4D004654204E4DCC
:10A4CF00004D2F53003230305E003530305E00319A
:10A4DF002200322200332200352200382200464C5F
:10A4EF003700464C313600464C333300464C363538
:10A4FF0000463130300046313630004632363000BB
:10A50F005E252640534F47005E2526405441530099
:10A51F00414C540056415200225E2F24004B54539D
:10A52F0000532F4E002224004B5400225E004E4D4C
:10A53F0000302C3500312C3000322C3000302C36CE
:10A54F0000312C3200322C3500332C3800372C35AB
:10A55F000040313500403330004036300054415315
:10A56F004B00464C2D4441544500545000544F4627
:10A57F00005354410046494E004C414E0053455440
:10A58F00204F4646534554004953412048454947BB
:10A59F004854004155544F2D474F200053544152BA
:10A5AF00540020434845434B40414C4C00524144DA
:10A5BF002044495354004053454C4048454947486F
:10A5CF00543A00475053404241524F40414C4C0087
:0DA5DF0053494E4B40312D3221632F230094
:1063FC00304D2475A7049005C2E0F51CE0F51DE0B6
:10640C00F51EE0F51FE0F56DE0F56EE0F56FE0F5DB
:10641C0054126FBE1269FC2275C70375C6E475B9B8
:10642C0001E5BCB48143126FBE1255E48E628F63DA
:10643C007568F97569001264D2203C2D203B2B1233
:10644C0066071265DB856D1C856E1D856F1E855478
:10645C001F12653E203C12203243201D231266077A
:10646C001269FCE532242850DC2212653E203CF9EE
:10647C00203DF6203205201DBD80EF301DB880EA8E
:10648C001266071269FC856D1C856E1D856F1E8555
:10649C00541F1265F11269FC203DCE809912682AB6
:1064AC00201D0D755310740012678D203DBB808626
:1064BC00E553540FC553C4540F2035051266A28002
:1064CC000312678D808BC23CD23B12658EFD126528
:1064DC008EFC12658EC39573F565EC9574F564EDC1
:1064EC009575600504600A800EE56424E050118007
:1064FC0006E5642420400912658E12658E02658EB5
:10650C0012658EFD12658EFC12658EC39576F5674D
:10651C00EC9577F566ED9578600904600122E566E7
:10652C00F48002E5668562F0A474E025F04002C2B6
:0D653C003B22C23C12658EA2E7923DA2E612
:10654900921DA2E592324026A2E492E592E692E7F4
:10655900FC12658E2565F565EC3564F56412658E6A
:10656900FC12658E2567F567EC3566F56622A2E4AF
:106579009235540F79C6F712658E09F7301D051249
:10658900658EF55322E5697023E56860302404407F
:106599002CE56875F004A485F0C7F5C675B901E561
:1065A900BCB4811985BD68756902801E54037010D9
:1065B90005C675B901E5BC056953690F22D23C22AC
:1065C900147004E5BD80F0147004E5BE80E9E5BFF0
:1065D90080E575A7009006F6E56DF0A3E56EF0A3DA
:1065E900E56FF0A3E554F02275A7009006F6E0F5F3
:1065F9006DA3E0F56EA3E0F56FA3E0F55422E56421
:10660900B2E7F56D85656EAB67E566FC30E707C3F4
:10661900E49BFBE49CFCAA62A9631252E4E56630A0
:10662900E707C3E49DFDE49EFEEEB2E7F56F8D54E6
:106639002275380C1268931268DED5530122753819
:106649000C1268641268D4D5530122753800126897
:0E6659007C1268A3D5530122753800126864C4
:106667001268A3D553012275380312689312690F74
:10667700D5530122753803126864126905D5530191
:106687002275380F12687C126934D5530122753888
:106697000F126864126934D55326229066A72373B4
:1066A7008091807780688059804A803B802C801D4C
:1066B700800E80DA80CB80BC80AD809E808F80800A
:1066C700753815126893126956D553012275381516
:1066D70012686412694BD553012275380912687C18
:1066E70012691CD553012275380912686412691C96
:1066F700D55301227538061268931268C6D553011F
:10670700227538061268641268BBD55301227538A2
:106717001212687C1268ECD5530122753812126880
:10672700641268ECD553012202663A75381512686F
:1067370093126956D553012275380F12686412698E
:1067470034D553012275380F12687C126934D5533A
:106757000122753803126864126905D55301227541
:10676700380312689312690FD55301227538001246
:1067770068641268A3D553012275380012687C1229
:1067870068A3D55326229067922373809E80A980A1
:10679700B480BF80CA80D580E08010801B802680AF
:1067A70031803C80478052805D806875380C126864
:1067B700641268D4D553012275380C126893126895
:0E67C700DED55301227538121268641268EC98
:1067D500D553012275381212687C1268ECD5530125
:1067E500227538061268641268BBD55301227538C4
:1067F500061268931268C6D55301227538091268C6
:106805006412691CD553012275380912687C126916
:106815001CD553012275381512686412694BD5537E
:10682500012202673278C686040886037AED125281
:10683500A278CAA60408A60378C686040886037A41
:10684500621252A278CCA60408A60378C68604086C
:1068550086037AB51252A278C8A60408A603227543
:106865001A6A751B0A78CA8618088619126AA778E3
:10687500CC86060886072278C88618088619E4F5A6
:106885001AF51B126AA778C886060886072278C6F5
:106895008618088619751A00751B01026AA7E51D79
:1068A5002519F51DE51C3518F51CC3E51F9FF51FBA
:1068B500E51E9EF51E22C3E51F9FF51FE51E9EF5ED
:1068C5001EC3E51D9519F51DE51C9518F51C22E55A
:1068D5001D2FF51DE51C3EF51CC3E51F9519F51F7C
:1068E500E51E9518F51E22C3E51D9FF51DE51C9EA9
:0968F500F51CC3E51F9519F51F00
:1068FE00E51E9518F51E22E51F2FF51FE51E3EF528
:10690E001EE51D2519F51DE51C3518F51C22C3E5E0
:10691E001D9519F51DE51C9518F51CE51F2FF51F86
:10692E00E51E3EF51E22E51D2FF51DE51C3EF51C50
:10693E00E51F2519F51FE51E3518F51E22C3E51DA9
:10694E009FF51DE51C9EF51CE51F2519F51FE51E7F
:10695E003518F51E22E51A7009E51B70058C068D9B
:10696E000722ED851BF0A4A2F792D5ED851AF0A4AF
:10697E00AEF0FFEC851BF0A4A2D53FEE35F0FF92F2
:10698E00D5EC851AF0A42FFFE435F030D50104FEC6
:10699E0022E4F51AF51BEF4E7003051B22EF651965
:1069AE007006EE65187001227808C3EF33FFEE33E0
:1069BE00FEEF9519F5F0EE95184003FEAFF0E51ACF
:1069CE0033F51AD8E5F4F51A751BFF7805C3EF33C6
:1069DE00FFEE33FEEF9519F5F0EE95184003FEAF7E
:0369EE00F0E51BB6
:1069F10033F51BD8E5F4C403F51B22E51D9511E51C
:106A01001C9510500BE56E9511E56D951050012206
:106A1100E51F9511E51E9510500BE5549511E56F95
:106A21009510500122E51D9513E51C9512400BE5CB
:106A31006E9513E56D9512400122E51F9513E51E34
:106A41009512400BE5549513E56F951240012253C1
:106A51002CF8C3E51F9554FFE51E956FFE9260501B
:106A610007C3E49FFFE49EFEC3E56E951DF519E59E
:106A71006D951CF5189261500BC3E49519F519E455
:106A81009518F518C3E5199FE5189E9262500AE51D
:106A910018CEF518E519CFF51912699FE52C5407A1
:106AA10075F003A4F538E538906AAD73026AC50242
:106AB1006AD9026AE7026AFF026B12026B25026B56
:106AC10033026B4B851C16851D17C3E4951FF51505
:106AD100E4951EF514026B5E851C16851D17851E37
:106AE10014851F158077C3E4951DF517E4951CF5F2
:106AF10016C3E4951FF515E4951EF514805FC3E4F4
:056B0100951DF517E4ED
:106B0600951CF516851E14851F15804CC3E4951F2C
:106B1600F517E4951EF516851C14851D1580398517
:106B26001E16851F17851C14851D15802BC3E4951D
:106B36001FF517E4951EF516C3E4951DF515E495A6
:106B46001CF5148013851E16851F17C3E4951DF5C5
:106B560015E4951CF5148000C3E5179513E5169505
:106B66001210D70122E5159513E514951210D701D9
:106B760022E519F92517FFE518F83516FED3EF9526
:106B860011EE9510500122E5119517FDE5109516A9
:106B9600FC402A4D6027126963E5152FF515E514AB
:106BA6003EF514E5159513E514951210D70122E567
:106BB600199DF9E5189CF8851016851117E5172912
:106BC600FFE51638FEE5139FE5129E500BC3E5134D
:106BD6009517F9E5129516F8E51A700AE51B700681
:106BE600AA00AB018013E9851AF0A4E5F0FBE8855D
:106BF6001AF0A42BFBE435F0FAE5152BFBE5143A65
:066C0600FAE5119BE51008
:106C0C009A10D70122EB9515FDEA9514FCC3E515F6
:106C1C009511E514951010D717E5139BE5129A50B2
:106C2C0036E5139515FFE5129514FE126EDB8027E1
:106C3C00EB9511FFEA9510FEAA00C001126EDBD095
:106C4C0003E5172BFBE5163AFAEB99F517EA98F5DD
:106C5C0016851115851014C2D5E5466002D2D5AA49
:106C6C0056E98AF0A4ABF0E88AF0A42B30D5047571
:106C7C00F00384F8700122E5172513FDE516351293
:106C8C00FCED8AF0A4ABF0EC8AF0A42B30D50475A3
:106C9C00F00384FEE5152513FDE5143512FCED8A91
:106CAC00F0A4ABF0EC8AF0A42B30D50475F003847F
:106CBC00F9E538906CC373026CDB026CE7026CF084
:106CCC00026CF9026CFF026D0B026D12026D17C3A0
:106CDC00743E9EFFC3743E99FE8032C3743E9EFF89
:106CEC00AE018029AF06C3743E99FE8020AF06AE7C
:0D6CFC0001801AC3743E9EFEC3743E99FFD2
:106D0900800EC3743E99FF8007C3743E9EFEAF0197
:106D190008EF2437FFE51B7007E51A700CE8800EB1
:106D2900A2E7E51A50030460F488F0A4E5F06001D5
:106D390004F923FA98FBC3E998C333F9906D4BE53D
:106D49003873026D63026D90026DC5026DF2026EB9
:106D59001F026E4C026E79026EA605A7800BEB30FE
:106D6900E7032A8002291E1FFBEEC45403F583EEB4
:106D79005408C42FF582EE5407243883F5F0E04512
:106D8900F0F0D8DA05A72205A7800BEB30E7032A34
:106D99008002290E1FFBEEC45403F583EE5408C488
:106DA9002FF582EE5407240B83F5F0E045F0F0D877
:106DB900DA05A722804020100804020105A7800BEC
:106DC900EB30E7032A8002291E0FFBEEC45403F5BA
:106DD90083EE5408C42FF582EE540724EC83F5F0B2
:106DE900E045F0F0D8DA05A72205A7800BEB30E7DC
:056DF900032A800229BD
:106DFE000E0FFBEEC45403F583EE5408C42FF58238
:106E0E00EE540724BF83F5F0E045F0F0D8DA05A77D
:106E1E002205A7800BEB30E7032A8002291F1EFBF9
:106E2E00EEC45403F583EE5408C42FF582EE5407D6
:106E3E00249283F5F0E045F0F0D8DA05A72205A7F5
:106E4E00800BEB30E7032A8002291F0EFBEEC454A1
:106E5E0003F583EE5408C42FF582EE5407246583A0
:106E6E00F5F0E045F0F0D8DA05A72205A7800BEB88
:106E7E0030E7032A8002290F1EFBEEC45403F5836C
:106E8E00EE5408C42FF582EE5407243883F5F0E053
:106E9E0045F0F0D8DA05A72205A7800BEB30E70303
:106EAE002A8002290F0EFBEEC45403F583EE54081C
:106EBE00C42FF582EE5407240B83F5F0E045F0F075
:106ECE00D8DA05A7228040201008040201EC701FBA
:086EDE00ED20E740D2E023CFD4
:106EE60023CF30E7F980357B08801A7B1080167B2C
:106EF6002080127B40800E20E4ED20E3EE20E2EFBE
:106F060020E1F07B80EE8BF0A4CF8BF0A4E5F02F90
:106F1600FFEC8BF0A4CD8BF0A4E5F02D2499838FA4
:106F2600F0A433E5F033FBE98BF0A4E5F0C88BF071
:106F3600A428F9E435F0F822FFFEFCFAF8F6F4F29C
:106F4600F0EFEDEBEAE8E6E5E3E1E0DEDDDBDAD9FA
:106F5600D7D6D4D3D2D0CFCECCCBCAC9C7C6C5C458
:106F6600C3C1C0BFBEBDBCBBBAB9B8B7B6B5B4B372
:106F7600B2B1B0AFAEADACABAAA9A8A8A7A6A5A45E
:106F8600A3A3A2A1A09F9F9E9D9C9C9B9A99999822
:106F96009797969594949392929190908F8F8E8DC9
:106FA6008D8C8C8B8A8A8989888787868685858455
:106FB600848383828281818075A700906FE4E54691
:106FC600FA24FA50027A05EA2323F978107F04930B
:106FD600F60809E9DFF9906FFCEA93F556227FC2BD
:106FE600803E7F4680BA7E8C81747D1882E87A3036
:106FF60085D074608BA08080402010081270080233
:10700600725ED215D274D273C219C23A1255E48E88
:1070160047757D0075460575520212905112022180
:10702600E53524EB500E1290517F1990A021127570
:10703600F812DD18E55275F016A4F5701272147583
:107046007E151270DF7F237E09909FFC12760A124E
:10705600DD1810000810010D10021280E21271876F
:1070660075330180DA1271CC75330180D2757E00DA
:107076001270DF7E0090A00F12763D7F237E059072
:10708600A00412760A12713012DD18E55210000FB4
:1070960010010510028780D5045403F55280CE12E4
:1070A60070DF7F237E0B90A03E12760AE5466007CE
:1070B6001460041412405D12DD18E5461000081035
:1070C600010B10021180D860D6154680D2B4050295
:1070D60080CD054680C902702375320012DEEE7F30
:1070E600017E11909FEC12763D7E0012D5AFE57EB3
:1070F600D26612D60675170812DA3912409C7571D7
:1071060000C20612D756741BFFF5177E0F90A044D7
:10711600305D0390A04C12763D129094125C1512CD
:107126004602C206126424021D46E552601414602B
:107136001E1460297F647E2D791C12717A1E1FD958
:10714600F9227F6A7E1F792812717A1FD9FA227F67
:10715600487E2D791C12717A0F1ED9F9227F567E30
:107166003379281F12DE330F0F12DE331F12DE3380
:107176001ED9F0221E12DE330E0E12DE331E02DE82
:1071860033E552605514606814606D800075709E1A
:107196001272018003757000E5732540F573E435BE
:1071A60074F574E43575F5752275701612719E8046
:1071B6000375702DE5762542F576E5773541F57749
:1071C600E43578F57822E55260CB1460DC1460E192
:1071D60080007570441271BA800375705AE5739514
:0971E60040F573E5749400F574A2
:1071EF00E5759400F575227570711271E380037562
:1071FF007088E5769542F576E5779541F577E578F0
:10720F009400F57822E54690722A93F540FEAD473B
:10721F00E4FFFC1253778E418F4222020C1830602C
:10722F00C07F40120D8B121D5C12DD181274D9EB4A
:10723F007005909D46800B1272E790A39C500390AF
:10724F00A3E37F3F7E0412760A12DD1812DDF912D6
:10725F00DE29753709909FA6121C4290726E730239
:10726F00029302742E02700202750A02725E02729B
:10727F008602729F0272307F2E1215C980D17F361F
:10728F007E0490A37112760A12DD1812DDF980BF09
:10729F007F37120D8B121D5C12DD181274BD124751
:1072AF0092D2AC1000A9306DFA127397203BCF40E9
:1072BF00ED7568F97516001273E440FB1275807F47
:1072CF00367E29E51612D38F12DD1805161276B009
:1072DF0078C6B6F7E20274B77C0512479212DC3219
:1072EF00744112DC43745312DC00EB12DC21127672
:1072FF00C25003DCE5227515F975160010000EE576
:10730F0015602512733940051273605002D3227F26
:10731F003F7E29E51612D38F12DD187F1412DE106F
:10732F000516E51664F870D4C322127C7875B9017E
:10733F00E5BCB4811AE5BDF51570037516F778C66F
:0B734F00A616127DC1127DB9127DB997
:10735A00C3027DB9D3227F0575F019D5E0FDD5F0BA
:10736A00FA12479212DC32744112DC43744212DC84
:10737A00007E0F78C6E60812DC00DEF912DC241261
:10738A0076C2400122DF012275F00080CEC23B1294
:10739A004792D2AC12DB8B204C3CB440F712DB9004
:1073AA00B4400312DB90B4412DF53812DB90B4538C
:1073BA002512DB90FA12DB90E538701A12DB90B4D2
:1073CA000D1412DB90B40A0EC3E5169A4003027636
:1073DA00A7C2ACD23B22C2ACD32212770612479282
:1073EA00D2AC1000F112DB8B204CEBB440F412DB70
:1073FA0090B4400312DB90B441DCF53812DB90B450
:10740A0042D47E1078C612DB90F608DEF9E53870B1
:10741A00C512DB90B40DBF12DB90B40AB9C2ACC37B
:10742A002202725E7F0A120D8B121D5C12DD181287
:10743A0074BD1247ABD2AC1000E712DB90B440F532
:10744A00F53812DB90B46EED12DB90E538600A1263
:10745A0047AB744F12DC0C80DC1247AB744012DC71
:10746A0043E51612DC0C12DC167568F97516001263
:10747A0047ABD2AC10003912DB90B440F7F53812A2
:10748A00DB90B44EC07E1078C612DB90F608DEF9A7
:10749A001247ABE5386007744F12DC0C80D11275C5
:1074AA00800516745112DC0C78C6B6F7C212751D27
:0C74BA0002725E751500751603127C6FDF
:1074C60075B901E5BC30E70205160515E51524205A
:1074D60050EB227B007515F9127C7875B901E5BC75
:1074E600B481010B0515E515240450EC7515011240
:1074F6007C6F75B901E5BCB481010B0515E5152452
:107506002050EC227F1C120D8B121D9F4006751514
:10751600F912751D02725EE51560372404401A24BF
:107526001E5019E515240740028027127C78127533
:10753600590515E515240450F2751501127C6F7571
:10754600B901E5BC30E7031275590515E515242088
:1075560050EA2212756E124E2C05C6124E2C05C626
:10756600124E2C05C6024E2C74FF80057404800151
:10757600E4F5BCF5BDF5BEF5BF22E568606AF51514
:107586000515E5152404501D751501127C6F75B996
:1075960001E5BC30E70280190515E515242050EBFE
:1075A600751500800C241C60F750E0E51524065084
:1075B60037E56875F004A485F0C7F5C675BC81E5A6
:1075C60015F5BDF56878C6B6F70375BD00081275E2
:1075D600E31275DD1275DD86BC0886BD0886BE0819
:0975E60086BF08124E2C05C622D6
:10C00C0012AE0712C10B12818912C09012819112CB
:10C01C00C09D02AE0B12AE0712C10B1281897F5A62
:10C02C00C23C12806B128267783F79437F607EEA54
:10C03C0012C0FF1281917F6512806B128267783D6E
:10C04C0079417F207E4E12C0FF303C2012C2C112BB
:10C05C00C11C783F794312C07B783D794112C07B7B
:10C06C0012C2C178D7E65480F6753700029266C3C7
:10C07C00E796FF1819E796FE0809C3E69FF718190B
:10C08C00E69EF7227F5B7E0690A47512763D1F809C
:10C09C000A7F667E14745912D4A81F127EF47E395E
:10C0AC00E402D4C77866E620E73418C3E694720835
:10C0BC00E694045029C318E6941F08E69404401E25
:10C0CC007869E620E71818C3E6940E08E694015048
:10C0DC000DC318E6947508E694004002D322C322DF
:10C0EC00E67D0030E7011D08E62BFB18E63CFCE47E
:0EC0FC003DFD22C3EB9FF6F71819EC9EF6F7F8
:10C10A002212C0B0400CE47842F608F67840F608ED
:10C11A00F6227864C3E6946AF55708E6944CF55615
:10C12A000808C3E69458F55B08E694AEF55A7539E3
:10C13A0000AC56AD57EC12B1B4784C12B242AC5ABC
:10C14A00AD5BEC12B1B4785012B2427F2B7E867D81
:10C15A00777C1812B179785012B23612B08512B1C2
:10C16A0079785012B23612B08512B179785012B27B
:10C17A003612B08512B1797F367E847D257C6412B1
:10C18A00B179785012B23612B08512B179784C1260
:10C19A00B23612B08512B1797F3F7EA27D607C8B68
:10C1AA0012B179785012B23612B08512AE7312AE4D
:10C1BA007312B24E7F3F7E807D057CE6053912B050
:10C1CA0085784812B2427F2C7E937D477C7F12B1DC
:10C1DA0079785012B23612B08512B179785012B20B
:10C1EA003612B08512B179784C12B23612B0851275
:10C1FA00B1797F357EB47DF87CDF12B1797850123F
:10C20A00B23612B08512B179785012B23612B085B0
:10C21A0012B1797F3F7EED7D227CCD12B179784CC7
:10C22A0012B23612B08512AE7712AE73784412B2D9
:10C23A00427F317E397D9D7CE712B179784C12B20A
:10C24A003612B08512B179784C12B23612B0851214
:04C25A00B1797844FA
:10C25E0012B23612AE7712B1797F2C7E377D0C7CFE
:10C26E00A312B179784C12B23612B08512B1797828
:10C27E004C12B23612B08512B179784C12B2361217
:10C28E00B08512AE7712B24E7F3F7E807D027C9FCC
:10C29E00053912B085784412B242784812B236127D
:10C2AE00B1EB8E428F43784412B23612B1EB8E4010
:10C2BE008F4122753900AC42AD43EC12B1B47848CF
:10C2CE0012B242AC40AD41EC12B1B4784412B2425B
:10C2DE007F2B7E537D507C0912B179784812B2368D
:10C2EE0012B08512B179784812B23612B08512B1F9
:10C2FE0079784412B23612B08512B1797F347EF25B
:10C30E007DCD7CA312B179784812B23612B0851267
:10C31E00B179784812B23612B08512B1797F3F7E6C
:10C32E000A7D2E7CAE12B179784412B23612B085E7
:10C33E0012AE7312AE73784C12B2427F2B7E4F7DCB
:10C34E00AF7CB212B179784812B23612B08512B102
:10C35E0079784812B23612B08512B179784812B295
:10C36E003612B08512B1797F357EB17D4B7C951238
:10C37E00B179784812B23612B08512B1797844127A
:10C38E00B23612B08512B1797F3F7E497DCD7C45A4
:10C39E0012B179784812B23612B08512AE7712AE5B
:10C3AE0073785012B242784C12B23612B1EB8D55F0
:10C3BE008E568F57785012B23612B1EB8D598E5A67
:04C3CE008F5B7864A5
:10C3D200E557246AF608E556344CF608E555340468
:10C3E200F608E55B2458F608E55A34AEF608E4355B
:03C3F20059F622D7
:1090B40012AE0712974512AE0B7F6690A457127634
:1090C4003B1291227F5A78C41290FE12910678C600
:1090D4001290FE1290E97F6578C81290FE129106F4
:1090E40078CA1290FE7E2DE51B12D4C77E33E51A92
:1090F40012D4C77E39E51902D4C786040886030250
:1091040052417E15E51C12D4C77E1BE51B12D4C741
:109114007E21E51A12D4C77E27E51902D4C77F5AE7
:109124007E01E53A12D3DD7E0B909B39E53B930239
:10913400D4DAE6FF08E6FE08E6FD339217E45001B0
:10914400F4FC12B25F75130A75390112B45D78D755
:10915400E6C2E775F00A84F9303D02A9F012B25F65
:109164008913053912B43630170A053912B4490582
:109174003912B449A80302B24212AE07129745C28B
:109184003C7F5A7E0312841812912212DD181000BB
:109194000810011510022080EFE53A146004153A16
:1091A4008003753A3CD23C80DFE53AB43C05753A1D
:1091B4000180F2053A80EE7E031284137E0B128442
:1091C4001812912212DD1810000810011510022047
:1091D40080EFE53BB40205753B158002153BD23C9C
:1091E40080DFE53BB41505753B0280F2053B80EE5C
:1091F4007E0B1284137F5A78C41290FE12910612C9
:07920400926F12827778C41B
:10920B001292C778C61290FE1290E91292A1751CA9
:10921B000012827778C61292C77F6578C81290FECB
:10922B0012910612926F12827778C81292C778CA7F
:10923B001290FE1290E91292A1751C00128277789F
:10924B00CA1292C7303C14E53B24F4500B78C9E6A4
:10925B002410F618E63427F61292CD12AE0B127DBF
:10926B00F902DD18C2247E15E51C128368F51CD2A9
:10927B00247E1BE51B128368F51B1023E77E21E57B
:10928B001A128368F51A1023E67E27E519128368F4
:10929B00F5191023E822C2247E2DE51B128368F5F5
:1092AB001BD2247E33E51A128368F51A1023E77E4E
:1092BB0039E519128368F5191023E622ECF608EB51
:1092CB00F622129B5178C8E6FE0886073395E0FD1F
:1092DB00FC12B1797FE87E037D007C0012B45D1235
:1092EB00B17978CAE6FE0886073395E0FDFC12B427
:1092FB003612B1797F807E697D677CFF12B436ECC4
:10930B0012B1B012B1797F3F7E807D0D7C1D12B002
:10931B008512B1797F3D7E407D007C0012B179785A
:10932B00BC12B23612B08512B1797F3E7E807D00C1
:10933B007C0012AE7712B17978BC12B23612B085BE
:09934B0012B1797F3F7E807D00A4
:109354007C0012AE7312B17978B412B23612B085B1
:1093640012B0FD783C12B2427F407E807D007C00CA
:1093740012B179783C12B23612B08512B2DC12B155
:10938400797F3F7EA87D007C0012B17978B812B253
:109394003612B08512B08512B1797F407E007D000F
:1093A4007C0012B179783C12B23612B08512B2DC6C
:1093B40012B1797F3F7EC07D007C0012B08512AE71
:1093C4007712B17978B812B23612B08512B17978C1
:1093D4003C12B23612AE77785412B24212B2C67848
:1093E4005812B24212B17912B08512B17978C01212
:1093F400B23612B085784412B242785412B23612A0
:10940400B2DC783C12B24212B17912B08512B17951
:1094140078BC12B23612B085783C12B2427F3E7EDE
:10942400C07D007C0012B179783C12B23612B0854E
:1094340012B1797F3F7E007D007C0012AE7712B1BD
:1094440079783C12B23612B08512B1797F3F7E80B2
:109454007D007C0012AE7712B17978B412B2361264
:10946400B085787012B24278C4E6FE088607339558
:10947400E0FDFC12B1797FE87E037D007C0012B42C
:109484005D12B17978C6E6FE0886073395E0FDFCE7
:1094940012B43612B1797FE07E5E7DF87CFF12B49F
:1094A40036EC12B1B012B1797F3F7E7F7DE57CC985
:0594B40012B17978708F
:1094B90012B23612B08512B0FD785012B2427F3F17
:1094C9007EF07D007C0012B179783C12B23612B080
:1094D9008512B1797F3F7EC07D007C0012AE771284
:1094E900B179783C12B23612B08512B1797F3F7EDC
:1094F900807D007C0012AE77783C12B24278BC12B3
:10950900B23612B1797F3F7E807D007C0012AE7346
:1095190012B179783C12B23612B17978B412B236F6
:1095290012B08512B085784012B242785412B23620
:1095390012B314783C12B24212B17912B085787420
:1095490012B2427F417E107D007C0012B17978C051
:1095590012B23612B08512B1797F407E807D007CCF
:109569000012B179784412B23612B08512B1797FFE
:10957900417E207D007C0012AE7312B179784412CD
:10958900B23612B08512B1797F407E407D007C00F1
:1095990012B179787412B23612B08512B1797F405E
:1095A9007EA07D007C0012AE7712AE7712AE7312E8
:1095B900B179785012B23612B08512B17978501259
:1095C900B23612B08512B1797F3D7E2A7DAA7CAB75
:1095D90012B08512B1797F3F7E007D007C0012AE0A
:1095E9007312B179783C12B23612B179787012B22D
:1095F9003612B08512B179784012B23612B0FD1226
:10960900B179785012B23612B08512B17978501208
:10961900B23612B08512B08512B179785412B236C9
:0C96290012AE7312B1797F4A7E517DD2DF
:109635007CCB12B08512B1EB78AC12B2427F407E82
:10964500007D007C0012B179787412B23612B085B3
:1096550012B1797F3F7E807D007C0012AE7712B11A
:1096650079784412B23612AE7712B179785012B2C7
:109675003612B08512B179785012B23612B0851211
:10968500B179785012B23612B08512B1797F3E7E2B
:109695002A7DAA7CAB12B08512B179785012B23608
:1096A50012AE7312B179785812B23612B0FD12B1FA
:1096B500797F4A7E517DD27CCB12B08512B1EB12F7
:1096C500B179AF3AEF3395E0FEFDFC12B1797F40F9
:1096D5007E7E7D057C0012B45D12B1797F607E755A
:1096E5007D587CFF12B43612B43678B012B2427887
:1096F500AC751B6412971C8F1C78B0751B6712978D
:109705001CE51C75F00AA42FFF249C50027F0078ED
:10971500D7E654802FF62275390012B23612B17988
:109725007F0A7E007D007C0012B509A81BE513F6B3
:1097350008E512F608E511F6335004EFF404FF22AC
:10974500C23D78647BAC129136D23D78677BB0120E
:109755009136129B517F007EE47D577C0012B179D2
:1097650078AC12B23612B43612B1797F007E537DD1
:0E977500077C0012B50912B19885133B7F8066
:109783007ECB7DA47C0012B17978B012B23612B4CC
:109793003612B1797F407E7E7D057C0012B50912B9
:1097A300B198E513F56F04F53A85126E85116D8551
:1097B300106C7F407E7E7D057C0012B179786C123F
:1097C300B23612B45D12B1797F607E0C7DA27C004B
:1097D30012B17978B012B23612B43612B449786C39
:1097E30012B24278AC12B236EC12B1B012B1797F38
:1097F300347E9C7D2B7C5F12B085785412B242126A
:10980300B2C6785012B242786C12B236EC12B1B0D2
:1098130012B1797F347E9C7D2B7C5F12B08512B1AF
:1098230079785012B23612B085784012B2427F4036
:109833007E007D007C0012B179785412B23612B0EA
:109843008512B2DC12B1797F3D7EC07D007C0012AF
:10985300B17978BC12B23612B08512B1797F3E7EEF
:10986300C07D007C0012AE7712B17978BC12B2369B
:1098730012B08512B08512B1797F3D7E407D007CA8
:109883000012B17978BC12B23612B08512B1797F69
:109893003E7E807D007C0012AE7712B17978BC12D7
:1098A300B23612B08512B1797F3F7E807D007C0095
:1098B30012AE7312B179785412B23612B08512AE69
:1098C3007312B1797F407E807D007C0012B179787C
:1098D3005412B23612B08512B2DC12B1797F3D7EDA
:1098E300707D007C0012B17978BC12B23612B0855B
:1098F30012B17978BC12B23612B08512B08512AEAD
:109903007712B17978B412B23612B085785812B2A0
:1099130042785412B23612B2DC783C12B242785416
:1099230012B23612B314785412B242783C12B236E1
:1099330012B17912B08512B17978BC12B23612B075
:1099430085783C12B2427F3E7EC07D007C0012B11E
:1099530079783C12B23612B08512B1797F3F7E001E
:109963007D007C0012AE7712B179783C12B23612C8
:10997300B08512B1797F3F7E807D007C0012AE7787
:1099830012B17978B412B23612B085787012B2423D
:10999300785012B23612B17912B08512B17978C00B
:1099A30012B23612B085784412B242785412B236EB
:1099B30012B17912B085787412B242784012B2367D
:1099C30012B17912B085783C12B2427F407E807D1D
:1099D300007C0012B179784412B23612B08512B10C
:1099E300797F417E107D007C0012AE7712B17978C9
:1099F3004412B23612B08512B179787412B23612AB
:109A0300B1797F407EA07D007C0012AE7312AE77E9
:109A130012B179783C12B23612B08512B1797F3D1A
:109A23007E2A7DAA7CAB12B08512B1797F3F7E007E
:109A33007D007C0012AE7712B179785412B23612DF
:109A4300B179787012B23612B08512B179783C12BE
:109A5300B23612B08512B08512B179785812B23687
:109A630012AE7712B1797F3F7E7F7DE57CC912B05C
:019A7300856D
:109A740012B1797F4B7E187D967C8012AE7712B13D
:109A8400EB12B1797FE87E037D007C0012B50912E8
:109A9400B19878C8A61208A61308A60608A60778DF
:109AA4007412B23612B1797F3F7E807D007C001241
:109AB400AE7312B179784412B23612AE7712B1791C
:109AC4007F3E7E2A7DAA7CAB12B08512B1797840A4
:109AD40012B23612B08512B179783C12B23612B095
:109AE4008512B179784012B23612AE7712B1797F0D
:109AF4003F7E7F7DE57CC912B179787012B236124F
:109B0400B08512B08512B1797F487EF47D247C0043
:109B140012AE7712B1EB12B1797FE87E037D007C3F
:109B24000012B50912B19878C4A61208A61308A6A3
:109B34000608A607223F3F4344454647484A4B4C44
:109B44004D4E5051525354555657583F3FE4F539F2
:109B5400F5A7909B65791078B4E493F6A308D9F936
:109B64002232A5C24A4A19DC3A885CDB3BFFD6DCC8
:019B74003BB5
:10AE0700D2D58002C2D575A70490040078107F0BB5
:10AE170012AE3378267F0512AE33783C7F2212AE0E
:10AE270033786A7F0F12AE3375A7002230D506E656
:10AE3700F008DFFB22E0F608DFFB22D2D58002C252
:10AE4700D575A7049006FA78737F0612AE3375A7F7
:10AE57000022DA0CD902800BD906303701B350052E
:10AE670002AFE6923702AFD2D9F680F9D236800226
:10AE7700C23612B017303606C86002B237C89236EB
:10AE8700DAD0D9E4B8000A12B05EA236923702AF20
:10AE9700BB60FBB51300400F12B05EA23692F7A25B
:10AEA700379236A2F79237C398F40424E740DF2499
:10AEB70019AD29AC28AB277A00C394084008CDCC3C
:10AEC700CBCAE4CD80F424086010F9C3ED13FDEC80
:10AED70013FCEB13FBEA13FAD9F1A236303701B3AF
:10AEE70040308A17E5102BF518E5113CF519E512E6
:10AEF7003DF51A501A13F51AE51913F519E5181344
:10AF0700F518E51713F5170513E513700205140275
:03AF1700AF71E433
:10AF1A00C39AF517E5109BF518E5119CF519E5128A
:10AF2A009DF51A500DB237C378177F04E496F608D8
:10AF3A00DFFA7A047019E513C39408F51350021561
:10AF4A0014E4C517C518C519F51ADAE802B01220B3
:10AF5A00E7BAE5137002151415137817C37F04E6D0
:10AF6A0033F608DFFA80E8E51A20E7137817C37F7B
:10AF7A0004E633F608DFFAE513700215141513E533
:10AF8A00173378187F03E63400F6500E08DFF7759A
:10AF9A001A800513E51370020514E51420E75470AE
:10AFAA0027E513604E046020851A12851911851849
:10AFBA00105326F0AC10AD11A237E51313FFE512BA
:10AFCA0092E7FEA81302B198E4F512F511F510F50F
:10AFDA00147513FF5326F043260580D8E5FFF512B2
:10AFEA00F511F510751400F513D2375326F04326E0
:10AFFA000980C15326F0432603E4F512F511F51032
:10B00A00F514F513C23780AC5326F080EC79017A37
:10B01A00018512F0E513A2F7339237751400F51380
:10B02A006002D2F785F012A813B8FF0809E512C228
:01B03A00E72E
:10B03B006001098C278D288EF0A2F7EF3304700A7C
:10B04B000AC2F705F00AD5F0011A146002D2F7858F
:10B05B00F02922C88813C512C529C512C511C528E8
:10B06B00C511C510C527C51022DA03B8000302AFFE
:10B07B00E6D9028002D9F702AFD212B017303701EE
:10B08B00B392377004D9E78005DADEB8000302B05B
:10B09B0012D9E2C3947E500215142513F5135002F6
:10B0AB0005147815760008B81BFA78277915E60889
:10B0BB00FAE8FC78108AF0E608A427F709E5F037E0
:10B0CB00F7500989F00907E760FBA9F0B813E619F7
:10B0DB0019ECF8B82AD802AF7102AFFDB8FFFA022B
:10B0EB00AFE6D9FB02AFD2DAF6B800F002B012121B
:10B0FB00B24E12B017303701B392377007D9E3B89D
:10B10B0000E280DBDAE1B8000280E1D9D5C8C39850
:10B11B0050021514247F50020514F513781A76008B
:10B12B007A1A7B80C3E5109527E5119528E51295D2
:10B13B00294016C3E5109527F510E5119528F51153
:09B14B00E5129529F512E64BF618
:10B15400DA0302AF71EB03FB30E703187600C3E5B3
:10B164001033F510E51133F511E51233F51240CA29
:10B1740030E7DD80B6E53905396010D0F0D0E0C0A5
:10B1840010C011C012C013C0E0C0F08F138E128D16
:10B19400118C1022E539146010D0F0D0E0D013D017
:10B1A40012D011D010C0E0C0F01539227920800CE3
:10B1B4007910800479087D007E007F003392D55099
:10B1C4000312B228EC33400FEF33FFEE33FEED33BE
:10B1D400FDEC33FCD9EE22EECCF5F0747E29A2D539
:10B1E40013FF92F7AEF022EF8EF0A2F7D2F733926C
:10B1F400D5C3947F5006E4FFFEFDFC229420400456
:10B2040074FF80F304CCFEE4FFFAE5F0CC6012C3D3
:10B21400CC13CCCD13CDCE13CECF13CF0450EEDA56
:10B22400EC30D5D7C3E49FFFE49EFEE49DFDE49C8F
:03B23400FC22E613
:10B23700FC08E6FD08E6FE08E6FF22ECF608EDF658
:10B2470008EEF608EFF622CFC513CFCEC512CECD46
:10B25700C511CDCCC510CC22E4F513F512F511F5C7
:10B267001022E493FCA3E493FDA3E493FEA3E493E9
:10B27700FFA322C0E012B17912B08512B2AD12B2AB
:10B2870069D0E0C0E012B17912B2A412B08512B150
:10B297007912B26912AE77D0E0D5E0E722AC48ADBB
:10B2A70049AE4AAF4B228C488D498E4A8F4B227448
:10B2B700FF7809FFFEFDFCE52654F048F52622122B
:10B2C700B36D04A2E1927F1420E01590B3EE7404ED
:10B2D70012B27A802912B36D30E102B27F20E0EB1F
:10B2E7008C4C8D4D8E4E8F4F90B402740412B27AEF
:10B2F70012B179AC4CAD4DAE4EAF4F12B085307F29
:10B3070004EF6480FFEE33EF337001FF2212B36D59
:10B31700C0E08C4C8D4D8E4E8F4F90B42674031227
:10B32700B27A12B179AC4CAD4DAE4EAF4F12B0857B
:01B33700EC29
:10B33800C54CFCEDC54DFDEEC54EFEEFC54FFF906B
:10B34800B416740312B27AD08212B179AC4CAD4DF6
:10B35800AE4EAF4FE58230E00712B0FDB27F809D60
:10B3680012B0FA8098EE33EF3324605007D0E0D063
:10B37800E002B2B6EFA2E7547F927FFF12B1797C68
:10B38800837DF97E227F3E12B085EE33EF33248130
:10B39800501012B17912B1EB12B1B0EFB2E7FF124F
:10B3A800AE77EE33EF33602A2403F8C313FFEE922F
:10B3B800E7FEE82481E4501A12B17912B1EBEF04E8
:10B3C800C2E0FCF58212B1B8EFB2E7FF12AE77E542
:10B3D8008203FAEE33EF33600B148FF0A2F713FFFA
:10B3E800EE92E7FEEA2283FA703AE4E9AABCF8E0B2
:10B3F800813EE6E99DBF0000803F1A3C2839666916
:10B4080099BBE335A33DE75D25BFDB0FC93FCCDB27
:10B418008D41EE3649C43F91C9453DF8B0C500009D
:10B42800803F34F517C373FA2F45DDFD0AC6EF25B3
:10B4380013FFEE3512FEED3511FDEC3510FC02B1AF
:10B4480098C3EF9513FFEE9512FEED9511FDEC955F
:10B4580010FC02B198EFF88513F0A4FFE513C5F0CE
:0AB46800CEF9A42EFEE435F0CDFA73
:10B4720088F0E512A42EFEED35F0FDE433CC851301
:10B48200F0A42CFCE5128AF0A42CFCE51189F0A4AE
:10B492002CFCE51088F0A42CFC89F0E512A42DFD0B
:10B4A200EC35F0FCE51188F0A42DFDEC35F0FC8ABA
:10B4B200F0E513A42DFDEC35F0FC02B198E4CCF8D4
:10B4C200E4CDF9E4CEFAE4CFFB75F020C3E5133303
:10B4D200F513E51233F512E51133F511E51033F5E5
:10B4E20010EF33FFEE33FEED33FDEC33FCEF9BEE5A
:10B4F2009AED99EC98400CFCEF9BFFEE9AFEED99C9
:10B50200FD0513D5F0C622C2D5EC30E705B2D5123F
:10B51200B228E51030E70DB2D512B52C12B4BF1225
:10B52200B228800312B4BF30D515C3E49513F513C6
:10B53200E49512F512E49511F511E49510F5102237
:10A5EC00E57124885002D2191255E48E4712D1ED30
:10A5FC001290941259A0305E0F12593E128783129A
:10A60C00586F12BF9E12419712387D12473E10367A
:10A61C0029201F1C301219E412A77212A78712A846
:10A62C008712A8A930510302A93312AC0420510996
:10A63C00C251E4F552F545F5442275A70075830720
:10A64C00E559C454F0F582E0F538A3E0F518A3A35E
:10A65C00A3E0F51E74FF12A7721255E48E1C8F1B1B
:10A66C007510DF751100E51164B4700612A73D7505
:10A67C00111012A70A4028AE1CAF1B12566C2032C8
:10A68C001EAC03AB027A0C125279ED701275A70056
:10A69C00758304851182ECF00583E510F00511D566
:10A6AC0010C412A73D75C70375C6E075A7049005C5
:10A6BC00007F0412A6F8DFFB75A700122AC61259F8
:10A6CC003EE4F5A7F8F559758307E8C4F582E06513
:10A6DC00387011A3E06518700BA3A3A3E0651E707E
:10A6EC000388592208C3E5589850DC22E0F5BCE0F9
:10A6FC00F5BDE0F5BEE0F5BF124E2C05C622E51007
:10A70C0075F004A4F5C685F0C775B901E5BC3340F6
:0BA71C001F05C605C675B90185BE64A7
:10A7270085BF6505C675B90185BC6685BD6785BEEC
:10A737006885BF69C322E51124FE502E75A7007FE7
:10A7470010AE111E7583048E82E0FD1582E0CDB533
:10A7570005005012F00582CDF00583E0FD1582E07B
:10A76700CDF00582CDF0DEDCDFD72275A75490044B
:10A777000005A79005007FB4F0F0DFFC75A7002265
:10A7870012BDFBC2517B077AFFE4FFF5A7900400D7
:10A7970012A86DED244C4035EC603075A7008D8212
:10A7A70005A712A8337583058D82E02410401CF09D
:10A7B70005A7E02CF0500505A7E004F0BA000CBB94
:10A7C7000009D251EF24DC50027F23DFC3EA600582
:10A7D70012A7E68006EB600312A81E75A7002230B9
:10A7E700E0047553082230E1047553182230E2045F
:10A7F7007553282230E3047553382230E404755327
:10A80700482230E5047553582230E6047553682210
:10A8170030E7037553782230E0047553882230E11E
:10A82700047553982230E2037553AA22ED54F0C4FD
:10A83700232390A83D735302FE225302FD225302A5
:06A84700FB225302F72280
:10A84D005302EF225302DF225302BF2253027F2213
:10A85D005303FE225303FD225303FB225303FB221A
:10A86D0012BD3312BBC1E4F5F7C2B2C2B2ADF7F5FA
:10A87D00F7C2B2C2B2ACF7D2B22290050078B4E002
:10A88D006015FD54F0C4CD7C00540FFE1583E0FF20
:10A89D00125377EFF005830582D8E422758304788F
:10A8AD00FF088882E060FAF5D38812E512244C5037
:10A8BD00012285D3D288D4881279FF0512E5126062
:10A8CD00F00908E875F0B484A8F08882E060ECF532
:10A8DD00D3B9000280D5B9230050D0C395D292D1FF
:10A8ED005002F40409FEE4FFFCAD0112538474011F
:10A8FD00FA25D475F0B484A8F0AC06AB0712526BF0
:10A90D00EB30E7010CE5D22C30D1029C9C8882F013
:10A91D000AEAB501DCE512244C50012285D3D2851B
:10A92D0012D4A812809390040012A9F28C068B0504
:10A93D0012A9F2E4FFF512F5118C148B13C3ED9BE4
:0EA94D00F9EE9CFA4012E51199E5129A500AB3
:10A95B008C148B138A1289118F528F82E0F9C3EDFD
:10A96B0099FDEE9400FEE582245A5002244C75F0BA
:10A97B00B48485F082E0FA2DFDEE3400FEEB9AFBF9
:10A98B00EC9400FCE92BFBEC3400FC0FBFB4B0E5FE
:10A99B005224D3400224B4F552C3E51333FBE51420
:10A9AB0033FCE511FE2BFBE512FF3CFC1253D9E9FE
:10A9BB00F890AA0493F511FDEBF513FFECF514FEDB
:10A9CB007C001253778F44E890AB0493FAAB13AC33
:10A9DB00141252A2AF03AE04AD117C00125377EFE9
:10A9EB007002F552F545227C007B007F5AE02BFB71
:10A9FB00EC3400FC0582DFF522B4B4B4B4B4B4B4C7
:10AA0B00B4B4B4B4B4B4B4B4B4B4B4B3B3B3B3B300
:10AA1B00B3B3B3B3B3B3B3B3B2B2B2B2B2B2B2B203
:10AA2B00B2B1B1B1B1B1B1B1B0B0B0B0B0B0B0AF13
:10AA3B00AFAFAFAFAEAEAEAEAEAEADADADADADAC2E
:10AA4B00ACACACACABABABABAAAAAAAAA9A9A9A953
:10AA5B00A9A8A8A8A8A7A7A7A7A6A6A6A5A5A5A580
:10AA6B00A4A4A4A4A3A3A3A2A2A2A2A1A1A1A0A0B7
:10AA7B00A0A09F9F9F9E9E9E9D9D9D9D9C9C9C9BF1
:10AA8B009B9B9A9A9A999999999898989797979630
:10AA9B009696959595949494939393929292919173
:10AAAB0091919090908F8F8F8E8E8E8D8D8D8C8CB3
:10AABB008C8B8B8B8A8A8A898989888888878787F8
:10AACB00868686858585848484838383828282813E
:10AADB0081818080807F7F7F7E7E7E7E7D7D7D7C81
:10AAEB007C7C7B7B7B7A7A7A7979797878787777C3
:10AAFB00777676767575757474000203050608090A
:10AB0B000B0C0E101113141617191A1C1D1F2122D2
:10AB1B00242527282A2B2D2E303133343637393A3A
:10AB2B003C3D3F404243454648494B4C4E4F5052AB
:10AB3B0053555658595A5C5D5F606163646667682C
:10AB4B006A6B6C6E6F707273747677787A7B7C7EBF
:10AB5B007F80818384858688898A8B8D8E8F909167
:10AB6B00929495969798999B9C9D9E9FA0A1A2A429
:10AB7B00A5A6A7A8A9AAABACADAEAFB0B1B2B3B402
:10AB8B00B5B6B7B8B9BABBBCBDBEBFC0C0C1C2C3F6
:10AB9B00C4C5C6C7C7C8C9CACBCCCCCDCECFD0D005
:10ABAB00D1D2D3D4D4D5D6D7D7D8D9DADADBDCDC2B
:10ABBB00DDDEDEDFE0E0E1E2E2E3E4E4E5E5E6E76B
:10ABCB00E7E8E8E9EAEAEBEBECECEDEEEEEFEFF0C1
:10ABDB00F0F1F1F2F2F3F3F4F4F4F5F5F6F6F7F72E
:10ABEB00F8F8F8F9F9FAFAFAFBFBFBFCFCFDFDFDB2
:10ABFB00FEFEFEFEFFFFFFFFFFC251E4F544F8141B
:10AC0B00FB900400A9007C0FC2D112AD1FE82405F4
:10AC1B00F8B8B4F08B13E5122403FA244C5001FA64
:10AC2B00BBFF012275112C8A1912AD568F16203DD0
:10AC3B0012AA1975112312AD568F15751600303DDA
:10AC4B00E2801175112312ACFE751500303D05E83D
:01AC5B002FC9
:10AC5C0013F51575111212ACFE751400303D05E894
:10AC6C002F13F514EA2404F552244C5002F552E447
:10AC7C00F51AF51BF51CE516600AFB7A00AF137E7E
:10AC8C00FF12ACC4E515600AFB7A4FAF137EFF12BE
:10AC9C00ACC4E516600DFB7A00E5146006FF7ECFB0
:10ACAC0012ACC4AE1CAF1B7C00AD1A1253778F458F
:10ACBC00EF2513F544D25122EFF5F0A4FCADF0EBE7
:10ACCC00F5F0A49CFCE5F09DFDEB8AF0A4FAABF04A
:10ACDC00EF8EF0A49AF8E5F09BF9E833F8E933F934
:10ACEC007B0012541D051AE51B2BF51BE4351CF5D6
:10ACFC001C22EA2511F9244C5001F9C2D112AD1DC8
:10AD0C00303D428F00C3EA9511F9500324B4F9D2B7
:10AD1C00D17C09E4FDFEFF8982E060062FFFE43E52
:10AD2C00FE0D09B9B4027900DCEDED20D118F51E49
:10AD3C0024FE923D500F125384EFB503005006854C
:10AD4C001E1FFB881222F51D80E612ACFE203D432F
:10AD5C00740212ADF512ACFE203D38740412ADFD38
:10AD6C0012ACFE203D2D740612ADF512ACFE203D4A
:10AD7C0022740812ADFD12ACFE203D17740A12AD00
:10AD8C00F512ACFE203D0C740C12ADFD12ACFE2085
:10AD9C003D0122C3E89F605088148F158A16400825
:10ADAC001ABAFF0A7AB380060ABAB4027A0012AC55
:10ADBC00FE303D34C3E89FF9602EC3E5149515FBB6
:10ADCC006930E7D4E930E703F404F9EB30E702F437
:10ADDC0004C3995002AA16E5142515C82F28FFE4C0
:10ADEC00FC33FE7D04125377222AFA244C5001FACC
:0BADFC0022C3CA9AFA500324B4FA22C2
:10BB8800758000C2B212DE0ED2B275F8302275800E
:10BB980000C2B2F5F7C2B2C2B2D2B222758000C2F8
:10BBA800B2F5F7C2B2C2B2856CF7C2B2C2B2856B47
:10BBB800F7C2B2C2B2856AF722758000C2B275F7C1
:10BBC80003C2B2C2B2856FF7C2B2C2B2856EF7C203
:10BBD800B2C2B2856DF72212BC18740612BB9674F5
:10BBE8000212BBA48FF7C2B2C2B2D2B222909E7622
:10BBF8007F631275F812DD18D214120D8112757652
:10BC0800124E2C12BC18740612BB9674C712BB963F
:10BC180012BC1E40FB22758000C2B275F705C2B285
:10BC2800C2B2C2B2C2B275F705C2B2C2B2C2B2C221
:10BC3800B2E5F7D2B2A2E022120D8185BF6C85BEB3
:10BC48006B756A00E56B7015E56A701112BC1874A3
:10BC58000612BB9674D812BBA4D2B2D21F22E54BEF
:10BC68000475F03C8485F04B12BF23852E72E55F86
:10BC7800030354C0F8E55E543F28F57C3055012293
:10BC880012BCBD12BC1E40F7E54C60F312BC181282
:10BC9800BCD412BCA280F112BC18C21F740612BB1D
:10BCA80096740212BBA4787086F708B880FAD2B2EC
:10BCB80012BCF1808F787075A704758304E54CC4B5
:0CBCC800F5827F10E6F0DFFC054C8019CF
:10BCD400787075A704758304154CE54C30E701E4CE
:10BCE400C4F5827F10E0F6DFFC75A70022741025EE
:10BCF4006A54F0F56AE4356BF56BE4356C540FF572
:10BD04006C22E54B75F010A4256A54F0F56AE5F051
:10BD140080E4E56A24F054F0F56AE56B34FFF56BD2
:10BD2400E56C34FF80D7E56A24FF80ECC380EBE543
:10BD34006D24F054F0F56DE56E34FFF56EE56F3467
:10BD4400FF540FF56F2212BDA212BDCAC22DC254F8
:10BD5400C255E57F7002D255147002D254E54A30C0
:10BD6400E00122B4061C20540D12BD1612BE72123C
:10BD7400BF0212BF3A221284377E0412DE06754ACD
:10BD8400012220550D12BCF112BEE112BF2312BED6
:10BD94004B221284377E0412DE06754A0522740390
:10BDA40012BBA47870E4F5F7C2B2C2B2A6F708B821
:10BDB40080F3D2B222740312BBA4E4F5F7C2B2C278
:10BDC400B2E5F7D2B222E575F8541F30E40244E03C
:10BDD400F57585722EA2779226E57C543F30E502F4
:10BDE40044C0F55EE57C54C02323F55FE57FC2E7DC
:10BDF40079BCF709A77E22856C6F856B6E856A6DA9
:01BE0400221B
:10BE0500856F6C856E6B856D6A22E4FEFF74077520
:10BE1500A704F5838E8274FFF0DFFD75A7002274F9
:10BE2500067E007FB012BE14E4F55AF55B2275A7B5
:10BE350004758306E55A600A75F00A84E5F0700218
:10BE4500740AC4F58222307720E55A24024002059F
:10BE55005A12BE33E55AF0E573F0E574F0E575F076
:10BE6500E576F0E577F0E578F075A700223077F90B
:10BE750012BE337F1074FFF0DFFDE55A24F5500341
:10BE850012BE9D155AE55AB4FF02055AC3E55A95E7
:10BE95005B50D6755B0080D112BDFB7F0A056D0531
:10BEA5006D12BBC1E4F5F7C2B2C2B2E5F7D2B2304A
:10BEB500E704DF02800512BD3380E2056D12BBC1C8
:10BEC50012BE33E55A24F6F07F06E4F5F7C2B2C296
:10BED500B2E5F7F0DFF4D2B275A70022053FE53FE2
:10BEE500B43C17753F00053EE53EB43C0D753E007C
:10BEF500053DE53DB41803753D000249FE153FE5D6
:10BF05003FB4FF17753F3B153EE53EB4FF0D753E4B
:10BF15003B153DE53DB4FF03753D170249FE05425E
:10BF2500E542B43C0F7542000541E541B43C057559
:0CBF350041000540221542E542B4FF0F18
:10BF410075423B1541E541B4FF0575413B15402262
:10BF5100AC40AB41A842EC75F03CA42BFBE435F0BE
:10BF6100FC7A3C12526BEB28FBE43CFC22E53FC31C
:10BF710013F8AB3E79AEE7800E120D4AE5BE75F0BF
:10BF810005A4FB7800E5BF75F03CA42BFBE435F07C
:10BF9100FC7A1E12526BEB28FBE43CFC2212BF7AA6
:10BFA100AE04AD0312BF6E8C148B13120D54E5BF9A
:10BFB100FF24F650027F01E5BE75F096A4AAF0F9C0
:10BFC100C3ED9513FBEE9514FC924E4B70112011AD
:10BFD1000E30480B75364B3003037536FFD22E30C9
:10BFE1004E02DF1F7A0212526B75A7009004EEEC2D
:10BFF100F0A3EBF0C3E5BF9F04BF0102D2E79005B8
:0BC00100CBF022ED29FDEE3AFE80B5E9
:10DDF30012DDFC12DDFC12DDFC7E0480067E028057
:10DE0300027E017F0080087F6480027F017E00EF35
:10DE13004E6012E4FD0D1D0DEDC394AD40F7EF1FF1
:10DE230070ED1E80EA22753500C200C201C20222D3
:10DEDA00F5D8D2DCE5F520E7FBE5DA540FFEAFD939
:04DEEA0075D80022C5
:10DAE1007F767E06909B8912760A740412DEDA7CB8
:10DAF100007D52125377EFF875F00A84C0F07F76FB
:10DB01007E2312D4C77E29742E12D4DA7E2ED0E061
:10DB110012D4C77E35745612D4DA7F6B7E1190DB36
:10DB21004A12D506E824E04001220423F824E750F4
:10DB310002781812DB3AD8FB227F6CE82411FE79B7
:10DB41000512DE330E0FD9F922071DFFFFFFE0801A
:10DB5100000020C0000038E0000008F0000038F8A4
:07DB6100000020FFFFFFE0C0
:10DB680012DB9030E6022409540F75F00AA4F5156B
:10DB780012DB9030E6022409540F25152212DB909F
:10DB8800540F2275F000800875F044800375F00783
:10DB9800E4206D09D5E0FAD5F0F7D24C229247C2BD
:10DBA800ACE54F623885504FA26E926D859950C290
:10DBB8006FD2ACC24CA2472212DBCAC4FA12DBCA2B
:10DBC8002A2212DB9020E603540F2254072409224C
:10DBD800E612DBDF18E608FAC412DBE5EA540F4464
:10DBE80030F924C6E950112407800D75F00A84C065
:10DBF800F012DBFED0E0443030530975F00085E0C8
:10DC0800E0D5F0FA3099FDC299F599623822E538E5
:10DC180080F2E53812DBDF800812DC00E53812DC20
:10DC280000740D12DC00740A80CE744012DC00749B
:10DC38004080C5742C80C1742E80BD75380080B8B2
:10DF000085A0835383FE438380858384F0758400DA
:01DF100022EE
:10D98F0074A212DF0074A112DF0074A612DF0074FC
:10D99F00A412DF0074C012DF00742512DF0012DA48
:10D9AF001F75C70375C6FC75B90112B5427408120D
:10D9BF00DEDAEE75F020A4FEEF54F80303032E24F5
:10D9CF0092C313FE24EA50027E16EE90DA089325D6
:10D9DF00BCFE24E6501F24E8401B748112DF00EECA
:10D9EF0012DF0012DA2C744012DF00742F12DF00E6
:10D9FF0074AF02DF007E2680E1F7F7F8F8F9FAFB43
:10DA0F00FCFDFEFF00000000010102020203030300
:10DA1F00A8BCA9BDAABEABBFACC7ADC62288BC8986
:0ADA2F00BD8ABE8BBF8CC78DC622D6
:10DD1800C006C007C5F075A7019000007EB7E58C66
:10DD2800240340FA12DD3A1EBEAFF3C5F0D007D087
:10DD3800062275A700EE12DF00741012DF007404CB
:10DD480012DF0085A08343838185838475A7517F73
:10DD580020E0F0E0F0E0F0E0F0DFF6E4F5A7F5848D
:01DD68002298
:10DEEE0075A711900000E4C583F0C58330E2F8F504
:02DEFE00A72259
:10DE3300EF20E723EE20E71F20E61C05A7C45403C9
:10DE4300F583EE5408C42FF582EE5407240983F5B5
:10DE5300F0E045F0F005A7228040201008040201FD
:10DE6300EF20E723EE20E71F20E61C05A7C4540399
:10DE7300F583EE5408C42FF582EE5407240983F585
:10DE8300F0E055F0F005A7227FBFDFEFF7FBFDFEC3
:10D48700FDA42582F582E5F03583F583ED22905FD3
:10D49700B47A0475F00512D4877D05805E7A05801D
:10D4A700027A04547FC0E0C083C082C39420500135
:10D4B700E4905F6412D49A802E9060C27A0580054A
:10D4C70090617F7A0675F00712D4877D07802C7AE2
:10D4D7000580027A06C0E0C083C082C39420500151
:10D4E700E490610F12D4CCD082D083D0E022905E3A
:10D4F700D875F00A12D4877D0A7A07C2D18002D282
:10D50700D1C0A7C082C083C007C006C0E030D10920
:10D5170075A704E493FDE493FAEEFB75A704EBFE0D
:10D52700EAFC7901D9067908E493F5D4E5D423F523
:10D53700D420E01612DE630EDCEA0FDDE1D0E0D086
:10D5470006D007D083D082D0A72212DE3380E8909E
:10D557005E1875F00E12D4877D0E7A0812D50290E8
:10D567005EC075F00212D487E493FDE4A393FACE6C
:10D577002408CE7C0812D5837C06AD02ED23FD205E
:0ED58700E00712DE630FDCF42212DE3380F7C1
:10D37200F5D2C2D58036F5D2D2D58030F5D224F698
:10D3820050090E0E24A650030E0E0EE5D2F5D275EC
:10D39200F0648485F0D3C2D57009D2D5742012D43A
:10D3A200DA800312D4C7CE2406CEE5D375F00A8400
:10D3B20085F0D3700A30D507742012D4DA800312B4
:10D3C200D4C7CE2406CEE5D312D4C7E5D222F5D2F5
:10D3D20075F0648485F0D3C2D58022F5D2C2D5809F
:10D3E20025F5D2D2D5801FF5D275F0648485F0D3AD
:10D3F200C2D57009D2D5742012D4DA800312D4C0F7
:10D40200CE2405CEE5D375F00A8485F0D3700A30B8
:10D41200D507742012D4DA800312D4C0CE2405CEEC
:10D42200E5D312D4C0E5D222F5D2C2D58035F5D2E9
:10D43200D2D5802F30E70DF404C0E0742D12D4A8A9
:10D442000E0ED0E0F5D275F0648485F0D3C2D570AB
:10D4520009D2D5742012D4A8800312D495CE240404
:10D46200CEE5D375F00A8485F0D3700A30D50774FF
:10D472002012D4A8800312D495CE2404CEE5D31270
:05D48200D495E5D22263
:1075EF00909E761275F802DD187E00800E7405FEEF
:1075FF00F51EE4FFF51DF51F203C3375A700E4933E
:10760F00700122A3B40204051D8003B4010A051FF3
:10761F00EF2409FFAE1E80E612D4DA7D06B44002D5
:10762F007D03B421027D02EE2DFE80D27E0075A770
:10763F0000E493700122A3B40204051D8003B4017A
:10764F000F051FEF2407FFAE1E80E612D4A480089B
:10765F00B45B0050F612D4A80EB4210280D30EB43E
:10766F00400280CDB42C0280C80E0EB45F0280C1E0
:10767F00B45B0040BC0E0E80B8E60812D4DAEE24DC
:10768F0006FED513F422909BB7307409909BBB3044
:10769F007303909BC002760A75F019D5E0FDD5F003
:1076AF00FA12479212DC32744F12DC43744B12DC25
:1076BF0021C322C250127706124792D2AC12DB8B33
:1076CF00304C1212DB8B304C0C12DB8B304C06D251
:1076DF0050C2ACD322B440E512DB90B4400312DBAE
:1076EF0090B44FED12DB90B44BE712DB9012DB90AE
:1076FF0012DB90C2ACC32230530975F008D5E0FD00
:10770F00D5F0FA227F0575F019D5E0FDD5F0FA1204
:10771F00479212DC32745712DC43745012DC00743F
:09772F008112DC00E56312DC00AC
:10773800E56212DC0078D0E612DC0008B8D7F8E67B
:10774800F8795F30E702792FE912DC0012DC0012C9
:10775800DC0012DC00745812DC00744312DC00E414
:1077680012DC00E8C2E775F00A84C425F012DC00D8
:107778007864E612DC0008B869F8E612DC211276B3
:10778800C2400122DF02800A20508B75F000808001
:10779800D250C2ACD322127706C250124792D2AC52
:1077A8002002EF12DB8B204CE7B440F412DB90B4DC
:1077B800400312DB90B457DAF53812DB90B450D29C
:1077C80012DB9012DB90F56312DB90F56278D01231
:1077D800DB90F924A0500353015FE924E0400279CB
:1077E8005FA60108B8D8E8780612DB90D8FB12DB50
:1077F80090FC53040FC4540F75F00AA42CFC249C6D
:1078080050027C0078D78601E4B92F02D2E72CF623
:10781800786412DB90F608B86AF812DB90E53860F5
:107828000302779A12DB9012DB90C2ACC32290A2BB
:10783800B08003909EBA7F2012763B12DD1802DEDC
:1078480004753400C26B12790512DE04127CB5E5AA
:10785800166003127861020259127F17121D8912ED
:10786800DD1810002010010280F8127D205013123C
:107878001D9412783610000D10010280F8121D3682
:0578880080D7127AA573
:10788D0022C26BD22775480A122ABA753400127DAE
:10789D00EDC26A123312106A0512024A80ED12020D
:1078AD004A127C47127D9F127DF978D0E6642660DE
:1078BD0044127F17121D8912DD18100038100102B5
:1078CD0080F8127D20501BE965156018121D941269
:1078DD00783612DDFC10001D10010280F8121D36E5
:1078ED0080BCD26B127DCB751607855917122B33C1
:1078FD007535008096020259127CB5127927127DDA
:10790D00F97F1912794190A2DD7E1212763D7E2308
:10791D00E51602D44690A42A80EF7862E4127938F5
:10792D0078D0745F12793818E4F6227F08F608DFF4
:10793D00FC227F7B7E007810742012D4A8CE240404
:10794D00FED8F5227F197E0812763D7E28909E9CEA
:10795D00305303909EA102763DC26B1279271279A6
:10796D0071020259C251127DF990A2D512795112AC
:10797D001D5C127CB57F2012791012DD18E5167092
:10798D000512DDF9803675A6FF3051031276B0125F
:10799D004792D2AC200025306DFA1277A1400C121F
:1079AD007D204011127AA5D25180BB105003127860
:1079BD003BC25180D1D25112783680CAC2AC22D28C
:1079CD002775480A122ABA753400C26B127DEDC2B2
:1079DD006A123312106A0512024A80EB12024A1221
:0D79ED007C47127D9F127DF91279FD50DA62
:1079FA00020259909EB5127951121D6E12DD18C3FA
:107A0A0010001310010510020E80F41277134001C2
:107A1A002212783B80DDD3C2AC22D227C26B7548D2
:107A2A000A122ABA753400127DEDC26A1233121094
:107A3A006A0512024A80EDD26B127C47127D9F12B0
:107A4A007C6F75B901E5BCB2E7F5BC124E2C751610
:107A5A0007855917122B3380CB127CB5E516601FA8
:107A6A0078D0E53D127A96E53E127A96E53F127A8B
:107A7A0096765A08765F12C7AF127DCB027C867F54
:107A8A003E7E11909E8C12760A02DD1875F00A84E9
:107A9A004430F608E5F04430F60822D26B127DCB6A
:107AAA00127C86E51775F01084240AF54824E850FC
:107ABA000375480A122AC68558592275320012BE21
:107ACA000F75A704900700751500127C6F75B90130
:107ADA00E5BC20E705E515F0801004600D648260BE
:107AEA000975BCFF75B90575B9020515E515242098
:107AFA0050D8E58224FE4003027B9EA882187F00AC
:107B0A0075A7007583078882E0FE75F004A4127CCD
:107B1A001AA9BCAABDABBEACBF1582E0FD75F004C4
:107B2A00A4127C1AC3E995BC404C7052EA95BD4038
:0D7B3A0045704BEB95BE403E7044EC95BF8E
:107B47004037703DEE75F004A404127C1AA9BCAA54
:107B5700BDABBEACBFED75F004A404127C1AC3E93B
:107B670095BC4015701BEA95BD400E7014EB95BE91
:107B77004007700DEC95BF5008EEF00582EDF0154B
:107B870082E5826009C3EF95825003027B120FC31F
:107B9700E89F4003027B0A75A70490070075C70397
:107BA70075C6A8E0F5BCE0F5BDE0F5BEE0F5BF752C
:107BB700B90575B90205C6E58224204006E5C62445
:107BC7002050E00875C70375C68075B901E5BC127A
:107BD7007C04F5BCE5BD127C04F5BDE5BE127C0452
:107BE700F5BEE5BF127C04F5BF75B90205C6E5C64B
:107BF700245850D6E5320470FB75A70022B4FF0164
:107C070022F975A704900700E582686005E06970AE
:107C1700F7E922F5C685F0C775B901E5BC645F7061
:107C27000375BC27E5BD645F700375BD27E5BE64BA
:107C37005F700375BE27E5BF645F700375BF2722BA
:107C470075C703E54875F004A42480F5C6E55975A2
:107C5700F00484A8F00825C6F5C675B901A9BCAA21
:077C6700BDABBEACBF8615EA
:107C6E0022E515242050037515DFE51575F004A4E3
:107C7E0054FCF5C685F0C722E51724204028E517E9
:107C8E0075F00484A8F00824A8F5C675C70375B965
:107C9E0001A9BCAABDABBEACBFA61589BC8ABD8B63
:107CAE00BE8CBF124E2C22E4F516F51579FF127C10
:107CBE006F75B901E5BCB4FF040516A9150515E5E8
:107CCE0015242050E9891579FF75C70375C6A87567
:107CDE00B90109E5BC04601B09E5BD04601509E5A1
:107CEE00BE04600F09E5BF04600905C6E5C6242081
:107CFE0050DD09891722751600751501127C6F75F6
:107D0E00B901E5BC20E70205160515E5152420503E
:107D1E00EB227900E975F004A454FCF5C685F0C792
:107D2E0075B901E5BC20E73078D066702B08E5BD4B
:107D3E0066702508E5BE66701F08E5BF66701905FA
:107D4E00C675B90108E5BC66700E08E5BD6670081B
:107D5E0008E5BE667002D32209E9242050B6C3227C
:107D6E00127D8E127D76A8017F08E0F608DFFB22D9
:0B7D7E00127D8E127D86A8017F08E6B2
:107D8900F008DFFB2278D0796275A704758307EBC9
:107D9900C454F0F58222127C6F78D0127DB9E5BC0B
:107DA900F9C23C20E702D23C127DB97862127DB952
:107DB90075B901A6BC08A6BD08A6BE08A6BF0805D8
:107DC900C622127C6F78D0127DDB127DDB786212BD
:107DD9007DDB86BC0886BD0886BE0886BF08124EB4
:107DE9002C05C62212593E12DEEE12857902DD18E3
:107DF90012DEEE7F007E0990A2C212760A7F0A7E09
:107E090012E5150412D37E7F1412C999121D367F0B
:107E1900277E0875130778D0127688E6793E30E711
:107E290002792F7E34E912D4DA7F3D7E0190A4468F
:107E390012763D20311B3030031290B4C23B1280C0
:107E4900A9127E5FD23B1280A9127E711280F08046
:107E59007C12C00C80E6C23B7F4474532017027425
:107E69004E7E0012D4DA8017D23B7F4F7457201709
:107E79000274457E0012D4DA7E06E51E12D4C77E4E
:107E89000CE51D12D4C77E12E51C12D4C77E1774E7
:107E99008112D4DA7E1CE51B12D4C77E22E51A12A0
:107EA900D4C77E28742E302602742712D4DA7E2D88
:107EB900E51912D4C77E33E51812D4C77E393026A6
:0F7EC90007742C12D4D67E3BE53702D4C7742D34
:107ED800201702742B7F707E1512D4DA127EF47E7E
:107EE8003A12D3277E0190A47102760A7E1BE51C04
:107EF80012D4C77E21E51B12D4C77E27E51A12D4F7
:107F0800C77E2DE51912D4C77E33E51802D4C712EF
:107F18007F95127FC0128297127DF91282EF201787
:107F28001E10021B12483312C7AF127F7D121D416B
:107F38007F347E2F127695127E3212DD1880E2127F
:107F48001D36203026203128C23B1280A9127FD549
:107F580078661281A9D23B1280A9127FEA78691249
:107F680081A91280F012806402824C12917D80F205
:107F780012C02180EDE57D75F01084AAF075F00A35
:107F8800A42A547FFA78D7E654802AF6227F277EDF
:107F98000879D08700C001D224B9D002C224128344
:107FA80076D001A70010230909EE2406FEB9D7E30D
:107FB8002219EE24FAFE80DB7E3479D7E7A2E79215
:107FC8001712832379D7E7A21792E7F722C224C2B0
:107FD8003B751E007F447E00128333801E1023ED04
:107FE800802AD23BC2247F4F7E0012833BD2247E5C
:107FF80006E51E128368F51E1023E7D2247E0CE5E1
:108008001D128368F51D303BD41023E1D2247E1263
:10801800E51C128368F51C1023E17E1CE51B128306
:0380280068F51BDD
:10802B001023E67E22E51A128368F51A1023E87EE8
:10803B002DE519128368F5191023E87E33E5181224
:10804B008368F5181023E87E393026027E3BE5372E
:10805B00128368F5371023E3227F707E1512832B72
:10806B00C2247E1BE51C128368F51CD2247E21E5FD
:10807B001B128368F51B1023E77E27E51A12836812
:10808B00F51A1023E67E2DE519128368F5191023D6
:10809B00E87E33E518128368F5181023E82278D7A9
:1080AB00E6C2E775F00A847866F537303B057869E8
:1080BB0085F03712811930262BE53775F003A404B0
:1080CB000475F00584FBE51975F00AA4251875F005
:1080DB0006A42BFBE435F0FC12548DF53712548DAE
:1080EB00F5188B1922E563FC339217AB6250031220
:1080FB0054FE305C0A7AD2125279784012541BAE7D
:10810B0004AF037C277D101253848F1C8037E6FD50
:10811B0033921718860418860350031255067A09F2
:10812B00792778C01254188B1EADD3ACD2AB06791D
:10813B00EA78601254168B1DAF06AED27C177D7099
:10814B001253848F1CAF05AE047C037DE81253845D
:0F815B008F1BAF05AE047C007D641253848F1A16
:10816A00ED75F00A84F51985F01822EC3392175050
:10817A00031254FE751D30301786751D2D808178C7
:10818A00427B607CEA800678407B207C4E12C0EC01
:10819A00792778101254168B1CAF06AED280AB30FA
:1081AA00262AE51975F00AA4251875F00AA42537B8
:1081BA00FBE435F0FC7A0512526B8C068B077C00C7
:1081CA007D031253778E048F031280E3E51E75F048
:1081DA000AA4251D75F00AA4251C75F006A4251B02
:1081EA00FBE435F0FC7A0A12526BEB251AFBE43CED
:1081FA00FC7A0A125279EB2519FBE43CFCE43DFDBA
:10820A007A0A12528BEB2518FBE43CFCE43DFD3064
:10821A001703125506A60518A60418A60378D7E66A
:10822A00A2E7923DC2E775F00A84FCABF0303B0E40
:10823A00AB37EC75F00AA42BA23D92E7F622AC37D5
:10824A0080F0128267305C0A7A4012527978D21230
:10825A00541B3017031254FE8C638B6222128277EE
:10826A007A0A12526BEB2518FBE43CFC22E51C75DA
:08827A00F00AA4251B75F00AAF
:10828200A4251AFBE435F0FC7A0A12526BEB25198D
:10829200FBE43CFC221282C912DE00C202C223129B
:1082A20082C910000810010510021B80F51031ED83
:1082B20010300D102604D22680E3D230C23180DD88
:1082C200D231C23080D7227F3590A42F12763B90D4
:1082D200A44D20300F90A46920310990A43E20269D
:1082E2000390A4361F7E1712760A02DD187F357EB0
:1082F20001909E6912763D7F347E3A128418744E44
:1083020012D4DA12DD1812DE00C2027F347E3AD2B3
:108312001775115975124E802675112E7512278008
:108322001E75113E75122F801675112B75122D8038
:108332000E75114E7512538006751145751257123E
:108342008418E511301702E51212D4DA12DD181082
:10835200000810010510020B80F5D23C1017E3D281
:108362001780DF0284134430F8128372E8540F221C
:10837200C2218002D221A22492229223128418E8DE
:1083820030E709D23C7430302102745FF812D4DA3B
:1083920012DD1810003410010510025D80F5D23C88
:1083A200102266102367B43909745F2021DF74300C
:1083B20080DBB45F04742D80D4B42D04744180CD6D
:1083C200B45A04743080C60480C3D23C30240610F0
:0F83D2002237102338B44104742D80B1B42D0428
:1083E100745F80AAB45F04743980A3B43009745AED
:1083F10020219B74398097148094B48908D223E892
:1084010012D4DA800DF8C223800874898001E80251
:10841100838F90842D8003908429C007EF2408FF67
:1084210012D506D00702DD180205F8F80205000092
:10DCB80075A70090DCEA75F02D84C2D5C2D1601733
:10DCC800D2D1146007D2D514600DC2D1E5F093FC0F
:10DCD800742D95F093FB22E5F093FB742D95F0934A
:10DCE800FC220009121B242C353E474F58606870EF
:10DCF8007880888F969DA4ABB2B8BEC4CACFD4D959
:10DD0800DEE2E6EAEDF0F3F6F8FAFCFDFEFFFFFFCF
:10DDB200D23D8002C23DED8BF0A430E70205F0C3F4
:10DDC200E895F020D50425F025F0FEED8CF0A43086
:10DDD200E70205F0C3E995F030D10425F025F0FF04
:10DDE200203D0B2487500122EF24CC40012202DE89
:01DDF20033FD
:10D75600203A7A7E1C7F5312DE337F5912DE331E47
:10D766007F5712DE337F5512DE337E2312DE337F80
:10D776005712DE331E7F5912DE337F5312DE331FFC
:10D786007E2012DE337F5A12DE337E1E12DE337F98
:10D796005212DE33120D54E5BD20E0143006117F1F
:10D7A600357E1C90D812E571700390D81C02D50600
:10D7B600E5716018E57012DCB8781F79567D09129C
:10D7C600DDB6303A0312D7E50DBD16F3227E1C7F77
:10D7D6005390D7FB12D506200CD612C9F580C0C0CF
:10D7E600060E30D5021E1E12DE33D0061F30D102C1
:10D7F6000F0F02DE33070700386C446C380005054E
:10D806002070D8702005057088A888700807103821
:10D816007CFE383838000807102844C62828380007
:10C7D40090A47B7F717E2312763D120D54E5BC7EBE
:10C7E4003112D49530121AC23C120D54E5BCFB75BB
:10C7F400F00AA4F904FAC23D12BDFB12CA72303D1C
:10C804000122DAF712C9797C00EBF4042E4019AD49
:10C8140003125377EFA2D1203C077E237F6502D019
:10C82400F4AE16AF1702C91AAD01125377EF12D145
:10C83400E2203C077E237F6502D118AE16AF1702B3
:10C84400C93E7F567E0512C9A57F3D12C9B87F6FC8
:10C8540012C9B812C9F57E0A7F4112CA287E227F06
:10C864005912CA282012012212BDFB857A1D855E49
:10C874001C857B1B855F1A7AC0C23D12CA6E203D9F
:10C884005212C9797C007D1412537774562F20D12B
:10C89400029F9FFF24CB40028037EF248850028000
:10C8A40030EA1475F00384FE12DE33C3E51B957B76
:10C8B400FEE51A955F92D55004EEF404FEEEC31320
:10C8C400FE24E0400C741F2E30D5029E9EFE12DE24
:10C8D40033DAA8227F5212C8EA7F5A12C8EA7517BF
:10C8E40053751600802B7E0012DE630EBE12F922F1
:10C8F4007F157E28742012D4DA7F1C7E2812DE6312
:04C904000EBE40F92A
:10C90800223012E712C8F475171575162DD23C029D
:10C91800C7EDC23D6002D23D92D175F080305C0413
:10C92800F5F08001A4A2E792D5E5F075F03284F81D
:10C93800E5F075F00584C0E0E5F0A2D533C0E0E885
:10C94800601E12D4C7EE2406FED0E0F8D0E012D460
:10C95800C7EE2406FE742C12D4DA0E0EE802D4C7F1
:10C968007420303D07742B20D102742D12D4DA8044
:10C97800D4C3ED957AFFEC955EFE92D15003125424
:10C98800EE227F1512C9917F327E3E12DE33DEFB26
:10C99800227E0912DE330EBE36F9227E0112DE3304
:10C9A8000E0EBE3FF8227E3312DE330EBE40F92251
:10C9B8007E047D1112DE330E0E0EDDF81F1F7E354C
:10C9C80090A484305C057E3190A48802763D74057D
:10C9D800305C097E32740112D49574067E3612D406
:10C9E800957E3A740012D4957E3D02D4957F417E9F
:10C9F8001F7D0F12DE330F0F0FDDF8227F687D03D6
:10CA080080047F677D0512DE330FDDFA227F667DA5
:10CA18000780F37E1F7F5012DE331F1FBF3EF822B0
:07CA28007D0A12DE330E0E41
:10CA2F000F0FDDF722203D07123BB97003D23D22D5
:10CA3F00056D12BBC1E4F5F7C2B2C2B2ABF7F5F7A1
:10CA4F00C2B2C2B2E5F7FA30E411EB251DF51DE4D1
:10CA5F00351CF51C0519EA30E3010ED2B2801578AA
:10CA6F000380027801203D07123BB97003D23D22AB
:10CA7F00D8F3056DE56D2409F56D12BBC1E4F5F72B
:10CA8F00C2B2C2B2ADF7F5F7C2B2C2B285F71BF5AB
:10CA9F00F7C2B2C2B2E5F7FCD2B2543F30E502445E
:0FCAAF00C0CC54C02323F51AE56D24F6F56D2293
:10D67D007E017F0990D6FB12D5062051097E037FCE
:10D68D0000743F02D4DAE4FEFFC3E54512CD44FD3C
:10D69D00940AED403D9464ED4002746312D3787E9C
:10D6AD00017F09E552240575F02D84AAF075F0056A
:10D6BD00A4CA75F00B842A90D6E69312DCB8BCB8D8
:10D6CD00027BB87D04EE2DF8EF2DF90D12DDB2DDE4
:10D6DD00FB227E0312D4C780C6000C1622222D39E0
:10D6ED00444F4F5A66707C7C87939EA9A900090907
:10D6FD00080041000000000088800000000041008B
:10D70D000800120D68E5BCB4F8339004C3E0602C3A
:10D71D00FA24F340277F137E0012DE330F0F12DE43
:10D72D00330E12DE631F1F12DE630EDAEC7F147EE2
:10D73D000012DE330E12DE630EBE12F5229005CC02
:09D74D00E0C3941240F60480C709
:10CD4400305D0A75F08AA42480E5F0340022207452
:10CD5400157F017E1190CDCC12D5067F0A7E0AE59F
:10CD64002E540702D38F7F087E1190CDDC12D50696
:10CD740020730C7F0A7E1712DE630E0E12DE637FB1
:10CD8400007E0BE57112CD4412D37E7F0C7E11E53B
:10CD940071602F0EE57064B4602864B475F0328459
:10CDA400C0F012D4C0CE2405CED0E075F00584C006
:10CDB400F012D4C0CE2405CED0E023302D010402DD
:10CDC400D4C090877502760A070FFFFFC473BDAF06
:10CDD400A463B5FBCDE7FFFF030F0100FFFE038053
:10CDE400306701227F3F7E00748812D4DAE55160F7
:10CDF400F2120D6D85BCF01207E012CD4475F0649B
:10CE040084F87E06E5F012D3DDE860D77E0002D414
:10CE1400C7120D6DE5BE70012214600814603BE575
:10CE24003F1340367F367E00747712D4DA207301C4
:10CE34002279BC87040987031252137E05781DE604
:10CE440060097E0012D4C0EE2405FE18E6600712C5
:10CE5400D4C0EE2405FE18E68019909D3B7F377EF2
:10CE64000012763DAB60AC611252161F7E09781D2C
:10CE7400E6600712D4C0EE2405FE18E612D4C0EE14
:03CE84002405FE84
:10CE870018E602D4C0202C012290CE9602D50605C2
:10CE97000EFFF0E01CF004F81CFFF0301201227FB7
:10CEA700637E00909BD212D5067F1512C9917F1F12
:10CEB70012C9917F2912C9917F177E06E53F30E09D
:10CEC7000B90A498305C0390A4AC80132074077E69
:10CED70001909BF2800990A48D305D0390A4A2126B
:10CEE700760A307306E54E6002154E205718E54E58
:10CEF700B40113120D77C3E55C9560F5BCE55D954C
:10CF070061F5BD124E2C7F217E01E53F30E02130D7
:10CF17005705909D198016E54E7005909D24800D4C
:10CF2700909BFE12760A7E30E54E02D3E312760A14
:01CF370022D7
:10D24A001252137F207E05751900781DC2D5E6306B
:10D25A00D51712D4C0EE2405FE18B818F17E1F7433
:10D26A0063305C02748202D4DA7005B8191880E25D
:10D27A00D2D5CE24FACE7484301702742D12D4DAA1
:10D28A00EE2406FE80C8742012D4D680C8781C808A
:10D29A000D7F007E23AC5EAB7A125213781DC2D585
:10D2AA00E630D50C12D4C7EE2406FE18B818F122BF
:10D2BA007005B8191680EDD2D53017E4CE24FACE0F
:10D2CA00742D12D4DAEE2406FE80D5742012D4DA34
:10D2DA0080D5125213781DC2D5E630D51612D495D0
:10D2EA00EE2404FE18B818F10E745E305C0274273E
:10D2FA0002D4A47005B8191680E3D2D53017DACE55
:10D30A0024FCCE742D12D4A8EE2404FE80CB742003
:10D31A0012D4A880CBC23D12D3320F0F0E0E746303
:10D32A00305C02748202D4DA125213781DC2D5E636
:10D33A0030D50C12D4F5EE2408FE18B818F1227074
:10D34A0005B8191680EDD2D5301716740BCE24F80D
:10D35A00CE12D4F5EE2408FE80D5740C12D4F580D2
:08D36A00D5303DCB740A80E5CB
:10D826007F797E24E55F30E70122AC5F1CAB7B127B
:10D836005241E51B700E742012D4DAEE2405FE1256
:10D84600D874800C12D874E51B12D4C0EE2405FEE1
:10D85600E51A12D4C0EE2405FE742C12D4DA0E0E8C
:10D86600E51912D4C0EE2405FE745E02D4DA742DD6
:10D87600201702742B12D4DAEE2406FE22E55F305E
:10D88600E70122AC5F1CAB7B125241E51B700E74A4
:10D896002012D4A8EE2404FE12D8CD800C12D8CDC6
:10D8A600E51B12D495EE2404FEE51A12D495EE2457
:10D8B60004FE742C12D4A80E0EE51912D495EE248B
:10D8C60004FE742A02D4A8742D201702742B12D4D5
:06D8D600A8EE2404FE226E
:10D0E4007F097E2530040512D1DE8028A275E579FA
:10D0F400C23D6002D23D92D175F080305C04F5F0FF
:10D104008001A4A2E792D5E5F075F03284F8E5F049
:10D1140075F00584C0E0E5F0A2D533C0E0E8602AEC
:10D1240012D4F5EE2408FED0E0F8D0E012D4F5EEE7
:10D134002408FE0F0FE52B5403701F746012D4DA19
:10D144001F1FEE2404FEE802D4F5740C303D06746F
:10D154000A20D1010412D4F580C9205904742E8008
:10D16400DC205804747F80D5748080D1300405128B
:10D17400D1DE8028A275E579C23D6002D23D92D10C
:10D1840075F080305C04F5F08001A4A2E792D5E547
:10D19400F075F03284F8E5F075F00584C0E0E5F050
:10D1A400A2D533C0E07F3E7E1CE8602012D556D065
:10D1B400E0F8D0E07F3E7E2812D5567F447E32745C
:10D1C4002E12D4DA7F3E7E37E802D556303DE07425
:10D1D4000A20D1010412D55680D59005CAE075F015
:10D1E4000A84F8E4C5F0C2D522301105E54AB40238
:10D1F40050C39006E9E0957AFB9006E8E0955EFC62
:06D2040050031254FEEC81
:10D20A00C31360047B63800FEB13FB249C40F5245B
:10D21A004F4004C20480079005CAEBF0D20490067E
:10D22A00E6E09006E8F09006E7E09006E9F0E55EB1
:10D23A009006E6F0E57A9006E7F02212D22880DE20
:10CABE00E54424F64001227800E552206607C3952E
:10CACE0070500224B40475F00384F9E928FE24C4DE
:10CADE005001FE12CB0012CB0C1E12DE33C3E998AE
:10CAEE00FE5003243CFE12CB001E12DE3308B81F8C
:10CAFE00DA22EE2420FE24C250032402FE22E82471
:10CB0E00F1E8C2D55006D2D5E8F4241F23FF90CB0E
:10CB1E008E93CF0493FAE545F5F0A4ACF0FB1252D8
:10CB2E00A2E544F5F0A49BFBE5F09CFCEB2420FB76
:10CB3E00EC3400FC12CB6FFAE5458FF0A430E7021F
:10CB4E0005F0E5F020D502F4042A75F0052019034E
:10CB5E0075F00384FF24DF50027F20C374329FFFE1
:10CB6E0022EC24F0500BEB2460EC340090CBDE93DF
:10CB7E0022EB33FBEC33FCEB33EC3390CBAE932256
:10CB8E00FF00FF03FA0BF318EA2ADE40CF58BE73FC
:10CB9E00AB8D96A880C068D64FE835F51BFD00FF1B
:10CBAE0000080B0E101214151718191B1C1D1E1F32
:10CBBE0020212223242526262728292A2A2B2C2DFC
:10CBCE002D2E2F2F30313132333334343536363734
:10CBDE00373839393A3A3B3B3C3C3D3D3E3E3F3F90
:10CBEE004042444648494B4D4E5052535556585963
:10CBFE005B5C5D5F60616364656668696A6B6D6EE0
:10CC0E006F7071727374767778797A7B7C7D7E7FA4
:10CC1E00808182838485868788898A8B8B8C8D8E92
:10CC2E008F9091929394949596979899999A9B9C9C
:10CC3E009D9E9E9FA0A1A2A2A3A4A5A6A6A7A8A9B9
:10CC4E00A9AAABACACADAEAFAFB0B1B1B2B3B4B4E8
:10CC5E00B5B6B6B7B8B9B9BABBBBBCBDBDBEBFBF22
:10CC6E00C0C1C1C2C3C3C4C5C5C6C7C7C8C8C9CA67
:10CC7E00CACBCCCCCDCECECFCFD0D1D1D2D2D3D4B5
:10CC8E00D4D5D5D6D7D7D8D8D9DADADBDBDCDDDD0B
:10CC9E00DEDEDFDFE0E1E1E2E2E3E3E4E5E5E6E666
:10CCAE00E7E7E8E8E9EAEAEBEBECECEDEDEEEEEFC8
:10CCBE00EFF0F1F1F2F2F3F3F4F4F5F5F6F6F7F72F
:10CCCE00F8F8F9F9FAFAFBFBFCFCFDFDFEFEFFFF9E
:10CCDE00E54524FD400122E552206607C3957050BC
:10CCEE000224B40475F00384241FFE24C2500324CE
:01CCFE000233
:10CCFF00FE12CD39EEFD241EFE24C250032402FE87
:10CD0F0012CD39E544240275F00520190375F0039F
:10CD1F0084F4042432FF24EE500F12CD2EAE051EE4
:10CD2F001E7C0512DE330EDCFA227F1512DE330F66
:05CD3F000FBF2DF822DA
:10D595007E00206615E5700475F0B484E5F075F03D
:10D5A5000384FE6004C3743C9EFE745312D5C0749C
:10D5B5005712D5C0744E12D5C074457F2F12D4A80A
:10D5C500BE00077E3C12D4A87E00EE240875F03C10
:10D5D50084AEF00F0F0F12DE330E12DE330F12DEA4
:10D5E500331E12DE33EE240775F03C84AEF0223094
:10D5F500745C301259E54AB4040122B4060122E5EF
:10D605007112CB588F057C037E1E30662AE57004A7
:10D6150075F00384241EFE24C6501C24FB500424EC
:10D62500038013C00612D63CD0E024C67C016006F8
:10D635000C1460020C14FE12D6480EEE24C14002F2
:10D64500DCF5228D0712DE330FEF24CE50F722E5ED
:10D6550053206607C39570500224B40475F0038403
:10D66500241FFE24C250032402FE12D6730E7F230C
:08D6750012DE330FBF2DF92274
:10DD6900AF177E00E53C12D3727E0C742E12D4DA02
:10DD79007E12E53B12D3727E1E742E12D4DA7E24F3
:10DD8900E53A02D3727E0E78ADE612D3DD7E1874C1
:10DD99002C12D4DA7E1B18E612D3DD7E25742C12E0
:09DDA900D4DA7E2818E602D3DD6D
:10CF38007F797E00E54012D3DD7E0A743B12D4D699
:10CF48007E0CE54102D3DD7F797E16743B12D4D680
:10CF58007E18E53F12D3DD7F797E0078AEE612D3E6
:10CF6800DD7E0A743B12D4D67E0CE53E02D3DD305A
:10CF78005EE52043E27F6D7E0078AEE612D3DD7E6B
:10CF88000A743B12D4D67E0CE53E12D3DD7F757E43
:10CF98000075F00A84E5F012D4F50F0F7E08743A94
:10CFA80012D4D61F1F7E0DE53F75F00A84C0F0121B
:10CFB800D4F5EE2408FED0E002D4F5851C1E851BAE
:10CFC8001FAB1BAC1C305D0A7A1B125279783212E7
:10CFD800541BC3EB33FBEC33FC923D12524A303DF9
:10CFE800087409F51DF51CF51B7F75E51D60157E98
:10CFF8002412D4F57E2CE51C12D4F57E34E51B12E0
:10D00800D4F5803D7E22E51C601912D4F57E2AE510
:10D018001B12D4F57F787E31742E12D4D67F75E535
:10D028001A8019E51B12D4F57F787E29742E12D444
:10D03800D67F757E2DE51A12D4F5E5197E3512D402
:10D04800F57F777E3C125BD4851E1C851F1B227FD3
:10D05800397E1F12DE330FBF40F9781F79567A00E8
:10D068007D1A12DCB812DDB6EA2406FABAAEF378F5
:01D078001B9C
:10D07900C3E5119570500224B4FA604214603E145D
:10D08900603A2450603A146036EA24A540278A1E83
:10D09900751D007D1912D0A90D30740312D0A90D88
:10D0A900781F7956AA1DEA12DCB812DDB60AD3EA4E
:10D0B900951E40F2228A1D751EB380D708080808FC
:10D0C9007F367E1C90D812E571700390D81C12D55A
:0BD0D900067F3CAE0090842902D506C3
:10DA3900787512DA897453201702744E207406E53A
:10DA49002E54074430AF1712DAB37E3BE57DC45438
:10DA59000F12D4C72074077E07742012D4DA78789D
:10DA690012DA89E5172409FF745720170274452033
:10DA79007402742012DAB37E3BE57D540F02D4C7D9
:10DA8900E6FD3392171886041886033017031255DA
:10DA990006791778701254168B13AF06AED27C0034
:10DAA9007D641253848F148D15227E0012D4DA7E80
:10DAB90007E51312D38F7E19748112D4DA7E20E51B
:10DAC9001412D3727E2B742E2073030E742C12D46D
:08DAD900DA7E2FE51502D3727D
:10DC4800E54A602E7A2420E00E7A26141460087AB9
:10DC580028141460027A297F667E01EA12D4DA2039
:10DC68005505205406800B745B8002745C7E00129C
:10DC7800D4DA20110778A9B60007802130261EC201
:10DC880026909C937F681275F87F66A85AE54AB477
:10DC9800060108E875F06484E5F012CFB120080F9A
:10DCA800E537640260097F367E2E744112D4A822BB
:10D8DC0020144F740512DEDAEF33EE33F9EF030345
:10D8EC00541FF5F090D92FE993A4C5F013C5F0138C
:10D8FC00C5F013C5F013C5F0135403FCE5F013FB8E
:10D90C00E9242093C9244093C39BC4540FFBE99C86
:10D91C00C4FC540FF9EC54F02B2446F57BE934F697
:10D92C00F55F22FFFFFFFFFFE6C5AD9C8F857D777E
:10D93C00726E6C6A696A6A6C6F747A828D9DB4D9E6
:10D94C00FFFFFFFAE9DCD3CEC9C6C3C0BEBBB9B773
:10D95C00B5B4B2B0AFADABAAA8A6A4A2A09E9C9938
:10D96C0096918C00381CE735D137246F00C5B3C1B4
:10D97C00E61F66B60E68C21867AADBF4EDB94675E9
:03D98C0010A200E6
:10DEBA00D2A27408D2A1D2A300C2A3C2A1D2A30043
:10DECA00C2A3D5E0EF7405D2A300C2A3D5E0F8221D
:10DE9300C2A3D2A2D2A1D2A300C2A375F008339227
:10DEA300A1D2A300C2A3D5F0F5C2A175F003D2A3FA
:07DEB30000C2A3D5F0F82224
:10C3F50012DE93D2A300C2A3C2A175F008E4D2A3B2
:10C4050000C2A3A2A233D5F0F5FE75F008E4D2A3CD
:10C4150000C2A3A2A233D5F0F5FFD2A300C2A32286
:10C42500E478806608B88BFB70012274D512C3F5D9
:10C435007881C3EE13FEEF13F692D118EE2460F661
:10C4450074D612C3F57888EF33CE33CE33CE33CEE0
:10C4550033A2D192E25407FCEEFB7A0812526BEC40
:10C46500244FF608EBF674D912C3F5EF543F7882E2
:10C47500F67886EF33CE33CE33CE33CE335403F650
:10C4850008EEF618161608E6C4FF54F0F618E6C4CA
:10C49500CF540F2FF674DA12C3F5EF232354FC782B
:10C4A50083F67884EEF608EF54C0F67880E46608E3
:10C4B500B88AFBF62212C3FD7889C3EF96FF18EE02
:08C4C50096FEA2E7921650104A
:10C4CD001254EE740FF8F91252B8EF2CFFEE3DFE38
:10C4DD00788BEEF608EFF622E6182016072CF7E615
:10C4ED003D19F722C39CF7E69D80F66A405E8056A3
:10C4FD00E050F04B0044803DC0384031D02BA0259A
:10C50D00601F2018D014000F000AA001440158012B
:10C51D00680178018801A001B401D001EC0210027C
:10C52D0038026802A002DA030C034D78BE80208524
:10C53D008E8A9D8F4D95BA9A97A0BEA631AC53B2F7
:10C54D002AB801BD6AC1EDC4D1C78812C3FD788D6B
:10C55D00EEF608EFF67887798C1252B878837990D9
:10C56D0012C4E57885798C1252B87881799212C40B
:10C57D00E5788DE624E4FE08E63392D13392D55466
:10C58D00FCFFEEA2D133A2D533FE780F7992125271
:10C59D00B878947990C3EC97F61819ED97F67994CD
:10C5AD0090C4F87F1F7D11EF93C3971F19EF9397D9
:10C5BD001F091DED600240EF0F90C518798DEF93A7
:10C5CD00F7090FEF93F7788E79941252B890C5381A
:10C5DD00EF93C39BFB1FEF939C2420FC7897E62BD6
:10C5ED00F618E63CF618E436F6740612DEDAD237A3
:09C5FD00EE24F74006240250026E
:10C60600C237EEFCEFFD740712DEDAC3ED9FFFECD6
:10C616009EFE78B7E6FD337C0050011CEF2DFFEE41
:10C626003CFE789CEF26F618EE36F62220141220F1
:10C63600370F789DE6B4050912C6E312C71812C76C
:10C6460061222014577897799A12C792125476C3AA
:10C65600EE9420FE924550031254EE7C007D0512A6
:10C6660053843045031254EE8E618F60E531B40C6D
:10C676002B12DA1FE56120E71124F8500DFAC3E505
:10C68600609AF560E5619400F561120D77E5BC25C9
:10C6960060F57AE5BD3561F55E12DA2C7897799A00
:10C6A600C3E697FB1819E697FC7A0212526B3037ED
:10C6B6000B7A0212526BECFEEBFF800312C6E312FA
:10C6C600C71820140312C76178957998E6F77600A3
:10C6D6000809E6F776000809E6F7760022799CE76E
:10C6E6007700FB19E77700FC789DE6B40506EB3387
:0EC6F600FBEC33FCECA2E792D550031254FE8D
:10C704007A32125279ECFBEDFC30D5031254FEEC74
:10C71400FEEBFF22EE2408FE740420371674063064
:10C724007511789DE6B40504740C8007F42406C3DF
:10C7340023540FFD7C00125257789FE6FC08E6FB59
:10C74400C374109DFA125279EFF8EEF9125476E898
:10C7540078A02FF6FF18EE39F62480FE2292754059
:10C76400031254EE78BBE6F5F02438400375F0E18B
:10C77400EF33EE3378A8F6A485F07930E702057933
:10C78400C276307508E57924F15002D27622E62784
:10C79400FB1819E637FC1819E637FD2212BDA27FF3
:10C7A400087871793A12C7BB0249FE855E63857ABF
:10C7B40062787379647F06E6F70809DFFA22786401
:10C7C400797380F1787379AF80EB78AF797380E512
:1051F100E4FEFFFC7D0A791DE7540F2FFFE43EFE1C
:10520100B9190280061912525780ED301703125452
:10521100EE22305C2BEC33921750031254FEEC2437
:10522100D950047C277B007AD2125279EB33CC33EC
:10523100CD33CC33ED33FBEC33FC3017031254FE8A
:10524100EC33921750031254FE791912548DF70959
:10525100B91DF8A70322EFF88DF0A4FFEDC5F0CE3C
:10526100A42EFEEC88F0A42EFE22EB8AF0A4FBE52E
:10527100F0CC8AF0A42CFC22EB8AF0A4FBE5F0CC64
:105281008AF0A42CFCE435F0FD22EB8AF0A4FBE5C6
:10529100F0CC8AF0A42CFCE435F0CD8AF0A42DFDED
:1052A10022EB8AF0A430E70205F0E5F0CC8AF0A405
:1052B1002CFBE435F0FC2286F0E7FDA4FAABF019F3
:0652C100E786F0A42BFBC0
:1052C700E435F0FC18E68DF0A42BFBEC35F0FCE49C
:1052D70033FDE687F0A42CFCED35F0FD22EB89F0D9
:1052E700A4CBAEF08AF0A42EFEE5F03400FDEC89E5
:1052F700F0A42EFEE5F03DFDE433CC8AF0A42DFDAD
:10530700E5F03CCEFC22EB89F0A4CBAFF08AF0A409
:105317002FFFE5F03400FEEC89F0A42FFFE5F03E07
:10532700FEE433CC8AF0A42EFEE5F03CFCED89F0D8
:10533700A42EFEE5F03CFCE433CD8AF0A42CFCE57A
:10534700F03D8E058C068F04FF22C2D5EC30E705B1
:10535700B2D51254F6EE30E70DB2D51254EE125311
:10536700841254F6800312538430D5031254EE226C
:10537700C3EC13C0E0ED132FFFD0E03EFEBC000BE3
:10538700BE0029EF8DF084FFADF022E4CCF975F073
:0453970008EF2FFFED
:10539B00EE33FEEC33FCEE9DEC994005FCEE9DFEEE
:1053AB000FD5F0E9E4CEFD22EDF9F5F0EE8420D235
:1053BB001CFEADF075F008EF2FFFED33FD400799A4
:1053CB005006D5F0F222C399FD0FD5F0EA22EC334B
:1053DB00EE3400FEEF3400FF7D007A00790078098F
:1053EB00C3ED9AFDEE9BFEEF9CFFB392D54009ED0A
:1053FB002AFDEE3BFEEF3CFFA2D5E933F9ED33FD81
:10540B00EE33FEEF33FFD8D92279007A00C3801533
:10541B0079007A00C3EA13FFE913FEE8132BFBEEC6
:10542B003CFCEF3DFDE4F5D2F5D333FE7F19C3EE23
:10543B0098FEE5D299F5D2E5D39AF5D3B392D54040
:10544B000DEE28FEE5D239F5D2E5D33AF5D3A2D548
:02545B00EB3331
:10545D00FBEC33FCED33FDDF0122EE33FEE5D23301
:10546D00F5D2E5D333F5D380C3EDC454F0FEECC4CF
:10547D00FF540F2EFEEF54F0FFEBC4540F2FFF22FD
:10548D00EC75F00A84FCEB54F025F0C475F00A8439
:10549D00C4CBC454F025F0C475F00A842BFBE5F0A1
:1054AD0022AC10AB1112548DA904AD03FA7C197BFB
:1054BD009912526BAE04AF03EA75F006A4F8AC1264
:1054CD00AB1312548D2875F00A8485F014F8EF2B68
:1054DD00FFEE3CFEEF28FFE43EFEE43DFDE439FC2B
:1054ED0022C3E49FFFE49EFE22E4C39DFDE49CFCE9
:1054FD0022C3E49BFBE49CFC22C3E49BFBE49CFCE9
:10550D00E49DFD2275D4107B807A0079807800EAC5
:0A551D00F5F0A4FCADF0EBF5F0A4EE
:10552700FEAFF0EB8AF0A4C333C5F033C5F092D5D4
:105537002DFDC5F03EFEE430D501043FFFB5150D46
:10554700EEB51409EDB51305ECB51201224006EAD4
:1055570098FAEB99FBD5D40ABB0001220ABA0001DD
:105567000B22C3E913F9E813F8EA28FAEB39FB80B1
:10557700A478087B807D807C00EDF5F0A4FAE5F047
:105587008EF0B5F007EA8FF0B5F001224003ED9BEE
:10559700FDD827BDFF0122EDF5F0A4F9A8F0ED0431
:1055A700F5F0A4C399FAE5F09813CA1329F9E83A74
:1055B700F8C3E99FE89E50010D22C3EB13FBED2BC7
:1055C700FD80B6C374689511FB74019510FC8004C7
:1055D700AC10AB117A0B79B81252E480177473F8D8
:1055E700F9E627FB0809E637FC0809E637FD30E747
:0555F70003125506EB54
:1055FC0033FBEC33FCED3323FD242083F8ED241C2A
:10560C0083FFED241883FAED241483F9EF99F9E85C
:10561C009AFA1252E4EF9DFFE89EFE22FFFFFFB6BE
:10562C00FED7FD63FB5DF8C4F59BF1E3ED9EE8CF7F
:10563C00E379DD9ED743D06BC919C153B91CB0793E
:10564C00A7709E06943F8A237FB674FF6A045ECBD4
:10565C00535B47BB3BF1300423FB17DE0BB2FF80DF
:10566C00C21DC232532CF8C3E5679576FBE56895ED
:10567C0077FCE5699578FD30E705D2611255062473
:10568C00F05003125740AA06A90712530DEC2480C0
:10569C00E43DFBF9F51AE43EFCFAF519E43F60022F
:1056AC00D2321252E48B128C138D148E15C3E56416
:1056BC009573FBE5659574FCE5669575FD30E7051E
:1056CC00D262125506EBF9F51FECFAF51DED6002EE
:1056DC00D232303201221252E4EB2512F512EC35A3
:1056EC0013F513ED3514F514EE3515F51540E102EF
:1056FC00551112566C20323BEB242E40D3EA240178
:10570C00CB3400FC7A07793D1252E4C010C0118EE4
:10571C00108D118C128B13E4FCFD7E077FD012B41C
:0E572C00BF851203851302D011D010BB0005FB
:10573A00BA0002D21D22B261C374809BFB74F59C2D
:10574A00FC74209DFD22204D69204866303F637F0E
:10575A00697E0112C9A57E1F12CA1575A700900499
:10576A00EDE0A2E792171392E7FC1582E013FB30F3
:10577A0017031254FEBC003AEB603720E73420E6E8
:10578A003110E513201707C3741F9BFE80027E1F8A
:10579A0012CA0A0EDBFA22FB2017097E00C3742004
:1057AA009BFB8008EB241FFE74209BFB12CA040E8D
:1057BA00DBFA2275A700758307E559C4440FF58201
:1057CA00E0A2E792522212C7C81257BDC2E775F08B
:1057DA000A84FEAFF075A7045382F1786412584622
:1057EA00AE07786712584675A700E57DC4540FFEC8
:1057FA00E57D540FFF787312583AAE07787612583F
:10580A003A74AF1255E61256FE8B148A1312080D1B
:10581A00ACCCAB017A0A12526BE5139B9004ECF004
:10582A00FBA3E5149CF0FCA2E7923DD23F02C7CE4F
:10583A00860308860408860518188006E0FBE0FC43
:0A584A00E0FD7A0A12528B20E70CF1
:10585400EB2EF608E43CF608E43DF622C3EB9EF694
:1058640008EC9400F608ED9400F622204D09204837
:1058740006C23F302A0522C23380F6E54824F640AA
:10588400F5E5580460F075A700758307E559C4244D
:1058940008F582E0FEA3E0FF12080D7437125932B6
:1058A400500B30381BC23878C586468013743212C8
:1058B4005932400C203809D23878C5A646754600BE
:1058C400740D125932404A1257D0303D38201122FB
:1058D400204D1F20481C204019BCFF16EB243250D9
:1058E40011D240120D4FE5BF75F019A4F536D22E32
:1058F400D22F205238E55965586032204D2F204868
:105904002CD2338028201109204D062048037536F7
:1059140000303319204D1220480F1290510559C3FD
:10592400E55895595003855859C233C2402229FB82
:10593400E435CCFCC3EB9FEC9E22E558B4FF012276
:1059440085581175A704758307E54824F65002802D
:105954005C201259202905202A02805112C7C8E46C
:10596400F516F5177510001259CAE510700312C721
:0B597400C21259E3302910E51B251773
:10597F00F517F51BE51C3516F516F51C1259F01227
:10598F00C7C20510C3E511951050D175A70002C706
:10599F00CEE55AF51124F6500375110A75A7047553
:1059AF0083067510001259CA1259E31259F00510E7
:1059BF00C3E511951050EE75A70022E510C4F582CE
:1059CF00E0E0F564E0F565E0F566E0F567E0F568C1
:1059DF00E0F5692275A701125DDC123E1A75A70466
:1059EF0022E9F0E51CF0E51BF022E510C454F0F5B8
:1059FF0082E0F512E5822406F582E0F511E0F51C50
:105A0F00E0F51B22E512B426157F757E34740D1256
:105A1F00D4F520442575110012D057025B417F6DDC
:105A2F007E3BE012D4DAE5137E3512D4DAE5127E2E
:105A3F002F12D4DA20440312D05712CFC3025B4186
:105A4F00202852E558B4FF012275A704758307E596
:105A5F0059F51030330965586005204802051012BA
:105A6F0059F9E0F513305E07204304E5376095E000
:105A7F007F797E3D12D4A8E5137E3912D4A8E512A2
:105A8F007E3512D4A830480B7F7F7E3512DE330E61
:105A9F00BE40F980392012012275A704758306854F
:105AAF005B101259F9305E0A204307E53770030285
:025ABF005C6326
:105AC100E512700B7E3A7F79745D12D4DA800D7520
:105AD100F06484E5F07E397F7A12D42AE537B40286
:105AE10005128EE98045B403028040E51C7006E58D
:105AF1001B24FB5036E511F964B4602F20062CE518
:105B010037600D200C0AC3E99570F9500324B4F9EC
:105B1100E912DCB8781D79547D1D90D804E53F2049
:105B2100E00390D80B12DDB612D5067517797516FC
:105B31001930280375161DE51264266003125B8473
:105B410075A7009006E3E511F0A3120D68E5BC7599
:105B5100F01970040475F014A4951BFBE5F0951C75
:105B6100FC922450031254FEECF0A3EBF0C24FC29E
:105B710063EC700EEB24E64002D24FEB24C84002E6
:105B8100D26322E51C24ED402BAE1CAF1B125DA697
:105B91007C007D32125384C005EFAF17AE1612D3CD
:105BA100E3CE2405CE742C12D4DA0E0ED0E02312EB
:105BB100D3DD801B125D9D125BDECE2405CE742CDD
:105BC10012D4DACE2402CEE875F0058412D4C0CE08
:105BD1002404CE7422305D02748302D4D6EE243DB7
:0D5BE10050047EC37F4B7C017DF412538481
:105BEE00C004C005EF6007AF17AE1612D3E3D0079F
:105BFE00D0067C007D32125384A805EFAF17AE1687
:105C0E00CE240ACE02D4C0125D9DEE2450305D0328
:105C1E00EE24A150047EC37F4B7C017DF41253848D
:105C2E00C004C005EF6007AF177E2F12D430D00727
:105C3E00D0067C007D32125384C005EFAF177E373D
:105C4E0012D4957E3B742C12D4A87E3DD0E075F014
:105C5E00058402D4957F6D7E2F746312D4DAE5121B
:105C6E0075F06484E5F07E3512D37212D05702CFF0
:105C7E00C330480320740122E4FCF5A79006E3E04C
:105C8E00F9A3E0FE24FE40EFA3E0FF7D78E5376048
:105C9E0008304FE3200C2A800B120D54E5BD20E096
:105CAE0010304F0DD206E57124FE5015125D938013
:105CBE00107D3CE546600A7D141460057D0A147063
:105CCE00B689111252577D6F125377BE00A9EF2479
:105CDE00E240A4AD07E51112DCB8202404B2D5B21F
:105CEE00D1781F795612DDB6A806A907E511242D25
:105CFE0075F0B484E5F012DCB87407304F02740E00
:105D0E00FDFA12DDB6B2D5B2D112DDB6B2D5B2D130
:075D1E00DDF0AD0212DDB65D
:105D2500850616850717B2D5B2D112DDB685061ED2
:105D350085071F7A03304F027A06E511241675F0A0
:105D4500B484E5F012DCB8A816A917AD0212DDB6C9
:105D5500DDFBE51124EA400224B412DCB8A81EA933
:105D65001FAD0212DDB6DDFBE5377021304F1E9009
:105D7500A550305D0390A54C7F3C7E3312763D12D5
:105D85000D54E5BD20E00612CA1B12D7A522C3E9B2
:105D95009570500224B4F922E51B2402FFE4351C5A
:105DA500FE305D1ABEC305BF4D028012AC06AB07BF
:105DB5007A1B125279783212541BAE04AF03227843
:105DC5007379641255E81256FE751CC3751B4B207A
:105DD50032048B1C8A1B22125DC430320122AC199D
:105DE500AE1AA91DAF1FB90005BC00028010C3E99A
:105DF50013F9EF13FFC3EC13FCEE13FE80E8BF2984
:105E0500005006BE2900500122C3EF13FFC3EE1355
:105E1500FE80EB3E7FE3E3E3E3E3E3E3E3E3E37FFA
:105E25003E0C1C3C7C7C1C1C1C1C1C1C1C7F7F3ED3
:105E35007FE3E3E3070E1C3870E0E3FFFF3E7FE3FB
:105E4500E3030F0E0F03E3E3E37F3E070F1F3F77E7
:105E5500E7E7FFFF0707070707FFFFE0E0E0FEFFB3
:105E6500030303E3E37F3E1E3F73E0E0E0FEFFE351
:105E7500E3E3E37F3EFFFFE3E30303070E1C38384C
:105E85003838383E7FE3E3E37F3E7FE3E3E3E37FB8
:105E95003E3E7FE3E3E3E37F3F030303E77E3C000E
:105EA5000000181818FFFF1818180000000000005F
:105EB500000000FFFF0000000000003FF000003878
:105EC5001C38F00180C1F020F0FC0038F03FE00004
:105ED5000000007CC6C6C6C6C6C6C6C67C183878CD
:105EE5001818181818187E7CC6C60C183060C0C65D
:105EF500FE7CC6C6061C0606C6C67C0C1C3C6CCCC5
:105F0500FE0C0C0C0CFEC0C0C0FC0606C6C67C3CD4
:105F150066C0C0C0FCC6C6C67CFEC6C6060C183028
:105F25003030307CC6C6C67CC6C6C6C67C7CC6C6F6
:105F3500C67E060606CC78000018187E7E18180066
:105F450000000000007E7E00000000000000000050
:105F55000000000000C6E2E2D2D2CACAC6C6C2002C
:105F65000000000000000000008080A0C0A00030FC
:105F75004020C08080C0A0A0000060A0600000A0FC
:105F850040A05098D090882050A850888850A8509C
:105F95002060806000000040E040000000000080BC
:105FA5000000E000000000000040002040800040AC
:105FB500A0A0A04040C04040E0C02020C0E0E020BC
:105FC5004020E02060A0E020E0C02020C06080E00C
:105FD500A0E0E020404040E0A0E0A0E0E0A0E0201C
:105FE500C0004000400000800080002060E060208C
:105FF50000E000E00080C0E0C080E0E0E0E0E0001C
:106005000000000040A0E0A0A0C0A0C0A0C040A02B
:1060150080A040C0A0A0A0C0E080C080E0E080C01B
:1060250080806080A0A060A0A0E0A0A0E0404040EB
:10603500E0202020A040A0A0C0A0A080808080E01B
:10604500A0E0A0A0A0A0E0E0E0A040A0A0A040C0EB
:10605500A0C0808040A0A0C060C0A0C0A0A06080FB
:106065004020C0E040404040A0A0A0A060A0A0A06B
:10607500A040A0A0A0E0A0A0A040A0A0A0A040405B
:1060850040E0204080E02020A870202070A820203B
:0D60950008F030D0100000F0A8A8000000B6
:1060A200E0000000902048708898984000E0E0E00E
:1060B20000A0E0E0E04060301030604040E040404E
:1060C20060909090909060206020202020706090DE
:1060D20010204080F060901020109060103050909E
:1060E200F01010F080E010109060609080E09090CE
:1060F20060F010202040404060909060909060607E
:10610200909070109060C0E0F0F8F0E0C0000000E5
:10611200000000000000000000000050605000700D
:106122007050000078807008F000F8888888F800C5
:10613200C0C8102040981800C0B098B0C0006020BD
:1061420040000000000090D8FCD8900000246CFCB5
:106152006C24000020A870A82000002020F8202035
:106162000000000000000080000000F000000000BD
:1061720000000000606000081020408000708888E5
:106182008888887020602020202070708808102065
:1061920040F8F810201008887010305090F8101055
:1061A200F880F008088870304080F0888870F8081D
:1061B2001020404040708888708888707088887885
:1061C20008106000606000606000000080000080D5
:1061D20000002040F84020000000F800F800000015
:1061E2002010F81020007088081020002000000005
:1061F2000000000070888888F88888F08888F08815
:1062020088F070888080808870E09088888890E02C
:10621200F88080F08080F8F88080F080808070883C
:1062220080B8888878888888F888888870202020B4
:10623200202070381010101090608890A0C0A0909C
:1062420088808080808080F888D8A8A888888888FC
:1062520088C8A898888870888888888870F0888814
:10626200F080808070888888A89068F08888F0A084
:10627200908870888070088870F820202020202064
:106282008888888888887088888888885020888844
:1062920088A8A8A850888850205088888888885064
:1062A200202020F80810204080F800CCAC9CACCC18
:1062B2000000CCD4E4D4CC0004781828C800FC40F8
:1062C200A04018202018000000000000F800000084
:1062D20000A040A050007888889868708840308874
:1062E20070200000F0A8A8A8A878484848487888F4
:1062F20070888080887020A88898A8C88888805074
:1063020048FC485080304C5C6060603C00E0F00823
:106312000808F88044485C484480F8808080808087
:106322008078484848484888B8A8A8E8A8A8B88803
:1063320088888888F808500070888888708080F083
:1063420088888888F8888888888888F090909090D3
:1063520090F0A8A8A8A8A8A8F8888888F80808082B
:1063620050008888888878A8A8A8A8A8F8080000FB
:1063720000000000000000000000000088888888FB
:10638200E8A8E8A8A8A870A8A8A800000000000033
:1063920000000000000000000000000000000000FB
:1063A200000000000000000000600060600060006B
:1063B20060006060205020000000005090B890D033
:1063C20090886050500070705000882020887000C3
:1063D2000080C0A090F8003048B4B4483000304883
:1063E200B4B44830FC0098D02058C800F8E8D880EF
:0A63F200D8E8F8404050F850404051
:0300000002005E9D
:03000B0002B54FEC
:0C000E00206E06859950D26E32D26F32FF
:0E00230010990AC298206DE385994FD26D3274
:10003800E4F537F534F52F12DE29C229C22AC26841
:09004800C227C214C215022CDF0C
:03005B00022A6D09
:10B542008530F0C5F065308530F060F722C0D0C09C
:10B55200E0C0F0C0A775A700C083C08275D008758F
:10B562008A00300503758A7A758CEA0532E53270F5
:10B572000215320530E530640A6026201520E531D7
:10B58200B40C0BE530B4010612BA1412D8DCE53162
:10B59200B4180BE530B4060612BA1412D8DC02B79E
:10B5A20069C2AFD2C075C07AD2AFF5300531E5318C
:10B5B20064197040F531201529C225C22C7D0A7408
:10B5C2000412DEDAEF33EE339005CCF0EE24F540D0
:10B5D200112402400B24014005DDE4022A6DD2252C
:10B5E200D22CE5A6600215A678B5E660011678B6FB
:10B5F200E6600116302E0BE5367007C22FC22E12FE
:10B60200B8F9E5367004C24B8002153678A9E660B7
:10B61200011678D8E66001160535E5357002153554
:10B62200E590307B0B30E008D278C27BC200801AF2
:10B63200307C0B30E108D279C27CC201800C307DB3
:10B642000930E206D27AC27DC202E59044F8F47073
:10B6520003753500304A09E53324FA500375330582
:10B66200E5336005153302B70EE590F45407700315
:0DB6720002B70EA2E09200A2E19201A2E256
:10B67F00920230100320143D75330820001B201058
:10B68F000C2011098013E59030E10E8006E5372478
:10B69F00FC40F3E543541FF53320100375A6FF203C
:10B6AF002E5D301004E536705620100C201109E580
:10B6BF003524F55003753304D21BD2A5D2A612B888
:10B6CF00F975B44075B24078D8E67002053420277A
:10B6DF002E20682B202928202A25A2107211501FF6
:10B6EF00E52054076019E53424375004C24A800F0F
:10B6FF002401400B200026200119D27D7534C8206B
:10B70F001558E531702412DEBA74E812DE93802AE0
:10B71F0002B83CE53724FC40E6D27C80DF3011DFF5
:10B72F00E53724FC40D9D27B80D275F00384E5F055
:10B73F0070DE12C4BA74E812DE93E531B406051256
:10B74F00C6328016B40C0512C648800EB41205120C
:10B75F00C6328006B4180312C648E59030E10530B2
:10B76F00E202800620100820110520103C807D2069
:10B77F0027F82068F52029F2202AEFE534243040FD
:10B78F00E9240750E5600B205E088590F020F20257
:10B79F00740190B7B193D2A5201002C2A512B8E4DC
:10B7AF00806FC8A08269554646202F12E536603C4F
:10B7BF0024AA500AE53675F01984E5F06040D2A648
:10B7CF00201002C2A6D2A5202F0C7418304B027481
:0EB7DF006412B8E4803BE53675F00C30480388
:10B7ED0075F00684A2E0744640E9743780E5E52BD8
:10B7FD005403600C20100E301106E54A64026005FA
:10B80D0012B8FF800312B854101B08A25892A5A2BB
:10B81D005992A675A700D082D083D0A7D0F0D0E0E2
:10B82D00D0D0201009C5A67003022A6DC5A632C25C
:10B83D0018B40202D21812C55830180874E412DE7A
:10B84D009302B74902B74478A7E5B4600924E040F4
:10B85D0005760002B8FFE534702920412220751FBE
:10B86D00300D1CE57924CE40167AFFE5B110E701C5
:10B87D000A2325B3F5B3EA35B4F5B4C313F5B2E62F
:10B88D0060021622C2412075028077C246E579FF1B
:10B89D00605820120424FD5051206502C21CD2654F
:10B8AD00EF24B050027F4FEF90B9C49375C7037565
:10B8BD00C6FC75B90185BFF0A4E5F0F624F440028D
:10B8CD00760C301C2DE5BEC39FF5F0A4E5F024E009
:10B8DD00400375F020E5F0C21C79AA770375B3001B
:10B8ED00F5B4C31375B100F5B222C26578A77680A1
:10B8FD00D24179AA7703D21CE4F5B3F5B4F5B1F5CD
:10B90D00B222C26579A1E57924CE500DE720E7E298
:05B91D007628301CDD5E
:10B92200743C80BE7680E720E7D3E57997404DC22C
:10B932004679AAE7FAE5792323B4C500400274C424
:10B942002437300E31F42437300D15F7BA0302FADA
:10B952000AC39AF5B175B300EAF5B4C313F5B2227E
:10B96200101C07D21C76C802B8E6763274FF200E8D
:10B9720002749B02B8E6C313247E80CC75C703759C
:10B98200C6FB75B901E5BD6026C395795004C24670
:10B99200801D78A720461B301C11E57975F008A49C
:10B9A2002432F6E5792324AA02B8E47605D24602C7
:10B9B200B8FF301C077614747802B8E47696C24653
:10B9C20080EDFFF3E8DDD3C9C0B8B0A9A29A948F85
:10B9D2008A85817D7975716E6B6865625F5C595687
:10B9E20053504E4C4A48464442403E3C3A38363424
:10B9F200333231302F2E2D2C2B2A2928272625258C
:10BA0200242423232222212120201F1F1E1E1D1D2C
:10BA12001C1CD2B5C28EAE8DAA8DAF8BAB8BE4F55A
:10BA22008DF58BD28E3014012278B6BE0007EF243A
:10BA3200E24002800806E624EC50027614206705F4
:10BA4200E624F64005E4FEFAFFFB7C007D0A125272
:10BA5200577C007D5E1253778F51EE60037551FF64
:10BA6200EAFC7A3312526BEBF5F0A4E5F0CB8CF0E2
:10BA7200A425E0C5F035E0CB92D525F050060BBBEE
:0EBA82000002D2D530E7060BBB0002D2D5EC95
:10BA9000F5F0A42BFBE5F03400FC30D5010C78A6C2
:10BAA000E6C39BFF18E608F6EB18F618E69CFE18AE
:10BAB000E608F6EC18F6301401227A0050040A1257
:10BAC00054EE7C007D6E1253778FF078A2E6A4FBD3
:10BAD000ACF012548DEBBA0002F404FAE4F8FFEA79
:10BAE00030E70118E57960062075031FF4042AF594
:10BAF00079EF38D27520E70860037579FF02C784B3
:10BB0000C2750470F5E579F40460EFF57980EE1202
:10BB10000D4A78BBA6BC120D68E5BE78A2F624F6E5
:10BB20005007E4F5BEF6124E2C120C33E5BEF54874
:10BB300024F65008E4F5BEF548124E2CE5BFF54357
:10BB400024F3503924F34035120D5E78A1A6BCE5EC
:10BB5000BF789DF61424FB50087403F6F5BF124E0F
:10BB60002C78B7A6BE120D54E5BDA2E39266A2E4FE
:10BB70009267035403C253B40102D25322740DF5E9
:08BB8000BFF543124E2C80C0FA
:10005E0078FFE4F6D8FDF4F5A6D2B4D2C075C07A16
:10006E0075D75075AE1375AF017581D87590F8754B
:10007E00EFBC75FDFFD2A412DE00C2A47450122A8A
:10008E0085758951D28C75A882D2BC12BB8812DEBE
:10009E00BA12C43012BB0F12D98F12294B7F407E79
:1000AE0001909B7E12760A124C8D12DE0012DAE15E
:1000BE0012DD1812DE297C1412DE0A300003022A29
:1000CE006DDCF51247E2753A00124830E53A7016CB
:1000DE0012DEEE7F437E0690A33412760A12DD18EE
:1000EE003000FD022A6D75A6FF1247E212BB0F12F9
:1000FE00294B12DD1812DDFC12DE2978B5761E12A0
:10010E00D98F12C425C215C21412294B909BC57FDC
:10011E00781275F8205E0A7F767E12909BD212D5E9
:10012E00067F4012DD8E7F497E0978AEE612D372CD
:10013E007E15743A12D4DA7E1AE53E12D3727E26FA
:10014E00743A12D4DA7E2BE53F20E00805A6E5A628
:10015E00700215A6E53F12D3727F5312C9997F57CD
:10016E007E0B12D29F12D3277F60207303020208E8
:10017E007E0BAC5DAB5C12D2A312D3277E3112760E
:10018E00957F697E1212D82A3025087E1290DB4A9E
:10019E0012D506E5A60303543FFDFE0D7F7312DE56
:1001AE00330F12DE331EDDF478B5E57124F640020E
:0801BE00761E307419E660564C
:1001C6007F727E16744012D4A87E17E612D4307E53
:1001D6001F745312D4A812DD1810003710013710FF
:1001E6000237124782D2AC75369612DB90B4E00520
:1001F600124878800AE53670F11247D012DDF9020E
:10020600010D2074097E2BE52E540712D4C77E17E4
:1002160002018C022A6D022CA58072E53524C85095
:1002260049E59020E244D0E0D0E012027102725E0D
:10023600E53524D25034E59020E22FD0E0D0E0120C
:10024600DEEE8038E53524D25020E59020E21BD042
:10025600E0D0E012DEEE306B0B7F091275EF124E26
:1002660064127AC51202710205AB2212DEEE90A369
:10027600ED7F001275F812DD1802DDF912DEEE9040
:10028600A3ED7F001275F812DD1812DDFCC215C24F
:1002960014C227C26812DE29753701909CAE121C63
:1002A600429002AB730200F7021705020A43021ED0
:1002B60055021E510205AB0205E802725E0202C635
:1002C60012DE2975370790A054121C429002D6738D
:1002D6000202930208580208920208C60202FA02B3
:1002E600049A0202C60202C60203180202FF024A6A
:1002F600F6020326124833805A7F517E007472122A
:10030600D4D6121D9F40B9124D7812D98F12BB0F49
:1003160080AE7F49A25E120C1E925E120C3D80A03A
:100326007F64120D8B121D9F401DE5352480F475E8
:0C033600F0198460157F727E1F12D4C77E
:1003420012DD181001E810000280E30202C612BB9F
:10035200F50202C6124E2C12DE2975370290A23126
:10036200121C42900369730202C6020D95020DFA35
:10037200020E4E020EA3020EE7020EF60203CA029C
:1003820004000212B702038A7F5B120D8B120D6DFD
:10039200A8BE1203AE12DD181000081001071002E9
:1003A2000780EF18180880EA88BE80A85300037FF0
:1003B2005A7E0590A284E875F00BA42582F582E5A9
:1003C200F03583F58302760A7F40120D8B120D6D94
:1003D200E5BCF8E87F3F7E3212D3E912DD18100047
:1003E2000810010D10021280EA18B84AE6787D80E2
:1003F200E208B87EDE784B80DA88BC02035612DE51
:10040200EE7F0F90A5DF1275F8121D5C12DD18C287
:1004120014C21512DDF97510651000DFE53170F9AF
:10042200E5106465700D855E14857A15E4F512F5A4
:1004320013800C78A8E51326F513E43512F5127F24
:100442001E7E19E51012D38FC3E57A9515F517E5CF
:100452005E9514F5167F287E0BAC16AB1712D2A34D
:1004620012D32712DD1812DE0AD510ADAB17E5162E
:10047200FC30E7031254FE7A0A79001252E4A91200
:10048200A81312541DEBF510243840037510C8123E
:100492000D4A8510BC02035612DEEE909C0A7F01C3
:0204A2007E09D1
:1004A40012760A909C137F0A7E0912760A7F131231
:1004B400C991751700120D59E5BC12057AE5BD12F4
:1004C400057AE5BE12057AE5BF12057A909C637F32
:1004D4005F7E0612760A121DE112DD1875170012EE
:1004E400055A10000810011510024880F20517E59E
:1004F4001724F7500375170075100080E2E51764A0
:10050400087015120D5975BC0175BD2375BE45756E
:10051400BF67124E2C02049AE51012058C12DD18E6
:1005240012053A0510531007E51724FE4003531033
:100534000380AC0202C6A9BCAABDABBEACBFE51722
:100544001304F8E640085407C42510C4800454700A
:100554002510F6027CA97800E875F009A42417FF99
:100564007E3B7D20E8651770027D89ED12D4DA08A0
:10057400B809E502DD18F8C4120580E812058C7E7E
:10058400030517E51702D4C7540775F009A4909C16
:100594001B2582F58250020583E51775F009A42412
:1005A40017FF7E0C02760AC26812DE2975370590A1
:1005B4009DF0121C429005BD730202930278490219
:1005C400788E027A240205AB0205E102796602798B
:1005D400CC0216CE0205AB0216B4020B4F7F2E12CC
:1005E40015C980C312DE29753706909ECB121C42B2
:1005F4009005F87302029302170B02176D0217E6B7
:100604000218B30218E502195C02063D020636021E
:1006140019A5021A4A02061C7F64120D54E5BDA2F4
:10062400E7120C1E120D54E5BD92E7F5BD124E2CD7
:1006340080B27F491215C980AB1207F9122AAC1295
:10064400DEEE121D36E558046077909F9D1206E693
:1006540012862912DD1810000810011310021C80E4
:10066400F50559C3E558955950D575590080D015ED
:1006740059E55930E7C985585980C4E559B40F0282
:10068400802FB51F02802A75F007A42408F517757A
:10069400162774B82559F987001206D412DD1810EC
:1006A400002810012810020280F574B82559F9A712
:1006B40000E53524FA508878C7A6481207F012DE00
:1006C400EE12DD1812DDFC0205E81880CC0880C9A2
:1006D400E875F005A485F01CF51BC000125B84D0FE
:1006E40000221286BAB4FF0122751000751FFF1292
:1006F40086D1E510640F601712071D401274B825E7
:1007040010F8E675F005A485F01CF51B125C1505C0
:1007140010C3E558951050D72212109BF8602E6430
:1007240004602AE814B51025F51F120D68E5BC70A5
:10073400060475F014800375F019A485F01CF51BEC
:10074400125C157E2290A58012763DD322C322E549
:01075400584C
:10075500B4FF0122751000E510640F602EE51075D9
:10076500F007A42409FF74B82510F8E61207DA7516
:10077500F00A84C0F07E2012D4307E28742C12D466
:10078500A8D0E07E2A12D49512079A0510C3E55821
:10079500951050C32212109BF8603964046035E847
:1007A500146510702F120D68E5BC1207DAF8C31333
:1007B500923D7E1C12D4467E28742C12D4A8E430B7
:1007C5003D067405B80001147E2A12D4957E18746E
:1007D5002312D4A822305D1275F036A42432FBE42E
:1007E50035F0FC12548D12548DEB2212080212754D
:1007F500DDDFFB22120802127DB9DFFB2275C7037C
:1008050075C6F078B87F042275C70375C6F375B948
:1008150001E5BFB54831E55924F1402BE55975F09F
:100825000484A9F024F0F5C675B901C5F0A9BC602A
:100835000CA9BD146007A9BE146002A9BFE975F033
:1008450005A4F985F0CC22120D68A9BD75CC00224E
:10085500124E2C12DE2975370390A0C1121C42904E
:100865000868730202C6020B6802120C020B7D02B5
:100875000B880216290212D0020C49021304021336
:100885004A02167B02128602138F124E2C12DE29A3
:0608950075370490A185F7
:10089B00121C429008A2730202C6020B97020BA213
:1008AB00020892020BB8020BC3020F10020892024D
:1008BB000BD2020BAD020BEC124E2C12DE2975374C
:1008CB000B90A1D6121C429008D6730202C6020FDF
:1008DB00BE020FBE02095C02099A0208FD02092042
:1008EB0002171102106302112B0210D40211BC0269
:1008FB000C06120D54E5BF1470C17F2E120D8B1F09
:10090B00120D54E5BDA2E6120C1E120D54E5BD925C
:10091B00E6F5BD80A37F37120D8B120D4FA8BFE8F4
:10092B0012095412DD1810000810010D100212806C
:10093B00EE18B802EA780A80E608B80BE278038072
:10094B00DE120D4F88BF0208C37F367E2CE802D320
:10095B00787F1C120D8B120D54A8BE12098E12DD5E
:10096B001810000810010D10021480EF18B800EBDE
:10097B00780B80E708E824F450E1780180DD88BE2D
:10098B000208C37F1B7E35E875F005A402D3727F86
:10099B0025120D8B120D54A8BF1209CC12DD1810A5
:1009AB00000810010D10021480EF18B800EB780945
:1009BB0080E708E824F650E1780180DD88BF020863
:1009CB00C37F247E3BE802D4C7120D4AE5BF75F006
:1009DB003CA4ACF0FDE5BE75F005A42DFDE5F03CA7
:0D09EB00FC120D54E5BF14603675F005A434
:1009F80085BEF0A42DFFE5F03CFE7C007D3C125343
:100A080084C005EF75F01884E5F07F2D7E2412D39D
:100A1800727E30743A12D4DA7E35D0E012D3720284
:100A2800DD187F2D7E0590A5A212760A120D54E5D9
:100A3800BDA2E67F2D12155802DD18D25712DEEE40
:100A4800121D36120A510202937F177E02909D0EE4
:100A580012760A7F4C7E02909D2412760AAC5DAB1A
:100A68005C7F577E0412D31F120D7785BC6285BD4B
:100A780063E56124F84044909D2E7F371275F8AEE7
:100A880061AF607C017D5E125384C3741F9FFAAC12
:100A980063AB62EC33921750031254FE12526BABE5
:100AA800047C003017031254FE74F52BFB74033CCE
:100AB800FC1252417F377E1512D297909D3B7F6979
:100AC8007E0F12760AE560240FFBE43561FCA25C18
:100AD800923BD25C7E1E12D2A3A23B925C7E307403
:100AE8002012D4DA7E36742012D4DAE5602562FB4F
:100AF800E5613563FC7F227E0412D31FE5624563FE
:100B08007016742E7E3A12D4DA12DD1810000D1009
:100B18000115100226020A79742080E81562E56240
:100B2800B4FF0C156380080562E56270020563E591
:050B38003524F5500317
:100B3D00753301020A79120D778562BC8563BD029A
:100B4D004E2C7F637E00747212D4D6121D9F400806
:100B5D007F631275EF124E330205AB120D5EE5BCCD
:100B6D00A2E77F0A120C21E5BC92E7F5BC020855FD
:100B7D007F1CA20D120C1E920D80097F25A20E1254
:100B8D000C1E920E120C3D0208587F0AA20F120C79
:100B9D001E920F802A7F13A208120C1E9208801F2E
:100BAD007F52A20C120C1E920C80147F25A20B12E8
:100BBD000C1E920B80097F2DA209120C1E92091298
:100BCD000C3D0208927F49120D54E5BDA2E3120CB3
:100BDD001E120D54E5BD92E39266F5BD02088F7F9E
:100BED005B120D54E5BDA2E5120C1E120D54E5BDB0
:100BFD0092E59243F5BD02088F7F6D120D54E5BD50
:100C0D00A2E0120C1E120D54E5BD92E0F5BD0208D6
:100C1D00C3120C338F1F9217120D8BAF1F1F7E390E
:100C2D00128313A21722120D6385BC2B85BD2122C1
:100C3D00120D63852BBC8521BD024E2C203714125D
:100C4D000D5E85BE12120C76120D5E8512BE124E11
:100C5D002C80057F3F120C680208587E0390A14E30
:100C6D0012760A12DD1802DDF975A6FF12DEEE12FC
:100C7D00B542740712DEDA8FF0740612DEDAEF2554
:100C8D0012C395F0A2E7923D4010FD24CD50027D98
:060C9D0032AC05C3743FF8
:100CA3009DFD800FF404FD24C850027D37AC05740C
:100CB300402DFD7F4012C9917E1212DE330EBE1EFF
:100CC300F91F303D020F0FEF6D70EDE536700A75B9
:100CD3003606EC2513F5148C13120CF412DD1810E0
:100CE3000007100108300207221512800205128046
:100CF300827F377E28742E12D4DA7F347E21740AE1
:100D0300303D010412D4F5E514FC249C50027C63AD
:100D13007F347E2DEC12CFB17F437E1E12D29F7E95
:100D230000E51212D4367F057E0290A15912760A8D
:100D33007F6D7E0190A16412763D7F747E0490A145
:100D43007512763D021D3675C6F4803575C6F5807D
:100D53003075C6F6802B75C6F7802675C6F88021D8
:100D630075C6F9801C75C6FA801775C6FB801275A7
:100D7300C6FC800D75C6FE800875C6FF800375C668
:100D8300FD75C70375B9012274721F12D4D60F0201
:100D9300DD187F0A120D8B7E2A124833120D68A8C4
:100DA300BF120DC910001210010510021580F508BD
:100DB300E824E750EC781880E818E830E7E3780097
:100DC30080DF88BF805F7F097E0590A463B80C0332
:100DD30090A45D12760A7E27E53D28240C75F01851
:060DE30084E5F012D3725A
:100DE9007E33743B12D4DA7E35E53E12D37202DDCE
:100DF900187F13120D8B120C33120E2B10000810D2
:100E0900010510021780F2105C07205D0BD25C808F
:100E1900E8105DE5D25D80E1D25C80DD852BBC0206
:100E29000356205C10205D1890A4B67F127E231211
:100E3900760A02DD1890A4CA205DF090A4BD80EB6B
:100E490090A4C380E67F1C120D8B120D63A8BF12FC
:100E59000E8510000810011110021A80F2E824F220
:100E690050031880EA780D80E6E824E740030880FB
:100E7900DE781980DAE8F5BFF54380A37F1B7E266B
:100E8900E412D4C7E82323B464087E26740112D47B
:100E9900C7E47E2E12D37202DD187F25120D8B1244
:100EA9000D72A8BCE8120EDE12DD18100008100140
:100EB9000D10021F80EEE824E050E9188006E824AE
:100EC900CF40E108120D7288BC124E2CD21512D9EE
:100ED9008F80D180157F247E3724E202D3E37F2ED1
:100EE900A20A120C1E920A120C3D0203597F3712F4
:100EF9000D54E5BDA2E4120C1E120D54E5BD92E499
:100F09009267F5BD0203567F367E00747212D4D6FD
:100F19000F7E16743F12D4A8120D5EA8BD120F8958
:100F290012DD1810000810010510021080EFE824E6
:070F3900875004240A800226
:100F400024E8F880E17F377E16742012D4A87E2C26
:100F5000743F12D4A8120F8912DD18100008100176
:100F60001410022080EF18B80904787880E7B87868
:100F7000E478E780E008B87904780A80D8B8E8D542
:100F8000787980D188BD02088FE82487923DE850A7
:100F90000224917F367E30C313923B12D3E37E3C12
:100FA000E4303B02740512D4C07E1A90A3AB303DEE
:100FB0000390A3AF12760A7F3C7E3A02DE337F12A3
:100FC0007E00747212D4D60F7E20743F12D4A81201
:100FD0000D4A85BE1085BF11121045100008100182
:100FE0001110021B80F21511E511B4FFEB751117FA
:100FF00080E60511E51124E850DE75110080D91254
:1010000010457F137E20742012D4A87E31743F12C5
:10101000D4A812DD1810000810011110021B80DF87
:101020001510E510B4FFD875100B80D30510E5102E
:1010300024F450CB75100080C6120D4A8511BF856F
:1010400010BE0208C37F127E24E51112D3727E30D7
:10105000743A12D4DA7E35E51075F005A412D37215
:1010600002DD187F49120D8B12109BF81210A1108F
:10107000000810010D10021280F218B8FF02780467
:1010800080EA08B80502780080E2120D4A88BD1295
:101090004E2CB800030208C602112B120D4AE5BD02
:1010A000227F487E0590A3C512760AE8601CB4042E
:1010B0000A7E0590A3BA12760A800C90A3D112760C
:1010C0000A7E38E812D4C702DD1890A3CC7E29121C
:1010D000760A80F312109B601D640460197F5B1216
:1010E0000D8B120C33121106120D6310000B100140
:1010F0000810020C80EF0208C6105FE9D25F80E59D
:10110000852BBC0208C312109B601F6404601B7F08
:101110005A7E0590A3C512760A7E2390A3D5305F30
:101120000390A3DC12760A12DD182212109B7003C2
:101130000208C67F527E11120D8B120D68A8BC12D8
:10114000116B120D6810000810010810020880EFE2
:101150001880EC0880E9120D6888BC124E2C120D24
:1011600072E875F005A4F5BD0208C312109B604B30
:10117000E875F03270040475F028A4ADF0FC305D21
:1011800011ACF0FB7A8A125279EB30E7050CBC0007
:10119000010DAE05AF047C007D64125384C005EFE1
:1011A0007F517E1A12D38F7E2C742C12D4DAD0E0A9
:1011B0007E2F12D3721240FA12DD18227F64120DB4
:1011C0008B120D68A8BD1211ED10000810010F1050
:1011D000021680F218E824CD50EC783280E808E856
:1011E00024CD50E2780080DE88BD0208C37F63E82A
:0611F00023C2E012CD4411
:1011F60075F06484C0F07E2612D4C77E2C742C123F
:10120600D4DAD0E080A47F13120D8B120D5EE5BCFC
:10121600A2E7923DC2E7F8E812125012DD1810005C
:101226000810010D10021280EE18B800EA7832801C
:10123600E608B833E2780180DEE8A23D92E7F5BC25
:1012460079A1F70213017F6380027F12547F305C1D
:1012560001237E2875F06484E5F075F00A84C0F0F9
:1012660012D4C07E2D742C12D4DAD0E07E2F12D484
:10127600C00F7E3590A4D0305C0390A52C02763D3D
:101286007F64120D8B120D6DA8BDE812124C12DD93
:101296001810000810010D10021280EE18B8FFEAAF
:1012A600780F80E608B810E2780080DE88BD020874
:1012B600557F52120D8B120D68E5BE7F517E2C12A2
:1012C6008368F5BE79A2F70203567F37120D8B129B
:1012D6000D63A8BC5300037F367E32E812D4C712D2
:1012E600DD1810000810010710020780E71818081B
:1012F60080E2E5BC54FC48F5BCF52B0208557F4955
:10130600120D8B120D72A8BE12133B12DD181000BF
:101316000810011110021A80EFE8240AF82424505C
:10132600E778DB80E3E824F6F8247F40DB788180E9
:07133600D788BE80C6E8F471
:10133D0024DC75F00A847F487E3B02D4C77F5212AD
:10134D000D8B120D72A8BF12138212DD181000083A
:10135D0010011110021A80EFE82408F8245750E705
:10136D0078A880E3E824F8F824A040DB786080D7E3
:10137D0088BF021301E8F424A923C47F517E3B02E8
:10138D00D4C7122BB7754A00D210C211D214D27520
:10139D0075791475340012DEEE7F007E0290A13057
:1013AD0012760A9041237F087E2612D506E52B542E
:1013BD00030F7E3912D4C7121D5112D170128DDC5C
:1013CD0012DD1810000810011A10022480C52075B6
:1013DD0004057980BE1579E579B4FF05C275757977
:1013ED000180B02075EB1579E57970A7D27580A3D2
:1013FD00C210C214020858120D63E5BE7F097E3A71
:10140D0002D4C7120D68A8BF120DC9120C33120EEB
:10141D002BA8BF120E85120D72E5BC120EDE7F2DAC
:10142D00A20A1215587F36A267121558120D6DE5D6
:10143D00BC7F3F7E3212D3E9A8BE1203AE120D4A15
:10144D00E5BC7F487E3212D3E9120D68E5BE7F51AF
:10145D007E2C02D4C7120C337F1BA20D1215587FA0
:10146D0024A20E121558120D5EE5BC1212507F0902
:10147D00E5BCA2E7121558A8BF121667120D6DE54F
:0F148D00BD12124CE52B54037F367E3212D4C7AA
:10149C00120D72A8BE12133BA8BF121382120D5468
:1014AC00A8BC0216AC120C337F09A20F1215587F80
:1014BC0012A208121558120D54E5BDA2E37F481272
:1014CC001558E5BDA2E57F5A1215587F51A20C1292
:1014DC0015587F24A20B1215587F2DA209121558EE
:1014EC00120D5EA8BD020F89120D4A85BE1085BF74
:1014FC0011121045120D54A8BE12098EA8BF120964
:10150C00CC1209D4120D63E5BE7F3F7E3A12D4C7CC
:10151C00120D4FA8BF120954120D4AA8BD1210A1EA
:10152C00120D68A8BC12116B120D63121106120D6C
:10153C0068A8BD1211ED120D54E5BDA2E07F6C80C0
:10154C000B7F098040120C337F48A25E744E400220
:10155C0074597E3A02D4DA127CB57F731279131265
:10156C007D047F6C1279227F2D801A120D54E5BDFB
:10157C00A2E77F63121558120D63E5BE7F097E3A10
:10158C0012D4C77F481215B1B40104BF0901E4F5A8
:10159C001075F005A47E1E909E9C2582F58250024B
:1015AC00058302760A120D54E5BD035403C234C2FE
:1015BC005330E103D2342230E002D25322120D8B8D
:1015CC001F12159112DD18E51010001210010610F3
:1015DC00020280ED22045403B4030AE4800714547D
:1015EC0003B403011423C5BD54F925BDF5BD124E3A
:0115FC002CC2
:1015FD0080CE1274D9EBF516F5147F6C1279221288
:10160D0074BD7F647E23E51612D446C3E51695148A
:10161D00F5167F731279137F2D0215917F2E120D02
:10162D008B120D5EA8BFE824FA4003303702780311
:10163D0012166712DD1810000810010D100212802D
:10164D00E518B800E1780580DD08B806D978018085
:10165D00D5799DE8F7F5BF0208557F2D7E2C7420B6
:10166D00B80502742E12D4DA7E32E802D4C77F5B3D
:10167D00120D8B120D54A8BCE81216AC12DD181009
:10168D00000810010D10021280EE18B800EA780360
:10169D0080E608B804E2780180DE88BC0208557F38
:1016AD005A7E2CE802D4C7D26875480A124833D244
:1016BD0014122ABA127DED123312C26B12024A8035
:1016CD00F3D214751501127C6F75B901E5BC20E7D5
:1016DD001C127D9F75A6FF127DF9121D5C12DD187F
:1016ED0012771310000F500512783B80E70515E5B2
:1016FD0015242050D10205AB1217170202931217B1
:10170D00170205E81217170208C6121723120D63E8
:10171D008548BE024E2C122AAC122AC612593E1210
:10172D00DEEE909F44D24912865612860F121D0C82
:10173D0012DD1810001410010510021B80F505486C
:10174D00E548640A7002F54880CF1548E54864FF06
:0A175D00700375480980C2854849F1
:10176700122AC6E55822124833122AAC854849C2C4
:1017770050E558B40F02D25012593E803AD227751D
:10178700480A122ABA12593E12DEEE12857990A340
:101797007B20290390A386121DCEC26A1233121032
:1017A7006A0280E1C227127C47854948121B7912D9
:1017B7002AC6D22912593E12DEEE909E5A1286543C
:1017C70020500E121DB812DD181000101001AE8047
:1017D700F8121D5C12DD1810000280FB0205E812EA
:1017E7002AACE55830E7137F1B90A3667E05127677
:1017F7000A12DD1812DDFC0205E8122AC612593E4C
:1018070085594912DEEE121D4690A38612865412A0
:10181700861912DD1810000810010A10020C80F555
:1018270012187E80DB12188B80D612DEEE121D4650
:10183700909F5412865412861912861D12DD1810B5
:10184700000810010A10020C80F512189780DB12AD
:1018570018A580D6121B3F122AC612593E12DEEE79
:1018670090A2CB128654121D8412DD1810000510A9
:10187700028880F80205E80559C3E55895595003D1
:10188700755900221559E55964FF70038558592287
:101897000549D3E549149558400375490022154970
:1018A700E54964FF7005855849054922122AACE5C8
:1018B7005830E7057F240217F0122AC612593E1244
:1018C700DEEE909F5F128654121DC312DD181000C2
:1018D7000A10010280F8121BE880DE0205E8122ACE
:0618E700ACE55830E705F6
:1018ED007F2D0217F0C26B7559FF12593E12DEEEB5
:1018FD00121D36E55930E703121D51909F71128666
:10190D005412862912DD18E55820E706100008103C
:10191D00011110021B80F00559C3955950CF75590F
:10192D00FF80CA1559E55964FE70C285585980BDAE
:10193D00E55920E711D26B75A700758307C4F582B1
:10194D00E0B2E7F080A7306B03121B960205E81298
:10195D002AACE55830E7057F360217F0122AC61279
:10196D00593E12DEEE909F7D128654121D9F400946
:10197D00121BDD121C121219890205E8120D68E501
:10198D00BD75F00584F5BCF5BDF5BEF5BF120802B9
:10199D00124E2C05C6DFF922122AACE55820E708B5
:1019AD007F51909F870217F312DEEE90A39112865E
:1019BD0054121D5C12DD18124792D2AC10001FE5B7
:1019CD005830E7F8306DF5121ADF7E207F00501386
:1019DD0090A3E312763D12DD1812DDFC80CAC2AC75
:1019ED000205E81B8B13909E7612763D12DD18C210
:1019FD006B7B007514B8121BD2127D6E127D2050B8
:101A0D0025A814E824384004A60105140BC3E513DA
:101A1D009B50E678B8121C14306B03127AC5122A4B
:101A2D00C612593E8082127CB5E51660E6D26B1265
:101A3D007DCBC003127C86D003A91580C4122AACBD
:101A4D00E55830E7057F5A0217F0122AC612593EA3
:101A5D0012DEEE909F92128654121D7912DD18102F
:101A6D00003510010280F8754605121AA750157F32
:101A7D00007E357407954612D44612DD1812DDFC32
:101A8D00D546E7D390A39C500390A3E3128654123E
:101A9D00DD1812DDFC80B30205E812479212DC322C
:101AAD00745212DC43745412DC00E558047559006D
:101ABD0012DC211276C24016127C47127D9F1277DE
:101ACD0013400B0559C3E558955950ECC322C2ACD0
:101ADD00D322124792D2AC12DB8B204CF1B440F7DB
:101AED0012DB90B4400312DB90B452E2F53812DBF6
:101AFD0090B454DA12DB90FA60D424EF40D012DBAC
:101B0D0090E53870C912DB9012DB901276A77B003E
:101B1D007E0312779E50102050B412DB90204C03A0
:101B2D00B440F7DEED80A7127D7E0B1276A7DAE0CA
:101B3D00C322121C23E55924C8F88602E54924C89E
:101B4D00F9986013146010500F18E608F618E8693C
:101B5D0070F7A702121C1222E559640F60F91908DB
:101B6D00E618F608E86970F7A70280E8121C2378DA
:101B7D00C8C250E6B4FF02800708B8D8F6D250228A
:101B8D00B8D702D250A615807C78B8121C25E4F97E
:021B9D00F5A7AA
:101B9F00758307E9C4F582E030E70AE924B8F82431
:101BAF0038400276FF09C3E5589950E7121BDD78DC
:101BBF00B879C8E6B4FF028002F70908E824385064
:101BCF00F2804079B877FF09E9243850F82279C8B4
:101BDF0077FF09E9242850F822121C23C23D78D739
:101BEF00B6FF04A900D23D18B8C7F5203D0279D839
:101BFF001978C8B6FF0122C3E8995007C6C7C608AF
:101C0F001980F478C8121C34127DDB127DDB127D33
:101C1F00DB027DDB78C8121C34127DB9127DB9123C
:101C2F007DB9027DB975C703E54875F004A424801A
:101C3F00F5C62212DEEEC23C1275FCE53760531476
:101C4F00604D14604514603D14603514602D1460B0
:101C5F002514600E14600B14600D14601414600CC6
:101C6F008030121551802B1215FF80261214F4802C
:101C7F002112154D801C12157780171215638012D3
:101C8F001214B1800D121462800812141080031206
:101C9F00140412DD1812DE00121D3612B905A81F2A
:101CAF0008E814C23BB51D02D23B75F007203C0378
:051CBF0075F009A4FF0F
:101CC4007E00303C0C7420303B02743E12D4A88059
:101CD4000A740B303B02740A12D4C0D8CF12DD1838
:101CE400E51D10000810011010021880B9651F705E
:101CF40003751DFF051D80AE7005851F1D80A7158A
:101D04001D80A375F003A4227F7B7E0090A2E312C2
:101D1400763DE54824F640087E0A90A34912763DB4
:101D24002212793F7E05745B12D4A47E1D745C027A
:101D3400D4A4121D257E3490A2F402763D12793F7C
:101D44008003121D257E3190A2F802763D121D25D6
:101D54007E3190A3EE02763D12793F7E008005121B
:101D6400793F7E2D90A3EE02763D121D797E31904F
:101D74009EB002763D121D5C7E1A909EB502763DA1
:101D8400121D5C80C0121D5C7E18909E6302763D1D
:101D9400121D5C7E1A90A3F302763D121D5C7E1A1E
:101DA40090A3F812763D12DD18D3100006C310017B
:101DB4000280F622121D5C7E1A909F4E02763D121E
:101DC4001D5C7E18909F6A02763D7F007E2012760D
:101DD4003D02DD1812793F90A3FD02763B12793F54
:101DE40090A40D02763B12BE0F120D81E5BDF55E87
:101DF400F56CE5BCF55FF56B756A007561FF75A759
:101E04000490070012BDB9B4FC23E582C313F56145
:101E1400E56CF0E56BF0E582600F12BD30E56C65B2
:0D1E24005E70E1E56B655F70DB75A7002265
:101E31003024EA0460E7240F40D380E1E560758334
:101E410007C333F582E0A3F56CE0F56B756A0022F8
:101E5100D2248002C224D214C21F121DEA7560006E
:101E6100E561B4FF1612DEEE909D3E7F0A7E0512FB
:101E7100763D12DD1812DDF9020293C210C2111271
:101E8100DEEE121D36301F0A7F07909D4D12763B04
:101E910080647F007E01C3E56012D4467E0E742803
:101EA10012D4A48560487407F51FFF7E00743E12AA
:101EB100D4A8E548121E3F12C7A012241B0548C32F
:101EC100E5619548FD401CE51F2407F51F24C85016
:101ED100E17F387E01ED0412D4467E0E742912D4BE
:101EE100A4800DE51F2407FF7E0190A3ED12763D2E
:101EF100201F0312245E12DD1810001910012C108E
:101F0100020280F5120236301F3D020282101F02CA
:101F1100D21F021E7CE56160F4E5606561700520F9
:101F21001FF080E9201FE6056080E7E56160DEE5DE
:101F31006065617005201FD58009201FD5E560709F
:101F41000280CA156080CB121DEA121E3D12C7A085
:101F5100122552756A1012BDA2122609909D57D200
:101F61003C1275FC121CA7901F6C73021E7C02327E
:101F710052021F8C021F78121D9F40CB121E3D1270
:0B1F8100BDB9C2E2FF12BBDF021E551B
:101F8C0012DEEE7F6490A5C51275F87F7990A5D20C
:101F9C001275F812DD1875160010000A10010910E0
:101FAC00020280F505160516C253121E3D12C7A07B
:101FBC0075370A909D73121C42901FC973021F48FB
:101FCC00021FF00221BF0221C4021FB4021FF7023C
:101FDC001FFC021FB402203A02203E0220420220C3
:101FEC004902204D7F0A1215C980BD1247AB8003F0
:101FFC001247A0780A12211C740112DBFE12215B1D
:10200C0012DC1A12219612BDA212BDCA12BCF11218
:10201C00BEE11222A5D5150C75150A1221A91223A1
:10202C00CC12DC1A100204E57F70DB021F48780A20
:10203C0080067804800278011247AB8009780A8008
:10204C000278011247A012211C740112DBF3122139
:10205C005BE54812DBDFE5165403443012DC0074F8
:10206C002A12DC0012DC0012DC1A12219612BDA21C
:10207C0012BDCA12BCF112BEE11222A5D5154885BB
:10208C0048151221A9E51C12DBDFE51B12DBDFE58D
:10209C001B2548F51BE4351CF51CE4A27792E7A23E
:1020AC007492E0A27392E112DBDFAD75AC74AB738A
:1020BC00E57DC41220DDAD78AC77AB76E57D1220E2
:1020CC00DD1223EA12DC1A100204E57F709F021F56
:1020DC0048540F2375F00584F8C3EB33FBEC33FC49
:0620EC00ED33FDC3EB33F0
:1020F200FBEC33FCED33FD20E713EB28FBE43CFC67
:10210200E43D12DBDFEC12DBDFEB02DBDFC3EB983B
:10211200FBEC9400FCED940080E88848121D63E417
:10212200F54AF549756A2075150112BDA212BCF176
:10213200D5150E854815E5492401F549E4354AF5DA
:102142004AE57F70E5744012DC43747812DC007457
:102152006312DC00742302DBF31223A7E56012DBB7
:10216200DF121E3D12C7A0E53A12DBF3E53B12DB9C
:10217200F3E53C12DBF3E53D12DBF3E53E12DBF364
:10218200E53F12DBF3740112DBDFE54A12DBDFE528
:102192004902DBDF121E3D756A20E4F51CF51BF5D2
:1021A20014F51375150122753800E51412DBDFE50D
:1021B2001312DBDF0513E51370020514221247AB7D
:1021C2008003124795121D631222FF12DE04756A04
:1021D2002075150175A6FF754A0112BD4A12BCF1A0
:1021E20012BEE11222A5D5150975151E1222C912B9
:1021F200DE0E1223CCE57912DBDFE412DBDFE571C0
:1022020012228A12DBDFE57012DBDFE57B24ACFFF2
:10221200E55F340912DBE5EF12DBDFE51520E03381
:10222200857D56E412DBDFE52EC412DBE512DC29E4
:0E22320012DE0E10021A30559B744012DC00B2
:10224000744512DC00744F12DC00744612DC00127C
:10225000DC29021F48E556122264C4FAE57D1222E9
:10226000642A80C2FBC41222712323CB1222712B59
:1022700022540FFC24F650027C00902280EC932222
:1022800000000101010202030303FA2440400A2472
:10229000804003EA3322D2E72274FF2220E703C3FF
:1022A000132224C022E53F701F7F7B7E0078AEE6BC
:1022B00012D430EE2404FE743A12D4A8EE2404FEA4
:1022C000E53E12D42A12DD1822C015C016D2121211
:1022D000A61DC212D016D01578AEE612DBF3E53E8D
:1022E00012DBF3E53F12DBF3E54512DBDFE55212CB
:1022F000DBDF740A12DBDF74C012DBDF02DC29745F
:102300004012DC00745412DC43744E12DC00743052
:1023100012DC00E5165403443012DC001223A774CB
:102320002312DBF3E53D12DBF3E56012DBDF121E67
:102330003D12C7A078ABE60812DBF3E60812DBF328
:10234000E60812DBF3E612DBF3E53E12DBF31229BB
:1023500032E51212DBF3E51112DBF3740112DBDF5D
:1023600090A41E12240C756A1012BDA2057F057F71
:10237000787F12DBD8787B12DBD8787D12DBD878B7
:042380007712DBD81D
:10238400E4FEFF780712DBD812DBD8E57412DBDF3A
:10239400E57512DBDFE412DBDFE412DBDF12DBD8EE
:1023A40002DC2975C70375C6FF75B901C217751D0F
:1023B4000085BC1C85BD1B85BE1A85BF191251F151
:1023C400EE12DBDFEF02DBDFE57512DBDFE5741213
:1023D400DBDFE57312DBDFE57812DBDFE57712DBA9
:1023E400DFE57612DBDFE51664016011E55E12DBE2
:1023F400DFE57A12DBDFE516640260012278BCE6D1
:1024040012DBDF08E602DBDF75A700E4937001222C
:10241400A312DC001A80F4AF1F7E0478ADE612D458
:102424002A7E0C742C12D4A87E0E18E612D42A7EAE
:102434001A78AEE612D42A7E22743B12D4A87E24E3
:10244400E53E12D42A7E2FE54012D4307E37743B09
:1024540012D4A80E0EE54102D42A753200121E3D94
:1024640012C7A0857946787A796412C7B974641260
:1024740055E68E47122552756A20D23D12BDA2122E
:10248400BDCA122589303D09307406C23D8E1E8FA7
:102494001FE57F602BE54C24FFF54CE54D34FFF53B
:1024A4004D454C600512BD0680D2751D3C12BDA27F
:1024B40012BDCA12BCF1122589E57F6003D51DED5A
:1024C4001225EA90260212D506203D0DAE1EAF1F3E
:0924D4001225EA9025FB12D50641
:1024DD00E546FD700B90A554305D1190A550800C14
:1024ED0004701090A550305D0390A54C7F381240BC
:1024FD00F5804BE4FFFC7E05305D047E027FB31258
:10250D005377AC06AB071252417F38C23DE51C60D4
:10251D0007D23D7E2C12D495E51B203D026007D2DB
:10252D003D7E3012D495E51A203D026007D23D7EE6
:10253D003412D495E5197E3812D4951240FAE5324D
:10254D0024C850FA22E54075F03CA42541FFF54C16
:10255D00E435F0FEF54D7C007D101253840F8F4B4A
:10256D00AF4CAE4D7C007D3C1252577C00AD4B12F2
:10257D005384EE4F70010F8F4C8E4D22786479731A
:10258D00C2D11225A0FF78677976D2D11225A0FE8F
:10259D0002DE33C3E796FB0809E796FC0809E796C8
:1025AD00FDA2E79217500312550675135A30D10E3E
:1025BD00751320B217AA4712528BAB04AC05E54632
:1025CD00600B04600BAA461252A2EB03FBEB03FB5C
:1025DD00EB543FFBE5132B2017029B9B22EE1414AB
:0825ED0030E701E4FEEF1414D5
:1025F50030E701E4FF2205057088A88870050520ED
:1026050020F8202075320012DEEE7E1E7F1C12DEC1
:1026150033DFFB12DE337E1E7F1C12DE33DEFB7ED4
:102625001D7F1D12DE33DEFB7F007E2178ADE612B5
:10263500D42A7E29742E12D4A87E2D18E612D42A07
:102645007E35742E12D4A87E3918E612D42A7F0757
:102655007E21745412D4A87E25744F12D4A87E2DE1
:1026650078AEE612D42A7E35743A12D4A87E39E5BE
:102675003E12D42A78AE1229327F0E7E21744C1276
:10268500D4A87E25744112D4A87E2DE51212D42A31
:102695007E35743A12D4A87E39E51112D42A7F15F5
:1026A5007E25744412D4A87E2DE54012D4307E35A3
:1026B500743A12D4A87E39E54112D42A7F217E01CD
:1026C50090A51F12763D7E0EAC77AB7612D2DC7EDE
:1026D5002B85795F85787B12D8837F287E0190A52D
:1026E5002312763D751D2B751E10E5741228E67EA6
:1026F50025742F12D4A8751D2D751E2BE57512286E
:10270500E67F367E0290A50F12763DE5721227937D
:1027150012282B121E3D756A209004E6E56CF09098
:1027250004E7E56BF0AE4DAF4C7C007D4012538461
:10273500BF00010F0FAC07AD07E4FED23D12BDA2ED
:1027450012BDCA1227D4E57F602CE54C24FFF54C59
:02275500E54D50
:1027570034FFF54D454C600512BD0680DE751D3C06
:102767000E12BDA212BDCA1227D9E57F600612BCA0
:10277700F1D51DED1227A97F7812C9A37F767E00B8
:10278700743012D4A8E53224C850FA227E2112CD23
:102797004412D4467E2F90A527305D0390A52C02C6
:1027A700763D9004E6E0FD9004E7E0FCC3E56A941B
:1027B70020FBE56B9CFCE56C9DFD50032410FD128E
:1027C70054769004E8EEF09004E9EFF022DD03ADD3
:1027D700040E7F78E55E20E72AE57A8549F0A4A90B
:1027E700F0E57A854AF0A429F9E435F0FAE55E8543
:1027F70049F0A429E435F02AFAE55E854AF0A42ACF
:10280700CF9FFF12DE33103D18C3EF9B50131BEF12
:102817006B600E8F018B0712DE331FEF6970F8AF05
:1028270001AB072290A4D4305C0390A4ED754A4015
:10283700754900AF76E577FE20E76B7005EF24104A
:102847005064EF24A8EE34FD401190A4D9305C0306
:1028570090A4F1754A1975499A8075EF2450EE34A2
:10286700FB401190A4DE305C0390A4F6754A0C750A
:0528770049CD805CEF7B
:10287C0024A0EE34F6401190A4E1305C0390A4FB4C
:10288C00754A067549668043EF24F0EE34F1401327
:10289C0090A4E4305C0390A500754A04754944800B
:1028AC002A8028EF2490EE34E8401190A4E7305CA5
:1028BC000390A505754A0275498F800F90A4EA30E4
:1028CC005C0390A50A754A0175499A7F4012763BC4
:1028DC007F4612C9A37F5F02C9A3AE1E75F0643098
:1028EC005C0375F03284C0F0F87004EE2404FEE54D
:1028FC001D12D4A8EE2404FEE8600712D495EE2431
:10290C0004FED0E075F00A305C0375F00584A8F085
:10291C0012D495EE2404FE742C12D4A80E0EE830BA
:10292C005C012302D495E53E2541F51124C45003E6
:10293C00F511D3E63540F51224E85002F5122212B7
:10294C00B8FFC21012DEEE7F057E09909B751276E1
:10295C000A7F137E0890297F12D5067F2B7E01906B
:10296C0029E712D50620370A7F277E27902A59128D
:10297C00D50622113007FE1FE001E101F80F000619
:10298C001B00F80C00180E007C10007006003C2098
:10299C0000E006003E4001E004001E8003C004007D
:1029AC001F0003C004000F00078000000F80078089
:1029BC00000017800F00000027C00F00000043C06C
:1029CC000F00100083E00F00200301F00700C00F80
:1029DC0001F80383007F87FE01FC000E3E18000007
:1029EC000300000000180000030000000038000085
:1029FC0000000000003000000000000000FC761F0A
:102A0C000E1C6030ECFCBC3F172DF0F97861386679
:102A1C00264F619A706070C60E1EE330E06060C68F
:102A2C000C1CC360C0E0618C0C18C7C0C0C0E18C2A
:102A3C001C39C611C0C4C19C9931963180C8C1FFE4
:102A4C001E31E7E180F0C0EE1C31C38180061630E8
:102A5C0091882892884924904927909248A0E3C8ED
:102A6C00BCC2AFD2C075C0107581D874FE122A8555
:102A7C00E4F5F9F5FBC2B480F7D2A6C2A512B8E40E
:102A8C0012DE0002B90575C703E54875F004A424ED
:102A9C0080F5C6C23C75B901E5BC047002D23C227B
:052AAC00120D63E5BE00
:102AB100F54824F65003754800753400753704C293
:102AC10028D229D22A75C703E54824E7500375485F
:102AD10000E54875F004A42480F5C675160775173E
:102AE10000C23C122B07122B07122B07122B078552
:102AF10017581558755900E548B40A09E558600595
:102B0100F46002055922203C1D75B90105C6AABC15
:102B1100ABBDACBEADBFEA122B28EB122B28EC12D9
:102B21002B28ED122B2822203C07F515B4FF03D2E8
:102B31003C22C0C7C0C6127C6F75A704851683E509
:102B410017C4F8F58275B90105C6E5BCF0C582F870
:102B51002406F92403C582E5BDF0E5BEF0E5BFF02A
:102B610075B90105C6E5BCF0E5BDF0E5BFF0851618
:102B7100838982E4F075B90105C685BC1385BD144E
:102B8100E4F0F08882E5BEF0E5BFF075B901E5BC7F
:102B9100F0E5BDF0E5BEF0E5BFF0758306E517236E
:102BA100541E24B0F582E513F0E514F075A700D0AA
:102BB100C6D0C705172212BB0F78BEA64808E4F697
:102BC100F55908761808F6D23608760A08F6060886
:022BD10076BECE
:102BD300C254C25512BE24122ABAC229C22AC2073B
:102BE300C227C268120D54E5BDA2E59243C24AE46E
:102BF300F52EF534F536F52F78B6F678B5F678A9CF
:102C0300F6789EF678B8A65E08A67A12D245C26B0D
:102C1300C233C238C240C223C222122C37754602C5
:102C230078C5A646C23AD221C219C226E4F542F5B6
:102C330041F54022E45407205E09B40400400274C5
:102C430003801B120D59C313A9BC600C14A9BD60EA
:102C53000714A9BE6002A9BFE94001C45407F537B0
:102C630022122AAC12593E1207F912DEEE121D840B
:102C7300E55804700A7F327E0590A36612760A90A7
:102C8300A5BC1286561207537F7290A5B11275F830
:102C930012DD1810000510020480F8D322C32202AB
:102CA30000F7120D54E5BD20E705122C6440F075C2
:102CB3004E50122BB712843475440312483012AEAF
:102CC30042D54403022A6D201EF1789F7680754A0F
:102CD3000012BC40D210C211C213C2121247827535
:102CE300A60C12D98F12C425E5A624FA4006124772
:102CF300D075A60C20250CE59054057009E5352404
:102D0300E25003022D97E5322418400D75F00C8430
:072D1300E5F070D412331546
:102D1A0080CFD21ED2AC306DC87532F012DB95B4BA
:102D2A00E0BF124878E53124F392052012031231EC
:102D3A00A7122D5DC014128D22D014200A03122E60
:102D4A008012331512A5EC1233151284371233157B
:102D5A00022CDF30122EE54024F0401C7A0AC3E52B
:102D6A003F954B6013401E24E2400D305405C25477
:102D7A00757F0112BC66DAE679BCE7D2E7F57F090E
:102D8A00877EC27722F40424E250ED80DE12DEEE62
:102D9A007F2A7E0E90A42212760A75A6FFC2101010
:102DAA0012137F367E08909E9312760A12DD18124D
:102DBA00DDF90200F7D22112485412BC707F1E7E40
:102DCA000B90A33F12760A12DD18122DEA7F3E7E7F
:102DDA000790A03312760A12DD1812DDF3022A6D6B
:102DEA00D215D21412BDFB120C3375B90575B9028E
:102DFA0012BE05D25512BD2A7F0012BBDF12BE05D4
:102E0A00E56A600512BCF180F7857A62120D818548
:102E1A00BEBC85BFBD856BBE856CBF75B90575B96E
:102E2A000285BD6C85BC6B756A2012BDFB12302110
:102E3A0012BE05756A0012BDA2E57064FE70347593
:102E4A0070FC854077854178851F797818797A12E0
:102E5A00C7B912BC9F12DE0E12BE05756A1012BDEA
:102E6A00A27F087810797212C7BB85627C855E7D65
:102E7A0012BC9FC215221247AB122FCD745212DC1C
:0B2E8A0000744D12DC00744312DC00E9
:102E9500122FDC12DC3B7441207402745612DC00E4
:102EA500122F29122F7312DC3BE53C12DBF3E53BB5
:102EB50012DBF3E53A12DBF3122FA912DC3B744562
:102EC50012DC00123012122FCD744712DC00744749
:102ED50012DC00744112DC00122FDC122F2912DCE7
:102EE5003BE43074010412DBFE12DC3B9004C3E0CA
:102EF50012DBF312DC3B9004E4E075F00A84AFF0DA
:102F050012DBF312DC3FEF12DBFEAC5EAB7A122F65
:102F1500EEAC5DAB5C122FEE12DC3B12DC3B1230EB
:102F2500120247827875C23D122F347878D23D124D
:102F3500DC3B128119303D05E51E12DBFEE51D1255
:102F4500DBFE122FB6E51812DBFEE57D203D01C440
:102F5500540F12DBFE12DC3B303D0974453017027D
:102F650074578007744E301702745302DC002074C6
:102F750008122FA9122FA9802775A7049004BFE076
:102F8500FCE0FB7A1B125279783212541B12524123
:102F9500122FB39004C1E0FCE0FB125241122FB393
:102FA50075A7002212DC3BE4F51AF519800D12DC39
:102FB5003BE51C12DBFEE51B12DBFEE51A12DBFE10
:102FC50012DC3FE51902DBFE742412DC00744712A3
:102FD500DC43745002DC0012DC3BE53D12DBF3E51B
:102FE5003E12DBF3E53F02DBF312817512DC3BE5B4
:0E2FF5001D12DC00781CE612DBFE18B817F87F
:1030030012DC3FE412DBFE12DC3B744D02DC00C039
:1030130038742A12DC00D03812DC1A02DE0E781063
:103023007F0EE4F608DFFCF564F565F567F5687572
:1030330015FC751AC0751DC0756640756940754AE3
:103043000112BD4A3055030230D712BCF1E571B508
:1030530010004002F510E4F511E512207502E513A6
:10306300C395795006207545857913D3E57A951470
:10307300E5156480FFE55E64809F400C857A1485C6
:103083005E15857B16855F173074B3C2D17864797A
:10309300731230B5786779761230B5D2D178187952
:1030A300731230B5781B79761230B5809185791219
:1030B30080B9D3E7960809E7960809E66480FFE735
:1030C30064809F20D101B3400AE7F61819E7F61888
:1030D30019E7F622E51AB4C00E7873791812C7B946
:1030E3007873796412C7B978187964C2D1123148F8
:1030F30074181255E68E47AE1EAF1F781B7967D240
:10310300D1123148C3E51F9FE51E9E50048E1E8FCA
:103113001F7EFF7FFFAC1EAD1F1253847A04EF8A1C
:09312300F0A4E5F0CE8AF0A42E20
:10312C00FEE435F0BEFF011E60051460057EFF8EC7
:10313C001F22EE7E0020E7F77EFE80F3C3E697FBAE
:10314C000809E697FC0809E697FD1818191930E7E5
:10315C0003125506C3EB33FBEC33FCED33FDEB33C1
:10316C00EC33FBED33FC30D105AA471252A20BBB5A
:10317C0000010C751E03751FFFEC24FC40048C1E13
:10318C008B1FE627FB0809E637FC0809E637A2E7A0
:10319C0013F618EC13F618EB13F62210131978B576
:1031AC00E624FA401AE57124F64008E57924F64045
:1031BC000280360606803212DE0AE59030E2DF75B8
:1031CC003612D22EE4F534F55A12BE561231F8C22C
:1031DC0019C257122C3712905112907ED212853F81
:1031EC004B754C00205E02D228022C2FD2141232C6
:1031FC0047E6F008DFFB857A6212323D7570FE7887
:10320C003A797112C7B912BC9F12323D85627A8528
:10321C005E7B120D7785BC7E85BD7F7570C012BC40
:05322C009F123247E093
:10323100F608DFFB75A700D254C2142274FF787020
:10324100F608B880FB2275A7049004F078707F100F
:1032510022121E3D122BB712DEEE12DD18C258C229
:1032610059754A01753901756A2012BD4A1255E432
:103271008E47C210D211D214D21212BE56129051E0
:1032810012907E12D98F75A6FF753609753200E549
:103291009020E206E5352405400CE5905405701FA9
:1032A100E53524E25019C211C21212DEEE12DD1808
:1032B100E4F535F52F7E0612DE06C202021F48C272
:1032C10021E54AB40202D22112BD4A12A5EC3026F0
:1032D1000F1259A0128437753606E53670FCC226E6
:1032E100128434123315E54A20E021B402097539FC
:1032F10000E53670F9808CE53960FAFD24E2400280
:10330100053912BD4A2026C9DDF880E975390080EA
:10331100E475370410003A100116100216E52F5417
:1033210007600312B8F920783D20790A207A1F221C
:1033310002350B02345FE537600914600914600936
:103341000235B702352A023588C2790235D40234F2
:1033510092E53724FC500FE5376407600302364FCE
:103361000236130234292011FAE59020E202805638
:10337100753400201203D2132278A9E67017C226F1
:0D338100767DE5377005106B02D26BD277B8
:10338E00753614D22E02BE4BE5376043146040B43E
:10339E000227200B24E6249B401F2414501C12905D
:1033AE005190A30F7F207E0812760A12DD18753613
:1033BE0008D22E78A9E624ECF622241940FB241418
:1033CE0050F712905112907E90A3197F2980D7202A
:1033DE0028E7E54824F640E1E5580460DC7F5D7E91
:1033EE0010E6249B40D324145015C2330559C3E56F
:1033FE005895595005855859D22690A2FD80A9247A
:10340E001940B6241450B2E559600215591026061B
:10341E00E5596002155990A306808D10780122752A
:10342E003900E53424384007754A0175340022709E
:10343E000AE54A30E0F2754A0280F0146008754AD7
:10344E000612907E8006754A0412905175390180DD
:10345E00DA302909C229D22A7559008005302A1B73
:10346E00D2291286051285D3E53524AF4004753472
:10347E000022753700C229C22A80F3206841302706
:10348E0003D26A22D2221237EB12DD18107A0122F1
:10349E00E53424384007122C3775340022700FAAF9
:1034AE0037122C376A70F27401122C3880EB04122A
:1034BE002C3824FC50E3E537B40706D22880DA8096
:0834CE0036C228E53724FC2377
:1034D60024BEF879C4E7F9A74809A75979C4E8F7DB
:1034E6008648088607E537B40505754818D23612AA
:1034F6002AC68F59E53764067002D2070234A7122E
:1035060037C7023771E537601B14607614600F14F5
:103516006009E53724F940090236C90235B7023693
:1035260002023696D223123FD910790122E53424BD
:103536003840077546017534002278D87020304A25
:103546000BC24AE624F85004B243800AD24A7614E3
:10355600E54624FE40DDE54660D9154680D8B6002E
:10356600D5B40500500C04F54624FA50C975460535
:1035760080C424F95005127A6380BB100FB8D20FAD
:1035860080B4D223E53464C86003123FD9107901B0
:1035960022E534243750097011105B32D25B802E3D
:1035A600100802D208123FD98024100C21D20C80B8
:1035B6001DD223123FD910790122D24BE53424378C
:1035C6004010C258C259201105D22E7536077534DF
:1035D600002224FD401524037006D258C25980EEFD
:1035E600C258D2591460E7D25880E3120D5EE5BC8A
:1035F600B2E7F5BC79A1F7124E2C80D278B8A65E58
:0B36060008A67A2011C8753605D22EE8
:1036110080C130122B12863F055BE55B75F00B8490
:10362100E5F0F55BE55A24F64009E55A955B500350
:10363100755B0012864312DD18E5346003D534D280
:1036410075340022D229D22A75480A023737C2407E
:103651001007F1302903023737128601128615103F
:103661002A1BC2330559C3E558955920E702500872
:10367100755900E548B41816E558B4FF03755900AB
:1036810012862912DD18E5346003D534C122D22A0D
:1036910012860580EE30122312863F155BE55B3002
:1036A100E70C755B0AE55A24F64003855A5B1286DE
:1036B1004312DD18E5346003D534DA75340022D2C3
:1036C10029D22A754817804CC2401007F22029449C
:1036D100128601128615102A22C2331559E5593076
:1036E100E71C855859E558B4FF03755900E548B4FE
:1036F1001802800AD22A128605800E855859E5588B
:10370100B4FF0375590012862912DD18E5346003F0
:10371100D534B52220106220115F7F180548E54895
:1037210064187008F54830270375480A122A923048
:103731003C2DDFE8802620105A2011577F181548AC
:10374100E54830E705754817800A64097006302797
:1037510003754817122A92303C05DFE275480A12B8
:103761002AC612593EE532244C50051285D38003F6
:1037710012857975340002DD181237AE7F15E548E0
:103781006B70048A4880020548122A92303CD0DFCF
:10379100ED80CC1237AE7F15E5486A70048B488006
:1037A100021548122A92303CB6DFED80B27A007BD6
:1037B10009E537B40401227A0A7B17B406012274A1
:1037C10018FAFBF5482275A704758307E559C4F576
:1037D10082E0E0F573E0F574E0F575E0F576E0F58B
:1037E10077E0F57875A70002593EE59020E23EE5C5
:1037F100342437503812382F12380C205E4F7F2C6A
:10380100909C2D123876909C36806AE53424377569
:10381100F009A42435FF205E0624BE50027F3EEF4E
:10382100249B50027F627E32748912D4DA2275A7FA
:10383100049000317E087F3AE4F0DFFDE582244602
:10384100F582E43583F583DEED75A700227F2C1226
:103851000D59E5BD12385FE5BE12385FE5BFF8C40A
:10386100123865E8540775F009A4909C1B2582F570
:0C3871008250020583EF2409FF0275F865
:108431000284EE12DEEEE53724FC40F4B4FE142093
:10844100110EE590F45407600122E532247450EFD7
:10845100028D2E12DEEE12D67D12D70F12CD5212E0
:10846100D29B12D0E47E197F3612CE8C12DC4812D8
:10847100CEA2C206E53760051460338053C23A12BA
:10848100859212409C1242311245171263FC12640C
:1084910024123D47E54864186009E54824F6500375
:1084A100124602128CC412CF771241378014D23A8D
:1084B1001285B812388512410612C909128CC412EC
:1084C100CF38125C7F12D756125750125A4F801272
:1084D10012859E12C84612D82612C8D8128CC41210
:1084E100CF4F30101412CE1512CDE4800C12DEEEF7
:1084F100E53724F9401E12857B3022091237EBE55E
:10850100347002C222302309123FD9E5347002C20D
:108511002302DD18121D3675170012DA397F121287
:10852100C99130124A75100075A704758306125956
:10853100F9E51075F009A42415FFF5177E00E51281
:10854100602F75F06484E5F00F12D42A1F7E0EE5CA
:108551001112CD9A751623125BB50510C3E55A9514
:10856100104006E51024F550BF30120312864380F7
:1085710088745D12D4DA80D5C249302905121D0CE8
:108581008003121D36909E5A128656202A76028644
:1085910029301223305E2030501D02893A301217E3
:0385A100305E0643
:1085A400200B11028F9B12C98A7F1712DD8E75175B
:1085B4002002DA3912D5F412D59530121120510562
:1085C40012D654800612CCDE12CABE1250B322E474
:1085D400FEFFE54824F6400D90A34912763D7E1631
:1085E400E54802D495B40E0690A34F02763D90A3BD
:1085F4005612763D7E12E54824F702D4307D208061
:108604000C7D3F302A077D633029027D3C7F00804A
:10861400247D2080127D3E800E7D3CE54975F00767
:10862400A42406800A7D3FE55975F007A42409FFB8
:1086340064027001FF7E1CED02D4A87D2080027DBF
:108644003FE55B75F009A42416FF7E09ED02D4A86A
:10865400C2491286BAB4FF01227510001286D1797C
:1086640020E030E702792F30491712109BFAB40446
:1086740008E510700C79658008EA146510700279B9
:1086840023E97E1812D4A87E20E51230E708909ED4
:108694009312763D8016E511128747125C1520105F
:1086A4000520110280063012031286F90510C3E575
:1086B40058951050A7227E207F0012763D1285D354
:1086C4007E007F0690877912D506E5582275A704A7
:1086D4007583071259F9E51075F007A42409FFF50D
:0D86E400177E00E51212D4A87805EE2404DC
:1086F100FEE012D4A8D8F622128801128817FD7C58
:1087010000AE1CAF1B125377BE003A8F00C3E57A4F
:108711009513FFE55E9514FE402B7C007D281253D6
:1087210084C3EF98401F75F0058404FB24F95002BF
:108731007B067E2CAF170F12DE330F12DE330F12C2
:10874100DE330EDBEF2264B4602464B475F032844E
:10875100C0F012D495CE2404CED0E075F00584C0CB
:10876100F012D495CE2404CED0E02302D495908784
:108771007502763D2D2D2D000140FFFFFFE0FFFF2B
:10878100FFFFC25030123F20283CE558F4603720EB
:108791004803200931D250E559F5103033066558A8
:1087A100600205101287CB12882775A7049006DC9A
:1087B100E512F0E511F0E517F0E510F075A704906A
:1087C10006E0ECF0EBF075A7002275A704758307AE
:1087D1001259F97813E0F608B819FA9006D0781111
:1087E100E6F008B819FAE51CF516F0E51BF515F0E9
:1087F1001288019006DAE514F0E513F075A700225E
:1088010075A704758306E51023541E24B0F582E094
:10881100F513E0F51422120D5EE5BD2487E5BD9246
:018821003B1B
:10882200500224912212881775F005A485F012F5E2
:1088320011E4F519FEF51CF51D12BDFBC23DC25631
:108842007F3C12CA34303D05751900807DDFF3E5A7
:10885200596558700A301007EE24D35002D2568C54
:108862001B8D1AE519FD24E250DEAE1CAF1D7C0003
:10887200125377EFF51924F650CEAC1BAD1A12C97C
:108882007920D1108E048F05E51975F0A7A4AEF0FA
:10889200FF125377AC12AB117AA01252A2EB33FB48
:1088A200EC33FC20D11AEF9BEE9C5014C3E512135B
:1088B200FCE51113FBC3EF9BEE9C4004AC06AB0737
:1088C200204807203B048C128B119006E2E519F038
:1088D20012890FAC16AB157AC8125279A912A811D7
:1088E20012541DED7005EC249E50057C807B0822FD
:1088F200C3E57A305602E55C9513FFE55E30560219
:10890200E55D9514FEC3EF9BFBEE9CFC22AE16AF19
:10891200157C00E519FD24F6501A1253777C007D70
:10892200061252577C007D051253778F10EEF51711
:0889320024E950037517FF2230
:10893A0012C98A12895712899A12D24A1289C020F8
:10894A004809128AAE128ADE028B4180747F177E32
:10895A002020480E748A204D101257BD500E742FD5
:10896A008007746A305F02746712D4DA75A70490BC
:10897A0006D07811E0F608B819FA7F177E00781247
:10898A00751905E60812D4DAEE2406FED519F42282
:10899A0075A7049006D8E0F516E0F515E0F514E0A1
:1089AA00F513E0F512E0F511E0F517E0F510E0FC3B
:1089BA00E0FB75A700227F187E26AC14AB1302D207
:1089CA00DC9006E4E0F51CA3E0F51B7F2A304E1389
:1089DA00120D54E5BF90A3B3B4010390A5AB127571
:1089EA00F880420F7E00745312D4A89005CBE0F8A9
:1089FA0030E705E53F30E0091F7E00E8540F12D446
:108A0A00C09004EEE0FEF51EA3E0FFF51F128A56A1
:108A1A00E51E24E9500C7E06742B12D4DA7E0C1261
:108A2A00D4DA128A86C20375172A751627125B844E
:108A3A00202415205F15D2037F2A7E1E908A743067
:108A4A004E03908A7D02D506205FEB227C007D3C96
:108A5A00125384A805EF7F2A7E0812D3E37E12748C
:108A6A003B12D4D67E14E802D3DD0707384C9EBAEF
:108A7A00F264380707387CE6C2E67C38AC1CAB1BCC
:108A8A007A48305D027A27125279A91EA81F125419
:108A9A001DED4C60027BFF7F207E28EB12D3E97E1E
:108AAA003902902E7F2B90A35C12763BE517F46077
:108ABA0022AE17AF107C007D3C125384A805EF7FCD
:108ACA002A7E0C12D3E37E16743B12D4D67E18E8A3
:108ADA0012D3DD22AE12AF117C007D0A125384A894
:108AEA0005EF7F207E3012D3E37E3A742C12D4DA5B
:108AFA007E3CE812D4C00F7E29744502D4A874853E
:108B0A008007748720560274867E2912D4DA3017B9
:108B1A0007742D7E3A12D4DA227C007D0A1253841D
:108B2A00A805EF7F2A7E3012D3E37E3A742C12D442
:108B3A00DA7E3CE802D4C0128C72E54824F650056D
:108B4A00128B2380B9E559046558600D128B2312E4
:108B5A008B08E559655860AA22A217923D8E1E8F8E
:108B6A00188515179006D0E0F511855810151012C2
:108B7A0044F7C3E51195105002F404F924A65005F0
:108B8A00C374B399F9E975F00584F924EE500279B2
:108B9A0011908CB2E993F5F012080DE5CC7004E956
:108BAA0030E702747F23A4A9F0E51B2517FDE51C15
:108BBA003516FEC3ED99F515EE9400F51675A70066
:108BCA00758306E55823541E24B0F582E0A3F513F5
:108BDA00E0F514128C72203D2C201729120D5EE547
:108BEA00BD2487E5BD5002249175F007A4FB9518B2
:108BFA00E5F0951E400FEB9FE5F09E4008EF9518B3
:108C0A00EE951E500EA23D9217AE1EAF18128B2380
:108C1A00028B08306B10128C0FE53F20E007748638
:108C2A007E2212D4DA2275A7009006E0E516F0A398
:108C3A00E515F0128B23128B0C74857E2312D4DA7D
:108C4A008558101287CB12895712899A8C168B1560
:108C5A001289C01288D51287BD12D24A9006E2E064
:108C6A00F51912890F028AAEC3E57A305602E55C1D
:108C7A009513FFE55E305602E55D9514FE92175096
:108C8A00031254EEAC16AB157AC8125279A906A88B
:108C9A000712541D7E037FE7ED700CEB2418EC34A9
:108CAA00FC4004AE04AF032200172E43576C809297
:108CBA00A4B6C5D3DFE6EDF3F8FD305E4F30504C75
:108CCA0075A7009006E0E0A3FCE0FBECA2E7921790
:108CDA00402024FE50047F3B8022AE04AF037C0078
:108CEA007D1412538474542F2017029F9FFF7462BD
:108CFA00800C1254FEEC24FE50E07F6D743D7E0021
:108D0A0012D4A87E017D197C03128D17227F3D1291
:108D1A00DE33EF2DFFDCF822E537B40206E5342412
:108D2A003750292212DEEE12D67D12CD52128EAEA5
:108D3A0012C7D412CF5F128F06125A4F7F207E2B92
:108D4A0012CE8C12D70F12DC481237EB12D17012E6
:108D5A008DDC12504D02DD1820041EE579FD24A099
:108D6A0050027D5FED24CD401E744520750C2DFF09
:108D7A00F512128DB11FBF44F922C39DFFF51212DD
:108D8A008DB10FBF46F92220750EED2413FFF5129F
:108D9A00128DB10FBF78F922C374779DFFF51212B5
:108DAA008DB11FBF12F922EF24BA40082433FCC345
:108DBA0074329C1404FC24D750047C238009EC23CD
:108DCA0075F005842413FC7E0512DE330EECB5061D
:108DDA00F822E59020E206E53424374003128D623A
:108DEA007F457E047D1212DE330EDDFA7F437E005C
:108DFA00746412D4A87F4F7D12128E977F3B7D1226
:108E0A00128E977F597D16128E977F317D16128E9C
:0F8E1A00977F637D1A128E977F277D1A128E978E
:108E29007F6D7D1E128E977F1D7D1E128E977E058A
:108E39007F1912DE330FBF72F97804E57924CD501A
:108E4900027809E8305C0123F87F1B128E867F6B5C
:108E5900128E8618305C01187F25128E867F61126A
:108E69008E8618305C01187F2F128E867F57128EDE
:108E79008618305C01187F39128E867F4D7E00E896
:108E890075F00A847004E802D495E802D430EF65DD
:108E990012600C7E04EE20E00712DE330EDDF622AE
:108EA90012DE6380F790A4717F287E2C12763D7EB6
:108EB9003B12D2F3AC5EAB7A7F307E19C23D12D33E
:108EC9003290A3607F5D7E2D12763D78B9C3E57A35
:108ED9009618FBE55E96FC7F507E19D23D02D3328F
:108EE900E51164B4700122E51112DCB87831790F0B
:108EF9007D0B12DDB61F1E908F9602D506E57160B7
:108F090012E57012DCB87831790F7D0412DDB20DEB
:108F1900BD0AF97F01128F6E7F1D128F6E7E23129B
:108F29008F787E3F128F787E247F17128F827E3949
:108F39007F02128F827E247F07128F8C7E397F1CDD
:108F4900128F8C7E317F0212DE337F1C12DE337F5B
:0F8F59000F7E2412DE337E3E12DE337F0C7E2E1F
:108F680090D7FB02D5067E2A12DE330EBE39F922CF
:108F78007F0812DE330FBF17F9227D0612DE330E8B
:108F88000FDDF9227D0612DE330E1FDDF922030301
:108F9800E0A0E012C98A7F18909C6B12763B7F2173
:108FA8007E01744112D4A87F2A7E01745312D4A87A
:108FB8009005BEE0F51AA3E0F519A3E0F51EA3E0BD
:108FC800F51D851A1C85191B75172012904BE5197C
:108FD800251DF51BF51DE51A351EF51CF51E751723
:108FE8002912904B9005BA12903BAC1AAB19751721
:108FF800201290099005BC12903BAC1EAB1D751752
:1090080029EC7006EB24CD4001227A48305D027AC3
:109018002712527912541DED4C600122AF177E07BA
:10902800EB12D38F7E1A0F90A534305D0390A537CD
:1090380002763DE0FEA3E0FD12BF51C3EB9DF8ECC4
:109048009EF922751627025BB512BF5175A70490C9
:1090580005B478737F06E6F008DFFBECF0EBF0E090
:10906800E0E0FCE0FDE0FEE0FFEF2DFFEE3C9005C8
:0D907800C0F0EFF0801275A7049005BAE07B
:10908500FBE0CBF0EBF0E0E0E4F0F075A700227533
:10909500A7049005B478647F06E0F608DFFB75A7A2
:0F90A50000125DC49005BEE51CF0A3E51BF02290
:10387D00D23C799E77008002C23C12BDFBE4F5106C
:10388D00F511F512F513F514F515F516F517C23DED
:10389D00123BCD203D1F123BCD203D19E51F30E5DC
:1038AD001130E40E1238F4303C08799EE724F550BF
:1038BD000122D510DBAE14AF157C00AD12125351A1
:1038CD008F55AE16AF177C00AD1312537712557886
:1038DD007E00E55530E7011E2DFFE43E30E7027F07
:1038ED0000740A2FF55622C235E51CAF1DBFFF052A
:1038FD000FD235F404FABF003F532CF8E518AF1979
:10390D00BFFF050FD262F404BF002D20E72A205B14
:10391D000123FF24AA4021E51AAE1BBEFF050ED2DE
:10392D0061F404BE00128547F0A4E5F020E70920FC
:10393D005B0123FE24AA5001227C807B80305166DE
:10394D00302163C006C0078AF0E545A4AEF0FFE55F
:10395D0056205B011375F009A4ACF0FD125377747A
:10396D00FFBE0001EFFA24C050027A3FD007D00607
:10397D00E55212DCB8303504B2D5B2D1EA8CF0A4E0
:10398D0030E70205F0748025F020D10495F095F014
:0A399D00FCEA8BF0A430E70205F00D
:1039A700748025F030D50495F095F0FBC3EC2F20FB
:1039B7006203C39F9FFFEB2E306103C39E9EFE20D1
:1039C7003C64200C05123A614064123A43405F128E
:1039D700DE33E51EFD24FB50550E12DE33ED24F6D3
:1039E700504C1E1F12DE33ED24F150421E0F12DE23
:1039F70033ED24EC50380F12DE33ED24E7502F1F40
:103A07001F0E0E12DE33ED24E250231E0F0F12DEBF
:103A170033ED24DD50180E12DE33ED24D8500F1E7F
:103A27001E1F1F02DE33123A434003799E0722E925
:103A3700242AFFE82461FE123A61401DEF2460400A
:103A470018243F5013EE2460400F243F500AEF2400
:103A5700D6FFEE249FFEC322D322532CF8432C0417
:103A6700EE10E706D2E7F404D261FE24D340EAEF72
:103A770010E706D2E7F404C262FF24D340DBEFB5B8
:103A870006005003CED26070057480FE8062FF246A
:0D3A9700FD5060903B4D938EF0A4AAF033DB
:103AA400CA33CA33CA33CA33CA33FA903B77938FC3
:103AB400F0A433C5F033CA903B9893FB123B1595A1
:103AC40070500224B412DCB8EA8BF0A430E702058B
:103AD400F0C3748095F020D50425F025F0FEEA8C1F
:103AE400F0A430E70205F0C3748095F030D10425CA
:103AF400F025F0FFC3227A01EE6F70097B16BF0236
:103B0400BB7A0380B7BF01047B0080B07B0D0A80C1
:103B1400ABE52C540723C3903B1F73800E800E80AB
:103B240024801E8010800A80108012EB22742D9B4A
:103B340022742D2B22745A9B22745A2B2274879B35
:103B44002274872B2274B39B22FFFFCCAA9280712C
:103B5400665D554E4944403C383533302E2C2A2876
:103B6400272524232221201F1E1D1C1B1A1A191865
:103B74001817178181818282838384858687898A45
:103B84008B8D8F90929496989B9D9FA2A4A7A9AC8D
:103B9400AFB1B4B400010203040405060708090A1E
:103BA4000A0B0C0D0D0E0F0F101111121313141418
:103BB400151516161612BD3312BBC1E4F5F7C2B2C1
:103BC400C2B2E5F7D2B264C022203D07123BB970FD
:103BD40003D23D22056D056D12BBC17D008DF7C278
:103BE400B2C2B285F71F8DF7C2B2C3E5F79573F57C
:103BF400188DF7C2B2C2B2E5F79574F5198DF7C204
:103C0400B2C2B2E5F78DF7C2B2C3E5F79576F51AFD
:023C14008DF72A
:103C1600C2B2C2B2E5F79577F51B8DF7C2B2C2B252
:103C2600E5F78DF7C2B2C2B2E5F7F51E8DF7C2B25F
:103C3600C3E5F7957AF51C8DF7C2B2C2B2E5F78DEA
:103C4600F7C2B2C2B2E5F7D2B2543F30E50244C081
:103C5600955EF51D156D156DE51024784001227EE3
:103C660000AF55EF30E7011E0512E51FA2E592D51C
:103C7600400EE515951EF515E5149400F514800B18
:103C8600E515251EF515E43514F5147800E51E60D6
:103C96000620D50318F404C39FF5F0E89E30E7012B
:103CA600220513E5F0A42517F517E5F03516F516E8
:103CB60022303D03D23D22123BB960F8123BB96077
:103CC600F3E546600A123BB960EA123BB960E505C6
:103CD6006D056D056D12BBC17D008DF7C2B2C3E5E2
:103CE600F79573F5188DF7C2B2C2B2E5F79574F57C
:103CF600198DF7C2B2C2B2E5F78DF7C2B2C3E5F7C6
:103D06009576F51A8DF7C2B2C2B2E5F79577F51B2F
:103D1600D2B2156D156D156D2230742412BDFBC21D
:103D26003D75101E123CB7203D167902123D8B40A0
:0A3D36000CA806A907123A36400354
:103D400012DE33D510E422200F4030123D2006CF82
:103D5000304806200C03204FC6E5467902601479EE
:103D60000614600F791614600A79361460057976A6
:103D700014701712BDFBC23D7896123CB7203D0A65
:103D8000123D8B400312DE33D8F022532CF8AB18CF
:103D9000E519FC339262123DDDBC002BEB89F05338
:103DA000F00784FF24DF401FAB1AE51BFC33926150
:103DB000123DDDAA471252A2BC000CEB89F053F071
:103DC0000784FE24DF5002D32274562F2062029F04
:103DD0009FFF741F2E3061029E9EFEC3225003126D
:103DE00054FEE920E40122C3EC13FCEB13FBE920B1
:103DF000E50122C3EC13FCEB13FBE920E60122C32F
:103E0000EC13FCEB13FB2274542F2062029F9FFFE4
:103E1000741D2E3061029E9EFE2279B4203249200C
:103E20001D46EFB506009260AC06AB074004AC0738
:103E3000AB06903E69EC2304938BF0A4A9F0EC232D
:033E4000938BF071
:103E4300A429F9903EC993C9903FC9E52C5407931F
:103E530013E95001F4903FD1F9E52C5407932975E8
:103E6300F0B484A9F022FFFFFFFF7FFF55553FFF0A
:103E730033332AAA24921FFF1C711999174515552C
:103E830013B1124911110FFF0F0F0E380D790CCC1E
:103E93000C300BA20B210AAA0A3D09D8097B09247D
:103EA30008D30888084207FF07C107870750071C84
:103EB30006EB06BC06900666063E061805F405D119
:103EC30005B0059005720000000000010101010129
:103ED30001010101020202020202020202030303C0
:103EE3000303030303030404040404040404040594
:103EF3000505050505050505060606060606060667
:103F0300060607070707070707070708080808083B
:103F13000808080808090909090909090909090A12
:103F23000A0A0A0A0A0A0A0A0A0B0B0B0B0B0B0BE7
:103F33000B0B0B0C0C0C0C0C0C0C0C0C0C0C0D0DBF
:103F43000D0D0D0D0D0D0D0D0D0E0E0E0E0E0E0E97
:103F53000E0E0E0E0F0F0F0F0F0F0F0F0F0F0F0F72
:103F6300101010101010101010101010101111114B
:103F73001111111111111111111112121212121228
:103F83001212121212121213131313131313131305
:103F930013131313131314141414141414141414E4
:103FA30014141414141515151515151515151515C3
:103FB30015151515151616161616161616161616A3
:103FC30016161616161600FFFF00FF0000FF002E40
:103FD300B5875B2D5A88E537607414603EB4025888
:103FE3007F347E12E5342437400810644B90A330AD
:103FF300801AF890412312D506E824FD501179A1C7
:10400300E77E0590A13B20E70390A1440F803A246B
:10401300040F7E2312D4C7D26480627F357E02E50B
:10402300342437401410641090A02A30081B1276F1
:104033000A7E1A90A32F801122700590A03C80095C
:10404300909C98200C03909CA312760A80C97F351C
:10405300E5342433402A2404501B7D0F600C7D1E5D
:104063001460077D3C1460027D78ED305D02C3135C
:104073007E2B12D38F7E0090A03D12760A02DD18AC
:104083007E0524FE5005909E808009909C7B200F26
:1040930003909C8712760A80E4E546604A14603CEC
:1040A30014602E14602014601290A568205D419066
:1040B300411C7F367E3412D506803C90A568305D66
:1040C3000390A564802A90A564305D0390A5608069
:1040D3001F90A560305D0390A55C801490A55C30B3
:1040E3005D0390A558800990A554305D0390A550B9
:0240F3007F3616
:1040F5007E3312763D7E3C7422305D02748302D499
:10410500DA305D0890A540305BE4800690A5482034
:104115005BDC90A54480D70508B28D8DB5BA091032
:1041250006000A10F248922492249224F2480A10BA
:104135000600305E5220434F20284CE55864FF604E
:1041450046E54824F640407F3FE55804F9C23D1254
:10415500418D12109B601AB404047401D23D75F0B0
:1041650003A4243CB5070A7E3A303D027E3612414F
:104175008F0F0F0FD9D7E55975F003A4243EFF1211
:10418500418D0F0F12418D227E3D12DE330EBE4052
:10419500F922C248C249305E56202853E55864FFCB
:1041A500604DE54824F6404712109B6042D249B461
:1041B5000402803B1465597036D248304E31E559BA
:1041C5006558602B3074281241FA120D54E5BFB4BE
:1041D500011DE5BD20E618202416205F129006E497
:1041E500E0700CA3E024CE40062425500205592298
:1041F500305FFC80E820113375A7009006E4E0707D
:1042050028A3E0302402F404305F02F4042404F906
:1042150024F74015E924FC4003D26C2270012230BA
:104225006C097536A7D22ED22FC26C22305E0830AB
:104235007405E558B4FF0122C244C24D780075A744
:0B4245000475830712457988188A1E53
:104250008E168F17C23EC23BE54824F65003024338
:104260000AD23EE55860F7E8655970F22048EF122F
:1042700043BF30D13BAE16AF17A818E546705512B4
:10428000080DE5CC49604DD244E5CC7033E924CD2E
:10429000402EE975F038A4ACF0FB12548D12548D09
:1042A000EBFDF511124320304D2CC206C23B80437A
:1042B000E546705C12080DE5CC7005E924CD505040
:1042C000124E8475A704758307A8181245798A1EB3
:1042D0008E168F178037120D54E5BDA2E0B3923BC6
:1042E0005011307428123A364026A907A806D20683
:1042F00012CA1B12433C12433312437C89078806BF
:104300001E1F90457412D506800630D10312435407
:10431000A81808C3E55898400302424375A7002235
:1043200074562F2062029F9FF9741F2E3061029EE7
:104330009EF822E51865586001227D057A00EA1290
:10434000DCB812DDB60A0AED24F240020A0AEA24B9
:104350004C50EB22AE16AF17123E071E303E021E27
:104360001EE51E12D4A8EE2404FEE51212D4A830D5
:084370003E09EE2404FEE513F2
:1043780012D4A822E5186558603CC001C000C012DC
:10438800C0138518101244F7D013D012D000D001F2
:10439800E510303B07C39570500224B412DCB820F6
:1043A8003B07AE16AF17124320E5112402FD7A062B
:1043B80012DDB61DDAFA2212109BB40457E87054C5
:1043C800120D72E5BD604D78C6A61308A61208A6A0
:1043D8002C12C7C875A7047583077510011259CA2E
:1043E80012C7C215101259CA1255E48E628F631291
:1043F800566C8B1C8A1B12C7CE20320E1244A72083
:104408003B08D24D12660712441D78C686130886EB
:104418001208862C22120D72AABD7C027BB312529E
:10442800A28C128B13AA1DA91F1252E4A91CA81B47
:1044380012541D8C1D8B1FAC12AB13AA19A91A128A
:1044480052E4A91CA81B12541D8C198B1AE56E2561
:104458001AF9E56D3519F8C3E56E951AFBE56D9502
:1044680019FAC3E554951FFDE56F951DFCE5542524
:104478001FFFE56F351DFEE52C23652C30E206ECA9
:10448800CEFCEDCFFD75A7049005C2E8F0E9F0EC8D
:07449800F0EDF0EAF0EBF09B
:10449F00EEF0EFF075A70022D23BC3E5649573C52C
:1044AF00659574F564E5669575600404600822E50A
:1044BF006424E0500822E5642420400122C3E5670C
:1044CF009576F567E5689577F566E56995786009FE
:1044DF0004600122E566F48002E5668562F0A4744B
:1044EF00E025F04002C23B2212C7C875A7047583AE
:1044FF00071259CA12C7C205101259CAC02C125935
:10450F00E3D02C891002C7CE30125120064E78000E
:10451F0075A70475830612457930D139123E07E528
:10452F004624FE500A0E0F90456F12D5068026EADC
:10453F007007745D12D4A4801C75F06484ADF070A4
:10454F000FED75F00A847008E5F00E12D495800512
:10455F001EED12D42A08C3E55A9850B475A700224D
:10456F00030340A040030340E040D2D1E8C4F582EA
:10457F00E0FA79731245D230D146AF06532CF8EDDD
:10458F00BFFF07F40460390FD262BF003312470632
:10459F00402E79761245D230D126E5822403F5825A
:1045AF00E0F512E0F513EEA2E713FEED13BEFF07E1
:0A45BF00F404600C0ED261BE000689
:1045C900124723400122C2D122C3E09709FDE09797
:1045D90009FEE097600904700AEE30E7068007EEED
:1045E90030E703C2D122E546600E14600BF9EDCE27
:1045F900A2E713CE13D9F8FD227C007B44E546607F
:10460900207C007BCC1460197C017B981460127C9F
:10461900037B3014600B7C067B601460047C0C7B8C
:10462900C08C148B157AE9125279A84712541B8C45
:10463900168B1775C70075C6047510DF75B901E5C6
:10464900BC20E76FF51385BD1205C605C675B9010E
:10465900532CF8C3E5BE9573FBE5BF9574FC05C6FD
:1046690075B901E5BC9575FD5005D262125506C3B1
:10467900E5159BE5149CE49D40338C198B18C3E523
:10468900BD9576FBE5BE9577FCE5BF9578FD5005B0
:10469900D261125506C3E5179BE5169CE49D400DB2
:1046A9008C1B8B1A1246CDE5322428401305C6E52A
:1046B900C68006E5C62404F5C6700205C7D51001F3
:0F46C90022024645AE19AD181245EFED12470615
:1046D800AE1BAD1A1245EFEE13ED13124723123E2F
:1046E80007E54624FB50080E0F90457402D5061EB8
:1046F800E51312D4A8EE2404FEE51202D4A875F03E
:10470800067FFDA946B9000575F0027FFF84C5F054
:104718002F500205F0C5F0FF24DE228547F0A430B3
:10472800E70205F0E5F0A946B9000280050475F036
:104738000384FE24E022E537B4020122E537700243
:10474800D23964027002C239E53724FC799EE760E9
:1047580005640B600C22D27E20081E401C107F10BE
:1047680022D27F2008134011107E012275370122C2
:104778007537002039037537022275F9FF75FB007C
:10478800800E75F9FF75FBFF801C2053F51247C09A
:10479800759E85759D2D80141247C0759E84759DE4
:1047A8002D80091247C0759E83759D09C2AC759806
:1047B80052C26DC26EC26F221215B1C253E4F5F92E
:1047C800F5FB30340215FB22D2A47F3212DE10C270
:1047D800A412D98F12DD1812DDF9C214C2151247BE
:1047E8008274C012DC4374A312DC00748F12DC00E4
:1047F80012481674C012DC4375A7049048207F1035
:10480800E49312DC00DFF912481675A70022E53898
:0548180012DC0074CA6F
:10481D0002DC00A29494859C8080808080818380BE
:10482D00819E8075A60A1247E2D269D2ACE5A62414
:10483D00FA500C306DF712DB95B4E0F1124878C2E6
:10484D00ACC26975A6FF22D21EC274C273E4FDF517
:10485D0071F570C22D124782D2AC12DB95C5F07086
:10486D0005DDF7C2AC22C5F0B4E0EFF538E4F53262
:10487D0012DB90A2E19273A2E2927475A7049004E8
:10488D00B4F012DB90C2D1124A5F20690330740B71
:10489D008D758E748F73E514C4F57D124ADF124A3F
:1048AD005F20690330740C8D788E778F76E5142533
:1048BD007DF57D124ADFD2D1124A5FEEF0F55DEF44
:1048CD00F0F55C207303E4FEFF79BCA70609A7078A
:1048DD0012DB907D0A124ACC8F71EE60037571FF69
:1048ED007D14124ACCC22DED24F150010F240A5033
:1048FD0002D22DBFB4027F008F7012DB90F05407EF
:10490D00C52E54F8252EF52EE571700EE4F571F5D2
:10491D0070C22D9004BFF0F0F0F012DB90E538601E
:10492D0009D21EC27412AE468005C21E12AE4212CC
:10493D00DB90B4E1FA75A7049004C412DB90F01279
:10494D00DB90F0F53A12DB90F0F53B12DB90F0F5D1
:0B495D003C12DB90F0F53D12DB90F007
:10496800F53E12DB90F0F53F12DB9012DB90B4E2DB
:10497800FA12DB90F07E0C12DB90FF12DB9012DB58
:104988009012DB9012DB9020E1027F00EFF012DB47
:1049980090DEE412DB90B4E3FA12DB90FF12DB90B6
:1049A800CF60027F7F9004E4EFF0E4F012DBC09068
:1049B80004D8124ACC12DB90B4EAFAC2AC75A70448
:1049C8009004DAE561F0E560F0E55EF0E57AF0E59F
:1049D80079F0E52EF0E55FF0E57BF0E551F0207425
:1049E80012E4F571F5709004B4F09004BDF0F0F0A5
:1049F800F0F0F075A70078ABA63A08A63B08A63CED
:104A0800120D68E5BF253D240C75F0188478AEA614
:104A1800F0186005640260182216E670121816E68F
:104A28007004760C181678ACE6904A529308F62271
:104A38000618E608904A52930466700D7601180627
:104A4800E6640D70047601180622001F1D1F1E1F44
:104A58001E1F1F1E1F1E1F12DB90FC12DB90FD1273
:104A6800DB90FE12DB90FFECA2E692E7921713FCB4
:084A7800ED92E713FDEE92E759
:104A800013FEEF92E7301701F4F513ECA2E713FCE5
:104A9000ED92E713FDEE92E7301701F4F512ECA268
:104AA000E713301701F4F510ED92E7301701F4F534
:104AB000111254AE20D10E8C1C8D1D8E1E8F1F1214
:104AC000B24E1254AE30170312B2282212DB90C33A
:104AD00013FEF012DB9092E7FFF07C00025384ACEF
:104AE0001CAD1DAE1EAF1F30170312B228ECF0ED47
:104AF000F0EEF0EFF022124AFF0202C612BC00C232
:104B0000101248337F5A7E0590A33F12760A12DDB9
:104B100018D214D215C255122C2F789F76800876A1
:104B20000012BC4012323D7570FE853A71853B72B1
:104B3000853C73853D74853E75853F7612BC9F121A
:104B4000323D7570C0757B03757A54E4F57FF57E50
:104B500012BC9F751421751348755F01757B007534
:104B6000750475745275780175776CE4F57DF551AF
:104B7000757F0190DF5C85836E85826DC23D124B2F
:104B8000DD851C1D75A6FF305505C221022DEA12D8
:104B90004BDDE572A2E59275A2E79277D274D273EB
:104BA000E51275F008A4AEF0FF2075031254EE1262
:104BB000C71812C761124C60E51C251D13F57185DD
:054BC0001C1D12BC18D1
:104BC50012BC70757F02E56A70B57F5A7E2FE5418C
:104BD50012D38F12DD1880A7856E83856D82C2552D
:104BE5007873124C417876124C41E493F570B4B465
:104BF50002D255A3E493F51CA3E493F512A3203D3B
:104C05000FA97BE493F57BC399502A20E702055F42
:104C1500A385836E85826D103D16D23DE582240500
:104C2500F582E43583F583E493F52654F0F5722295
:104C3500E526C480F630E7D8155F80D48601E49375
:104C4500F6A308C399500A20E70606B6000208062F
:104C55002230E70616B6FF0218162230750DE51349
:104C65002579F513E43514F514800DC3E51395790D
:104C7500F513E5149400F514AE14AF137C007D0A0A
:104C85001253848E5E8F7A22124D22851617203D8F
:104C950001227F5A909B8E1275F87F64E516640495
:104CA500700C909BA612763B12DD1802DDF3909BEB
:104CB5009A1275F87F6E7E0890A53012760A121D3D
:104CC5004612DD187515B87514047F6E7E20C22452
:104CD500A815E82404F9C23DE7124D6A203D06E611
:0A4CE50012D4DA8008E6128368E8B2
:104CEF00A815F60515EE2406FED514DA851716124B
:104CFF001D9412DD1810000510018D80F878B81280
:104D0F000D7C86BC0886BD0886BE0886BF124E2C59
:104D1F0012DEEE120D7CC23D75160078B87F4B7E09
:104D2F000890A53012760A7E20E5BC12D4DA124D17
:104D3F00617E26E5BD12D4DA124D617E2CE5BE12DE
:104D4F00D4DA124D617E32E5BF12D4DA124D610210
:104D5F00DD18F608080808F618181824D05005248E
:104D6F00F64001220516D23D2275C70375C6FE1205
:104D7F007576124E2C75C6FC75BC2675BD6475BE56
:104D8F00A975BF70124E2C75C6FB12757675BC6473
:104D9F00124E2C75C6FA75BC1475BD1475BE007510
:104DAF00BF0C124E2C75C6F975BC4E75BDBF75BEC6
:104DBF000075BF19124E2C75C6F875BC0A75BD7EED
:104DCF0075BE0075BF01124E2C75C6F775BC017507
:104DDF00BD2375BE4575BF67124E2C75C6F675BCE3
:104DEF000275BDAB75BE0175BF01124E2C75C6F5B0
:104DFF0012757675BE0275BF0A124E2C75C6F41267
:104E0F00757675BCE1124E2C75C6F3127572124E83
:104E1F002C15C6124E2C15C6124E2C15C675B9057B
:104E2F0075B90222751500127C6F75B901E5BC6466
:104E3F008160031275590515E515242050E975C7D2
:104E4F000375C68075B90505C6E5C6241C50F51255
:054E5F004E64027AC55B
:104E6400E4F5C7F5C6742612757775BD4E124E7EED
:104E7400124E7BE4124E7B127577124E2C05C6221D
:104E840020740122D24475A700758307E559C454E0
:104E9400F02407F582E0F51A244C40E7A3E0F5126C
:104EA400A3E0F51312080D8938120D54E5BDA2E0F4
:104EB400923BE51A40069570500224B4F51A203B43
:104EC40005D20612CA1BE51A124FE7E5152437F579
:104ED4001DE43514F51CE5172437F51FE43516F5E4
:104EE4001E85CC12853813AC12AB137A0412526BA4
:104EF40075380124FA401A05382402401405382470
:104F040001400E05380538240140060538053805EA
:104F140038C3E51A945A500224B4F51AC23BC23C71
:104F2400C23D751B00A23B823C406D203B2CE51A20
:104F340075F008A4951BFBE5F0303D049401800254
:104F44009400FC5008EB24A0FBEC3405FC124FEE5B
:104F5400124F9D923B4003124FC0203C2CE51A7522
:104F6400F008A4251BF9E4303D010435F0FAE99476
:104F7400A0FBEA9405FC5004AB01AC02124FEE1204
:0F4F84004F9D923C4003124FC0E51B2538F51B93
:104F93005094203D04D23D808D22E51F2517FEE568
:104FA3001E35167016EE24914011E51D2515FFE5FB
:104FB3001C35147006EF2491400122D3228E027C0B
:104FC3008A7B3B125279ED2402FE8F027C8A7B3B63
:104FD300125279ED2439FF02DE331255D780311294
:104FE30055CA804675F008A4ACF0FB751900C3EBF5
:104FF3009468F9EC9401FA40080519AC02AB0180FE
:10500300ED8C108B11531903E51920E0CD1255CA0D
:10501300125042AF05E51924FE50031254EE8E16CA
:105023008F17E51920E0B81255D7125042AF05E5A6
:10503300191460061460031254EE8E148F1522ACFB
:1050430006AB07AA12A9130252E412512F203D49BD
:1050530074857F227E0812D4DA7E0830173CAC1E9A
:10506300AB1FEB2418EC34FC402F12524AE51B60B3
:10507300077F207E0812D4F57F207E10E51A12D414
:10508300F57F237E17742E12D4D67F207E1BE51B5B
:105093007011E519C2E012D4F5227F207E0E740A46
:1050A30002D4F5E51975F0058475F005A402D4F56D
:1050B30012512F203D5E74857F227E3A12D4DA305E
:0450C3001753AC1EB5
:1050C700AB1FEB2418EC34FC4046EC7033EB249C0C
:1050D700402E7E2D12512112548DC0E07F2A7E2E44
:1050E700EB12D4F57E39D0E0C2E012D4F57F347EDE
:1050F7003712DE331E12DE331F12DE330E02DE33AB
:105107007E3012512112548DEB7F2A7E3112CFB19E
:10511700227F2A7E39740A02D4F57F2912DE630FB3
:10512700BF34F90EBE40F322D23D301266120D5E37
:10513700E5BDF51C75F00AA4F824E15002781EE4D9
:10514700FCFBFEFFC23D12BDFB12519B203D44D824
:10515700F8751DCEE51C146009751D9C1460037558
:105167001D6AC217EC30E705D2171254FE8C018B6B
:1051770000E9487003D23D22EE7008EF251D400379
:10518700D23D22AC06AB077A1C12527912541D8C01
:105197001E8B1F22203D07123BB97003D23D22050B
:1051A7006D12BBC1E4F5F7C2B2C2B2ADF7F5F7C2F3
:1051B700B2C2B2E5F7FAD2B230E4E3ED2FFFE43E34
:1051C700FEE56D2408F56D12BBC1E4F5F7C2B2C266
:1051D700B2ADF7D2B2EA30E508EB2DFBEC3400FCB8
:0A51E70022C3EB9DFBEC9400FC22B8
:0100030055A7
:10DF5C0069FC362E06FD69FC372F071169FD383038
:10DF6C0007FD69FD3931061169FE383107FD68FE80
:10DF7C003732091168FF373008FD68FF372D07115C
:10DF8C006800362909FE680036290C116801372B08
:10DF9C000CFF6801372F0A116802383009FF68023C
:10DFAC00372E08116803372C0AFE6803372E081128
:10DFBC006704373208FE67043633091167053535B7
:10DFCC0005FF6705353303116706362F02FF670619
:10DFDC00362B05116707362B07FF6707352F051101
:10DFEC006708353104FF6708332E0511670931289E
:10DFFC000700670931250A11670A35240B01670AE6
:10E00C003A240A11660A3C210801660B3D1E0B11CD
:10E01C00660B3D1E0C00660B3D200A11660C3B2165
:10E02C000CFF660C39220E11660C37231100660D9D
:10E03C0036240D11660D34260F01660E3226111191
:10E04C00660E32251401660F35251311660F37271E
:10E05C0016016610392918116610392B1502651135
:10E06C00392D11116511372E0C026512332F081141
:10E07C006512312F07026513302C0A1165132D29F7
:10E08C000E0265132A271011651429270E02651438
:10E09C002C290C1165153129080365153726071134
:10E0AC006515321F09036516411B09116516411CC4
:10E0BC0008036416461F081164164D2105046416E6
:10E0CC005922031164166425040563156A2407118B
:10E0DC0063156D23090663156C230D1163156C25EF
:10E0EC00130762146E2B151162146E2F1406621333
:10E0FC006E30161162136E30150761136F311211E9
:10E10C0061126F350F0761126F380D116011723A81
:10E11C000A086011763F0611601079420209600FFF
:10E12C007A3A0533600F7832040A5F0F742C01338E
:10E13C005F0E722B030A5F0E732E08115F0E743084
:10E14C00050C5F0D722C02135E0D6C2B010C5E0D19
:10E15C00622C05315E0D5F2B030D5D0D5E290833BE
:10E16C005D0D5F23030B5D0D5F1B01335D0D5A16B7
:10E17C00020A5D0D521B00115C0D4D26000C5C0E4D
:10E18C00462802335C0E3926040C5C0F2C2B08330A
:10E19C005C0F23320C0F5D0F172E0A335D0F0C2E04
:10E1AC0009105D0F043507335E0FB23C080F5F0F8B
:10E1BC00AB4209335F0EA43E070F5F0EA2430B3335
:10E1CC00600EA746120B600D9F490C73610C9C49A5
:10E1DC000F0C610B97460973610B8B440A0C610A97
:10E1EC008B420B336109843A080C6108823A043380
:10E1FC0061087934030C60086F2F063360086228BD
:10E20C00050C6008572505336008511F040D5F0885
:10E21C004E1B05335F08491B090D5F094120103760
:10E22C005F0938270D0D5F0A302F06335F0B2B3239
:10E23C00070F5F0B282F0A335F0B262E0E0E600C78
:10E24C0023361137600D1F3F160F600D18411277E2
:10E25C00610D0F320A13610D042B0633610D022E72
:10E26C00040E620D043A0231620E0343050D630D78
:10E27C00B1470113630DA94A000B640CA14D0511A4
:10E28C00640C9B44070E650B99490911650A944768
:10E29C00090D65098E49021365088848060D650845
:10E2AC0081400E336407793B130F6407722F187784
:10E2BC0064076D231A106407692911776407651CBC
:0DE2CC00080F63075D180B33630751190D30
:10E2D9000D630746220E336308402B110F6308387C
:10E2E900291837630932271B0D6309312B1477620B
:10E2F9000A372C0F0A620A3C280973620A441E0B6A
:10E309000C620A48150E33620B46190C0A620B4758
:10E31900260D33610B4C280C0B610B54251037610A
:10E329000B5E24170C600B63291A77600A66361492
:10E339000A600A68390B735F0A6C2C100A5F09724C
:10E349002015775F097422120A5F0873300F775F0F
:10E35900087639140A5F077D3816775F0785370F06
:10E36900095F068D3B0D735F058B4410075F048BB6
:10E37900490C735F048E3F0C075F03863604335FD5
:10E389000394280708600299300E1160029E400527
:10E39900076102A34A0C336101AA4810086201B15E
:10E3A90042127762020131150A6202062B13776362
:10E3B900020830110C63020B361277630310331114
:10E3C9000C6403182B147764032223110A640426AE
:10E3D90023107764042226110A64051C2715776423
:10E3E900051D251508640521271277640628270FBE
:10E3F9000764062F1D11776406350F140764063E5E
:10E409000A19776406401216086407431B117763DB
:10E41900074A22120663075228127763075A2713FD
:10E429000662075E2314776206612011076206649B
:10E439001E0E7362066A1E0E076206742110376289
:10E44900057828130661057A2F157761047A332038
:10E459000661047A301B7761037A281B0761037F01
:10E4690023187761028429160661028832177761B9
:10E47900018D371305610193340C7362009A2E09DB
:10E489000562009D2E043362009D370C0663FFA0D0
:10E4990040103763FFA844140564FFAF4612776440
:10E4A900FF014511056500043F12776500053E101F
:10E4B900076600073F117766000B430D07670110D8
:10E4C9003D117367011539120767021A321277670E
:10E4D900021A2C12076702192C107768031B2E0FDA
:10E4E9000668031F2C117768042729100468042E75
:10E4F9002A0F776705322F130467053330127767C0
:10E5090006362D140567063B291677670643231B34
:10E51900046706471E16776607491E150366074CEA
:10E529001B157766074C2217046607522214776574
:10E53900075B26150265066229157765066D291799
:10E549000165067529137765057D281A0265058217
:10E5590028187765047F1F160265048F2A117765CD
:10E5690003953211006602993D157766029C401C9D
:10E57900FF6602A13E1F776701A43F1CFF6701A741
:10E589004314776801AB4710FF6901B1490F7769F7
:10E5990001024911026A0207490D736A020B480C0C
:10E5A900056B030F480B336B03144A0D026B0419F7
:10E5B9004914376B051F491CFE6C06224824776CE9
:10E5C90006233F21FC6C07203023776C0721272184
:10E5D900FC6C07262420776C08292812FC6C082873
:10E5E9002C0F776C0927230CFF6C09251802316C55
:10E5F90009350F05FC6C094C1401116C09561D01F4
:10E60900FC6B095F2003136B086B2108FB6B087413
:10E619002509336B08772507FC6B0778210D336BC8
:10E62900077A1E0AFB6B077F220C336B06832E0ABF
:10E63900FA6B05853C09336B0489410EF96B048C2F
:0DE649003E10376B038D3C0FFA6B038D40C4
:10E6560013776B02904112FA6C01934110776C01AB
:10E66600984410F86C009B471A776D009F461EF879
:10E676006DFFA24519776EFFA14019F86EFFA640FF
:10E6860014776FFEAA4417FA6FFEAF4A127770FE30
:10E69600B34D18FA70FF024B1B7771FF054718FD43
:10E6A60071FF0942177772000E4012FD7200163D87
:10E6B6000C7372011B3510FA7201232E1577720244
:10E6C60029321AF872032C371D7772032F3014F88B
:10E6D600720336210F77710346190DF87103502026
:10E6E6000B33710353290EF87003572B143770033D
:10E6F600612712F870036F2911777002793017F7C6
:10E706007001803722777001843D1FF67000883FC4
:10E71600197770FF8D3F11F670FF933D0C7371FEF4
:10E72600973D0EF571FE9B3E0C3372FD9F4310F62E
:10E7360072FDA448127773FDAB4C13F573FDB14F10
:10E74600167774FD034F14F775FE074C127775FEA6
:10E756000A4510F975FE0E400F7776FF124111F843
:10E7660076001745167776001C4614F67601214288
:10E7760017777602263D17F3760229382177760336
:10E786002A3315F276032B3009737604302A07F004
:10E79600760439220A337604472110F07504512590
:10E7A60012777504552416F1750459210F777504EF
:10E7B6005F2111F0740463231477740468240EF245
:10E7C600740370230933740379270AEF74028030C7
:10E7D6000B33740185360DEF74018B3913377400D2
:10E7E600903D1BF075FF94441E7775FF984823EF04
:10E7F60075FE9B46207776FE9F4221F076FEA13F6E
:10E80600177777FDA44313EF77FDA747157778FDB4
:10E81600AA4915EF78FDAD4C157779FDB04D19EE87
:10E826007AFDB34D1C777AFD024E19F07BFD054F3C
:10E836001B777BFE094F24F37CFE0D531D777CFF6F
:10E84600114619F37CFF173F12777C001F3810EF33
:10E856007C00263613777C012B3115ED7C012F2B9E
:10E8660015777C02332513ED7C02392214777C025E
:10E87600402110EE7C0249210B737B02531F0FEBE4
:10E886007B02601E15777B026A2214EA7B017428DC
:10E8960019777B017B2D1AEA7B00833122777B0077
:10E8A6008A3320EB7BFF91371A777BFE953C1FEA74
:10E8B6007CFE983C26777CFEA74621EC7CFD9939A8
:10E8C60023777CFC9A3B1FEA7DFC9A3F1C777DFBF5
:10E8D6009A401EE87DFB9B3F20777EFA9B3F1FE612
:10E8E6007EFA9C431A777EF99E4717E57FF8A04A81
:10E8F6000E737FF8A34A0AEA80F8A548073380F822
:10E90600A94402EA81F8AE46041182F8B24C00E747
:10E9160082F80351021183F8085304EA83F90E4D75
:10E92600061183F914430CEC84FA1A400E1184FB89
:10E93600203F0AE884FC2540061384FC2B4008E6A9
:10E9460084FD3039073383FD36300EE483FE3C2BDD
:10E95600193783FE402A1EE783FE3D25187783FE7E
:10E96600371B16E783FF3114137783FF35170FE440
:10E9760083FF3E220D738200412C15E58200432C55
:10E986001A77820046251BE782004C201577810006
:10E99600552116E581005E2510778100682718E469
:10E9A60081FF72291E7780FF7A2E22E580FE7E3057
:10E9B600277780FE812B22E680FD85251C7780FD4A
:0DE9C600882618E281FC8A2F187781FC8DCD
:10E9D3003821E181FB903F287781FA924025E0813D
:10E9E300FA943D237782F9973C18E082F99A3F1510
:10E9F3007782F89E4412E083F8A347107783F8A741
:10EA03004A0CDF84F8AA4D133785F7AC5214E2851C
:10EA1300F7AF56107786F7B2580DE087F802560223
:10EA23003387F8055002E388F8094C051188F90C7F
:10EA33004E02E489F91052011189FA155004DF8955
:10EA4300FB1D45041389FB233304DE89FB292306BD
:10EA53003389FC2B1F05DE89FC2F23093389FD3302
:10EA6300280ADC89FD3B23103788FD471E0EDD880D
:10EA7300FD511E0E3388FD53200CDD88FD54210B00
:10EA83003387FD57200DDD87FD5C20093387FD5D4E
:10EA93002403DE87FD5B29013386FD592C04DE86C2
:10EAA300FD5D2C093385FD622F0CDC85FD652D0B87
:10EAB3003385FC672908DF85FC6722093385FC6BF6
:10EAC300210CDD84FC72280A3384FB783005DD8455
:10EAD300FA7C37073384FA7E390ADC84F9813B06F2
:10EAE3003384F8843F05DB84F8873F023384F78A55
:10EAF3003C04DB84F78D390A3384F6903908D985D1
:10EB0300F5923F113785F595430FD985F498440A5B
:10EB13007386F49B440AD986F39C440C3386F39C96
:10EB23004507DA87F29C47063387F19E4C0AD9885A
:10EB3300F1A251103788F1A65516D989F0A7571FAE
:10EB4300778AF0A9541BDA8AF0AA4D12778BF0ACBE
:10EB5300460DDB8BF0AC4906338CEFAB4D05DB8CFC
:10EB6300EFA95002318DEEA85209E28DEEA7530EA4
:10EB7300118EEEA75316E58EEDA44A20118FEDA05A
:10EB83004423E28FEC9C4821118FEB9A4A22E090B8
:10EB9300EB95411D1190EA8E391DDF90EA893621EC
:10EBA3001190E9873223E590E9852C2C118FE87DBC
:10EBB3002A26E08FE8762124118FE8662122E08F50
:10EBC300E856221F118EE947201DE08EE9392116F0
:10EBD300118EE9302518E28EEA2D2917118EEB30BC
:10EBE3003213E18EEB333711118EEC373C10E18E8B
:10EBF300ED393E07138DED3B4203DD8DEE3B3E09C0
:10EC0300338DEE3B310DDE8DEE392812378DEF3823
:10EC13002319DC8DEF382A18778DF0372A12DC8D13
:10EC2300F0382214778DF0361B0EDC8DF1361B0C79
:10EC3300338CF1371F0DDB8CF136250E378CF23414
:10EC4300270CDC8CF22A270D338DF31F2A0CDC8D65
:10EC5300F3173409338DF4143A08E48EF4123A0CA2
:10EC6300338EF4103D11EA8FF50E411A778FF50CB0
:10EC73004917EA90F50A50157790F5054F13E79178
:10EC8300F5B24F107792F5AD5408E492F4AB5A0104
:10EC93003393F4AB5C05E893F4A9500A3394F3A4DB
:10ECA300450CE094F3A041093394F29A3A05E295B6
:10ECB300F29734043395F1913208DC95F19E310DCE
:10ECC3003395F08A320CDA95F0872D0B3395EF806C
:10ECD300250EDE94EF73220C3394EF6C2412DD9433
:10ECE300EF6928157794EE6B2812DF93EE69280EEF
:10ECF3007393EE64270DDF93EE5C260B3392EE578E
:10ED0300270EDB92EE5828123792EE5E2610DB9226
:10ED1300EE64240D7391EE6C2108D991ED722304F6
:10ED23003391ED782904D991EC7C320A3391EB7F4E
:10ED33003A08D891EB833D093391EA883C0CD7918B
:0DED4300E98D3B103791E9903E12D792E820
:10ED50009143137792E794420ED792E7993E073397
:10ED600093E7A03901D993E7A63B0A1194E6A83F9F
:10ED70000CD794E6AB490E1195E6AE4F07D695E653
:10ED8000004D011396E6034601D996E6033E0811AD
:10ED900097E7043D0ED997E70740151198E70C4314
:10EDA00012DA98E812460F1198E918490CDA98E936
:10EDB0001D44081198EA243D05D898EB293A03111F
:10EDC00098EB2C3707D898EC2D38093398ED2E3D69
:10EDD0000ADC98ED2E3E0A3398EE2D3F0BDB98EFC0
:10EDE0002C420C3398F02B430ED998F02B3D113761
:10EDF00098F12D3710D898F130340D7398F23433E0
:10EE00000FD698F237330F7798F339331CD597F331
:10EE10003C32167797F43E2F11D797F440280973A8
:10EE200097F4422109D797F4461F0AB396F44B2171
:10EE300008D796F45325083396F45C2505D796F445
:10EE40006723023395F4722503D695F3782B0231AC
:10EE500095F37B3102D695F27E31063395F1832FFF
:10EE600004D695F18A2F023395F0913201D596F0B0
:10EE70009638061196EF9A3F02D497EF9D450213FC
:10EE800097EE9F4704D497EEA247073398EEA64427
:10EE900008D398EEAA430B3399EEAD440CD499EE07
:10EEA000B1400D339AEE013F11D39AEE054512772A
:10EEB0009BEE064A15D59BEE064712779CEF05425E
:10EEC00012D79CEF063E0F779DEF084111D39DEFBF
:10EED000094619779EF00B4718D39EF00D431C7717
:10EEE0009FF10F4015D69FF1114113779FF2134602
:10EEF0000ED9A0F2174A0B33A0F31C4A08D4A0F491
:10EF000023420333A0F42A3305D3A0F53127071198
:10EF1000A0F5382300D29FF53D2702339FF6442900
:10EF200003D39FF64F2808119EF55E2807D19EF562
:10EF30006C2D04119EF4752F01D09EF47C2D0433AA
:10EF40009EF3822B04D09EF3872E05119EF28B3503
:10EF500007D09EF2903D01119FF1954203D09FF0A2
:10EF600094400333A0F09F3F0BD0A0F0A13D0F379A
:10EF7000A0EFA33C0DD1A1EFA43C0C33A1EFA43C26
:10EF80000AD0A1EEA53D0533A2EEA63C00D1A2EE2B
:10EF9000A8390211A3EEAA3C04D0A3EEAD3F05119F
:10EFA000A4EEB24008D0A4EE03410C11A5EE064138
:10EFB0000AD2A5EE08450711A6EF094A05D2A6EF29
:10EFC000094C0111A7EF0A4807D3A7F00B420B1118
:10EFD000A8F00B420DD4A8F00D461311A9F111466B
:10EFE00014D9A9F1173F1B11A9F21E381ADAA9F397
:10EFF00021381811A9F31F3A17DFA9F41839151190
:10F00000AAF4163A1DDCAAF5183C1A11AAF51C3A06
:10F010001AD9AAF61F391A11ABF6203615D9ABF753
:10F0200021341711ABF8203B19D9ABF81E3F17114B
:10F03000ACF91D4011D9ACF91E3F0E11ACFA1F40BE
:10F040000CD6ACFB22410D11ACFC23450FD6ADFC18
:10F0500023490B11ADFD214A0DD6ADFE2047091104
:10F06000ADFE21450CD6ADFF22430E11AE00224568
:10F070000CD8AE01214B0A11AE0220500DD7AF03C0
:10F080001D4F0B11AF031A5109D9AF04174A0D11C7
:10F09000B00418470BDBB0051A500A11B0061C5516
:10F0A0000ED7B1071C560B11B10719470ED9B1087D
:10F0B000173C0C11B208183D0CDCB2091C490E11AA
:0DF0C000B20A1E4E0AD9B30B1D500B11B33E
:10F0CD000C1A5109D9B30C174F0711B40D17490B71
:10F0DD00DBB40D17480D11B50E19490ADCB50F1922
:10F0ED004F0B11B50F185605DBB61017550711B696
:10F0FD0011174C0ADBB61116430B11B711173F0D43
:10F10D00DDB71219430C11B7131A480BDCB8131ADB
:10F11D00450F11B81419410DDCB81418400B11B975
:10F12D001518430DDBB91618470F11B91618490DEF
:10F13D00DBBA1718470A11BA1717450CDBBB1814A1
:10F14D00460F11BB18134C0EDBBC1912510A11BC22
:10F15D001A125007DBBC1A12470B11BD1A10400DC5
:10F16D00DCBD1B10400A11BE1B124509DCBE1C156F
:10F17D00490B11BE1D184A0ADBBF1D1B4A0811BFE2
:10F18D001E1B480CDBBF1F1A470E11BF1F1A490B60
:10F19D00DBC0201B4B0D11C0211C4910DBC0211DF4
:10F1AD00470F11C1221D4711DBC1231C4B0F11C18C
:10F1BD00231B4B0EDBC22419441111C224193D0F20
:10F1CD00DBC2251B3B1011C2261D3F0DDAC2261EC8
:10F1DD00411011C3271D3F12DAC3271C3D0F11C368
:10F1ED00281B3D10DBC4291C401111C4291C450FDF
:10F1FD00DCC42A1C460E11C42A1B4510DCC52B1974
:10F20D00431111C52C184511DDC62C164A1011C617
:10F21D002D174A11DEC62D18491211C72E19471088
:10F22D00DEC72F1A460E11C72F1C4410DFC7301F23
:10F23D00471111C731214B0CDBC832224D0E11C8BD
:10F24D0032224A10DAC83321471111C83420460F33
:10F25D00D9C83520461111C93521430CDBC93623D8
:10F26D003F0F11C937253D11DBC93725400E11C997
:10F27D0038254211DCC93925431311C939254312EB
:10F28D00DCC93A25431111CA3B24400DDCCA3C248C
:10F29D00411011CA3C23400EDCCA3D22401111CA57
:10F2AD003E20420FDECB3E20451011CB3F204714B0
:10F2BD00DECB4021441211CB40213F10DFCB412248
:10F2CD003C0D11CB42234011DFCC42233E1111CC1A
:10F2DD0043202F0EE0CC4319221211CC43122011E2
:10F2ED00E3CC4311250E11CD43132B10E3CD441266
:10F2FD002D1111CD440F2B0FE3CD44092B1211CE3F
:10F30D004404320FE2CE4401360E11CF44B3370D13
:10F31D00E0CF44B3330E11D04401370EE0D0440595
:10F32D003D0D11D0450A3B0CE3D14512330D11D1E2
:10F33D00451A2D0EE3D1461E2B0F11D1461D2E0F52
:10F34D00E4D1471D300F11D1471E320EE3D24821B3
:10F35D00330F11D248233510E2D24923350F11D284
:10F36D004A20360EE3D24A1D360E11D24B1B3410F5
:10F37D00E3D34B1B320F11D34B1B300EE4D34C1B7D
:10F38D00340D11D34C1B3A0DE5D44D1A3B0E11D44F
:10F39D004D1B360AE6D44E1D340E11D44E1E360DBD
:10F3AD00E5D44F1F360C11D5501F350EE5D5501F26
:10F3BD00340D11D5511E340EE5D5511E370C11D516
:10F3CD00521E390EE5D652203B0F11D653223C0F5B
:10F3DD00E4D65423391111D654243710E3D65524CD
:10F3ED00360F11D655253310E3D65626330D11D6CB
:10F3FD005627350BE2D657273A0C11D658273C0F16
:10F40D00E2D75827391011D75927370FE2D75A2786
:10F41D00381011D75A283B0FE2D75B293C1111D771
:10F42D005C2B3C12E2D75C2D391111D75D2C3910B4
:0DF43D00E3D75E2B3C0F11D75E293B0EE399
:10F44A00D75F27371011D75F26360EE3D760273CE0
:10F45A000E11D761284310E3D76229451111D762EB
:10F46A00293F0FE4D763283A1011D763293A11E4E8
:10F47A00D7642A3E1011D7652C4211E4D7662E4272
:10F48A001011D7662D3F11E4D7672F3A1011D768AC
:10F49A002D3B0CE4D7682E3D0711D7692E4204E4B0
:10F4AA00D76A2E470111D76B2E4702E4D76B2D403E
:10F4BA000513D76C2B3503E4D76C2A2B0711D76DAC
:10F4CA002B2909E5D76D2B300611D76E2A3A04E4A9
:10F4DA00D76F28400611D76F283E08E4D77027381F
:10F4EA000C11D87026320DE6D871252F0911D87162
:10F4FA0024310AE9D87221340811D8721B3A08EA71
:10F50A00D9730D420A11D973104909EADA730C4505
:10F51A000811DA730A3B06E8DB74093D0211DB7451
:10F52A000A4003E9DB740B3C0213DC75103406EA6B
:10F53A00DC7517350333DC761A3F06EADD771C469D
:10F54A000433DD771F4001E8DD7824360731DD78A2
:10F55A002C3206E7DC7933320413DC79373409E7D5
:10F56A00DC7A3A340C33DC7A3C3508E7DC7B3D370D
:10F57A000233DB7C3C3A05E7DB7C3C3D0333DB7D35
:10F58A003B3A04E7DB7D3B320331DA7D3E2D09EA63
:10F59A00DA7E43270D11DA7E4D230AE9DA7E5726F1
:10F5AA000B11D97D5E2C0BE9D97D61300C11D97D07
:10F5BA00632F08EAD87D662F0511D87C683005EAE2
:10F5CA00D87C6D330611D77B733608E9D77B7C3834
:10F5DA000511D77A853A04E8D8798B3B0711D8798F
:10F5EA008E3809E9D8788F371011D878903B0BE814
:10F5FA00D87791420D11D976954A08E7D976984974
:10F60A000411D9759D4008E8DA75A23A0B33DA7508
:10F61A00A53C0AE8DB75A8430031DB74AA4603E976
:10F62A00DC74AF460213DC74004A02EADD75054C4D
:10F63A000333DD75084D00EDDE75084B0533DF76C3
:10F64A00064902EDDF76044A0131E076044902EA0E
:10F65A00E076044C0513E176045006EAE176014DA2
:10F66A000D33E276B1450FEAE276AD3F1077E375E6
:10F67A00AB3F0DEAE375AC430A33E475AE4604EAE0
:10F68A00E475B0400131E575B23908EAE575013C27
:10F69A000611E675054607ECE6760A4B0311E7768E
:10F6AA000F4604EEE777163B0611E778203405EC9F
:10F6BA00E77827350611E7792D3409ECE7793234F2
:10F6CA000B11E77A3B260AECE67A45250B11E67A16
:10F6DA004D230BEAE67A56250711E67A5F270AEAEE
:10F6EA00E579672A0C11E579731F0AEBE578792E1B
:10F6FA000811E578843302EAE5778D3B0313E67651
:10F70A00954104EAE676993F0733E6759A3801EAA5
:10F71A00E67595310531E6748F3202EAE6748E3564
:10F72A000111E773923301EAE77398310413E77220
:0AF73A009D3304EBE872B4370911A7
:00000001FF
